:020000040800F2
:1080000000800120BD770108592001085B2001088C
:108010005D2001085F2001086120010800000000C8
:1080200000000000000000000000000063200108C4
:10803000652001080000000067200108DD810008BC
:108040000978010809780108097801080978010808
:1080500009780108097801080978010809780108F8
:1080600009780108097801080978010809780108E8
:1080700009780108097801080978010809780108D8
:10808000097801080978010809780108D5920008E3
:108090006D9100082192000809780108898D000877
:1080A00009780108097801080978010809780108A8
:1080B0000B0301080978010809780108097801080B
:1080C000097801080978010809780108E5F5000830
:1080D0000978010809780108F98F00080978010872
:1080E0000978010809780108097801080978010868
:1080F0000978010809780108DDF600080978010807
:108100000978010809780108097801080978010847
:108110000978010809780108097801080978010837
:108120000978010809780108097801080978010827
:108130000978010809780108097801080978010817
:10814000097801080978010809780108F3AC0008EA
:1081500009780108097801080978010809780108F7
:1081600009780108097801080978010809780108E7
:1081700009780108097801080978010809780108D7
:048180000978010871
:1081880010B5054C237833B9044B13B10448AFF349
:1081980000800123237010BDC005002000000000EE
:1081A8005098010808B5064B1BB106480649AFF3BD
:1081B80000800648036813B1054B03B1984708BD12
:1081C8000000000050980108C4050020BC050020EC
:1081D80000000000684620F007018D4601B5124BEB
:1081E80019781A4679B15B68013353600F4B1968E7
:1081F800013119600E4B196811B1196801391960FC
:108208000023137001E001221A700A4B1A683AB170
:108218001A68013A1A601B6813B9074B01221A70D1
:10822800BDE8014085467047DC050020D8300120B4
:10823800782801207C28012080280120074B41F65E
:108248004B525A60064AF02182F8231000229A60A5
:1082580007221A606FF004000CF096BB10E000E0F3
:1082680000ED00E0014B5868704700BFDC050020B6
:108278002DE9F341694F01200146002402250BF046
:108288000BF9384609236946012600938DF8044006
:108298008DF806408DF807408DF805500AF050FF1C
:1082A800384648F21603694600938DF806408DF863
:1082B80007408DF804608DF805500AF041FF48F238
:1082C80011033B8306237B8338464FF4807369464A
:1082D80000938DF806408DF807408DF804508DF80E
:1082E80005500AF02DFF21464FF4800007F58067FE
:1082F8000BF02AF8284631460BF0CEF840F6FC730E
:108308003846694600938DF804408DF806408DF88C
:1083180007404FF480588DF805500AF011FF384691
:108328006946CDF800808DF806408DF807408DF835
:1083380004608DF805500AF003FFA7F8188031464D
:1083480007F5806704200BF0A7F838464AF2C233D5
:10835800694600938DF804408DF806408DF8074073
:108368008DF805500AF0ECFE384644F204036946DD
:1083780000938DF806408DF807408DF804608DF85D
:1083880005500AF0DDFE4FF480433B8304237B83D2
:10839800314607F5806708200BF07EF84FF68C739E
:1083A8003846694600934FF010088DF804408DF860
:1083B80006408DF807408DF805500AF0C1FE384692
:1083C80069468DF806408DF80740CDF800808DF895
:1083D80004608DF805500AF0B3FE40463146A7F810
:1083E8001A800BF059F88DF806408DF8074004F113
:1083F800804404F504344FF6FF7320466946009321
:108408008DF804608DF805500AF09AFE4FF6107347
:108418006383EF23238302B0BDE8F08100000240AC
:10842800C90802F099B907281ED8DFE800F0040748
:108438000A0D101316194FF4807213E04FF40072EE
:1084480010E04FF480620DE04FF400620AE04FF450
:10845800805207E04FF4005204E04FF4804201E0FC
:108468004FF40042014B5A83704700BF001002408E
:1084780007281ED8DFE800F004070A0D10131619A4
:108488004FF4807213E04FF4007210E04FF48062F2
:108498000DE04FF400620AE04FF4805207E04FF419
:1084A800005204E04FF4804201E04FF40042014BD7
:1084B8001A8370470010024038B50546002445FA73
:1084C80004F3DB07E0B202D5FFF7D2FF01E0FFF7C4
:1084D800AAFF0134082CF2D138BD08B507282ED8D8
:1084E800DFE800F004060B10151E232800200FE01B
:1084F800144B1869C0F3802008BD124B1869C0F3EB
:10850800C02008BD0F4B1869C0F3003008BD01201A
:1085180001F0AAFAB0F5006F34BF0020012008BDB1
:10852800084B1869C0F3403008BD064B1869C0F302
:10853800803008BD034B1869C0F3C03008BD002067
:1085480008BD00BF000C024007282DD8DFE800F066
:1085580004090E13181D2227144B5869C0F3002074
:108568007047124B5869C0F3402070470F4B586949
:10857800C0F3802070470D4B5869C0F3C020704786
:108588000A4B5869C0F300307047084B5869C0F36C
:1085980040307047054B5869C0F380307047034B33
:1085A8005869C0F3C030704700207047001002407F
:1085B800144B58695A69C0F3002091055A6944BFA1
:1085C80040F00200C0B252055A6948BF40F00400AA
:1085D80011055A6948BF40F00800D2045A6948BFDB
:1085E80040F0100091045A695B6948BF40F02000D0
:1085F800520448BF40F040001B0448BF40F08000D0
:10860800704700BF00100240034B202208B15A8374
:1086180070471A83704700BF0010024008B5082051
:1086280001F022FA592804D9064B1A784AB90122CE
:1086380006E0082001F018FA542802D8014B00225D
:108648001A7008BDE4050020044B18780138C0B240
:1086580001288CBF00200120704700BFE4050020DE
:10866800044B1878012802D102221A7070470020A2
:10867800704700BFE405002020B9034B1869C0F318
:1086880040207047002070470004024008B588B9B0
:10869800094B1A78094B2AB9D3E90023100C40EA90
:1086A800034008BDD3E9000142F2107200230EF026
:1086B8009BFD08BD002008BD75280120D029012098
:1086C80010B9024B1868704700207047B82901207C
:1086D800F0B50D4618BB72B6114B124C19782A46E4
:1086E800EB17114EC4E9002331B9D4E900010B049A
:1086F80043EA1043020407E042F21077D4E900018C
:10870800A0FB072307FB0133C4E90023074A002322
:1087180035601360064A1360064A536262B6F0BDBC
:1087280075280120D0290120B8290120A429012079
:10873800FC29012000040140024B1869C0F3002005
:10874800704700BF0008024010B580B9084A094BBD
:1087580012781960084C18681AB10EF05BFB0749CB
:1087680002E00EF057FB06490EF05CFC206010BDDD
:1087780075280120C82901207028012000401C46C6
:1087880000FF7F4738B5044648BB01F04403042B7B
:108798001C4B9A680BD1C80602D542F4807208E0D7
:1087A80022F480729A60DA6842F4807205E022F45A
:1087B80080729A60DA6822F48072DA6001F0080246
:1087C80002F0FF00104B12B101221A7000E018707D
:1087D80011F001010D4B1ABF01221A7019700C4BD0
:1087E8000C4D1A5D0C4B18681AB10EF013FB0B49AF
:1087F80002E00EF00FFB0A490EF014FC45F82400C5
:1088080038BD00BF003C0140742801206C280120BD
:108818007528012070280120C829012000401C4625
:1088280000FF7F47014B1954704700BF60280120A3
:10883800194B70B553F82050044607F0CBF905FAE8
:1088480000F0164B164D53F8243090FBF3F203FB5F
:108858001200060496FBF3F103FB11664EB10121E9
:10886800295542F21075684390FBF3F305FB02317A
:1088780002E001EB02412E550A4B21F07F4003EB49
:1088880044131A6902F07F4202431A612046BDE888
:108898007040FFF759BF00BF6828012064280120F5
:1088A80075280120DC29012070B5514D8CB00024B9
:1088B800C0230226284602A902938DF80C608DF881
:1088C8000E408DF80D608DF80F400AF039FC2846EF
:1088D800062103220AF0B1FC032228460721A5F548
:1088E80082350AF0AAFC012130460AF005FE284626
:1088F8000BF0CAF809A80BF0AFF94FF6FF7328463A
:1089080009A90A93ADF82440ADF82C40ADF82640EB
:108918000BF064F922462346284603210BF0D9FDC3
:1089280006A80BF00EFC284606A9ADF820400BF06F
:108938007FFC06A92846ADF818400BF079FC06A87C
:108948000BF0FFFB284606A9ADF820400BF070FCA1
:108958000423284606A9ADF818300BF069FC284610
:1089680041F65F610BF011FD6C62284601210BF0A6
:10897800CAF9082130460BF029F84FF480730493A4
:108988000125082304A88DF815308DF816508DF8A8
:1089980014400AF0FDFA174B01A89A6822F4807275
:1089A8009A60DA6822F48072DA608DF80750124D06
:1089B80017238DF804308DF805408DF806400BF02C
:1089C80097FF2969204621F07F41FFF7BDFE204629
:1089D800E97CFFF7D7FE094BC8221A60084B4FF411
:1089E800004220461A60FFF723FF0CB070BD00BF9D
:1089F80000080240003C0140DC29012068280120D1
:108A0800642801202DE9F0433E4B3F4C1A783F4B38
:108A18005B6A0AB1C3F580333D49236022680B685D
:108A280039489A4202680B682EDDD31A394EB3F5DD
:108A3800004F394F394DD6E900230DDAD0F80090B0
:108A4800D1F80080D7F800C0C8EB09070CFB07F77E
:108A5800D21943EBE77331E0D1F80090D0F80080E9
:108A6800D7F800C0C8EB090707F580370CFB07F7F4
:108A7800D21B63EBE773C6E900232A6800680B681A
:108A8800C31AA3F5803337E09A4237DA0A680368D5
:108A9800204ED31AB3F5004F1F4F204DD6E90023BF
:108AA80013DAD1F80090D0F80080D7F800C0C8EBEE
:108AB80009070CFB07F7D21B63EBE773C6E9002332
:108AC8002A6800680B68C31A16E0D0F80090D1F83D
:108AD8000080D7F800C0C8EB090707F580370CFB02
:108AE80007F7D21943EBE773C6E900232A68006841
:108AF8000B68C31A03F5803313442B6023680B609B
:108B0800BDE8F0836C280120A4290120000401405D
:108B1800FC290120D0290120C8290120B8290120D9
:108B2800164B10B55A6A164B5A6059689A689142A2
:108B380059689A680CDD8A1AB2F5004F114A106814
:108B48005C689968C1EB0401A8BFA1F580310FE00A
:108B580091420FDA99685A688A1AB2F5004F094AA1
:108B680010685C689968C1EB0401A8BF01F5803101
:108B7800014411605A689A6010BD00BF00080040A7
:108B8800E40500205C280120044B054A18600023F6
:108B98005362044A93605360704700BF5C28012009
:108BA80000080040E40500200C4B1A6912F0040F7D
:108BB8001A690CBF082000201B6911075CBF40F030
:108BC8000400C0B21A06054B58BF40F002001B69EA
:108BD800DB0558BF40F00100704700BF000C0240A1
:108BE800034B08B1034A00E0034ADA60704700BF4C
:108BF80000ED00E00400FA050100FA0500239A00E0
:108C080002F16042013302F561424FF0FF31082B57
:108C1800C2F88010C2F88011F1D1002303F160423C
:108C2800013302F561420021F02B82F80013F5D1DF
:108C38007047074B02225A83064A042313834CF2D7
:108C4800503300BF013BFCD104235383704700BF5E
:108C58000000024000080240064B04225A83064ADC
:108C6800022313834CF2503300BF013BFCD1022393
:108C780053837047000802400000024028B9044BA3
:108C8800186900F00800C0B270470020704700BFA4
:108C980000000240F0B589B000285CD0354E0024B1
:108CA80080230225304601A901938DF808508DF8DC
:108CB80009508DF80A408DF80B400AF041FA2A460F
:108CC800072130460AF0B9FA20232B4D01270393D8
:108CD80003A808238DF811308DF810408DF8127014
:108CE8000AF056F9394604200AF0FAFB28460AF039
:108CF800CBFE05A80AF0B0FF4FF6FF73284605A97A
:108D08000693ADF81440ADF81C40ADF816400AF0D3
:108D180065FF22462346284660210BF076FB28464D
:108D280041F65F610BF031FB144B6C622846394603
:108D38009C605C600AF0E7FF336913F0200F2B8812
:108D480003D09BB243F0100303E023F010031B048D
:108D58001B0C2B800BE0202303938DF810000823B5
:108D68008DF8120003A88DF811300AF011F909B036
:108D7800F0BD00BF0004024000080040E4050020E8
:108D8800684620F007018D4619B54FF480700AF047
:108D980057F910B34FF480700AF060F91C4C0020AA
:108DA800FFF730FE002007F08DF9237823B100206B
:108DB80006F074FF00232370164B1B786BB9164B13
:108DC8009A6822F480729A60DA6822F48072DA6013
:108DD800124B1A6922F080621A6120200AF030F9D9
:108DE80090B120200AF03AF90D4B0E4A1B6913F096
:108DF800200F138803D09BB243F0100303E023F045
:108E080010031B041B0C1380BDE8194085467047EE
:108E18006028012074280120003C0140DC29012041
:108E28000004024000080040014B53F8200070473E
:108E380064280120014B53F820007047682801205E
:108E4800024B43F82010FFF7F3BC00BF6428012051
:108E5800024B43F82010FFF7EBBC00BF6828012045
:108E6800C0B201F0A7BDC0B201F096BD704770470F
:108E7800704700BF70B5064688B058480BF056FBDF
:108E88004FF4003001210AF02BFB082001210AF0E1
:108E980003FB022500242023514802A902938DF8E0
:108EA8000C508DF80E408DF80D508DF80F400AF0DB
:108EB80047F940234A4802A902938DF80C508DF8CF
:108EC8000E408DF80D508DF80F400AF039F94448DE
:108ED800052107220AF0B1F94148062107220AF0C4
:108EE800ACF904A80BF0CEFB0B2E25D8DFE806F072
:108EF8002406090C0F1215181B1E20224FF461536B
:108F08001CE04FF4964319E04FF4E14316E04FF4A8
:108F1800164313E04FF4614310E04FF496330DE02D
:108F28004FF4E1330AE04FF4613307E02D4B05E0DD
:108F38002D4B03E02D4B01E04FF4165304A92748AD
:108F480004930BF047FB2623002401258DF80430F9
:108F580001A806238DF805308DF806408DF80750D6
:108F68000BF0C6FC1D4840F2FF310BF08BFC22468B
:108F78001A4828210BF068FC2A46184840F2277145
:108F88000BF062FC2A46154840F226610BF05CFCA7
:108F98002A46124840F225510BF056FC22460F484B
:108FA80040F224410BF050FC22460C4840F64601A2
:108FB8000BF04AFC2246094840F66A110BF044FCC3
:108FC8002246064860210BF03FFC054B10225A83CD
:108FD800024829460BF077FB08B070BD00440040FA
:108FE800000C024090D0030020A1070040420F006F
:108FF800684620F007018D46294919B50B889C065B
:109008001AD5284B5B69D80601D58B8814E0264B06
:109018001A6858680132202A08BF0022824205D007
:109028001C6888881919C0B208721A601F4A0A2178
:1090380011609A6A1E4B1A60194803881A061BD5D4
:109048001B4B1A68C2B9184BDC6A196B8C420FD0DB
:10905800144910240C83196B4C1C1C63194491F897
:109068003410C9B28180196B202905D11A6303E035
:1090780040F227710BF0E8FB094803885B060BD523
:1090880040F226610BF022FC074B1A6BDB6A9A420E
:1090980002D1044B10225A83BDE819408546704717
:1090A80000440040000C0240F00500207C2801200C
:1090B800782801200A4BDA6A196B0132202A08BF86
:1090C80000228A420AD0D96A194481F83400DA6247
:1090D800044840F2277101220BF0B6BB704700BF6D
:1090E800F0050020004400400A4B59681A68914274
:1090F8000BD05A68511C59601A44127A02705A6887
:10910800202A04D100225A6001E000207047012083
:10911800704700BFF0050020014B9862704700BF00
:10912800F0050020044B1A7802F0FF0012B100226B
:109138001A700120704700BF8028012072B6034BC7
:1091480000225A601A6062B6704700BFF00500201E
:1091580010B5441E14F8010F10B1FFF7ABFFF9E783
:1091680010BD00BF684620F007018D4631B5264C7A
:10917800264B25681B680135082D08BF00259D4230
:1091880086B023484FF0000137D001AA09F0B5FB9B
:109198009DF80C302268042B1E4B03EB021206D1FB
:1091A800012151702168029A03EB011105E00021A9
:1091B80051702168019A03EB01114A609DF80D2056
:1091C800022A226808BF012103EB021218BF0021FE
:1091D800917022689DF80E1012019954002221689E
:1091E80001A8104403EB01111144C07A0132082A86
:1091F8000872F4D1044B1D6001E009F0C7FB06B00A
:10920800BDE8314085467047102901208428012097
:109218000064004090280120684620F007018D4630
:1092280031B5264C264B25681B680135082D08BF2B
:1092380000259D4286B023484FF0010137D001AA8E
:1092480009F05BFB9DF80C302268042B1E4B03EBE6
:10925800021206D1012151702168029A03EB011113
:1092680005E0002151702168019A03EB01114A6061
:109278009DF80D20022A226808BF012103EB021283
:1092880018BF0021917022689DF80E1012019954A0
:109298000022216801A8104403EB01111144C07A8F
:1092A8000132082A0872F4D1044B1D6001E009F06C
:1092B8006DFB06B0BDE83140854670471029012096
:1092C800842801200064004090280120684620F08E
:1092D80007018D4631B52B4B2B4A1968126886B0A9
:1092E800914205D129480121002209F0D2FB44E02E
:1092F8001A68274901EB0212507800F0FF0248B1C2
:1093080004228DF80C20002201921A6801EB021247
:10931800526806E018688DF80C2001EB00104068D0
:10932800019002921A6801EB0212927802F0FF0093
:109338001AB102228DF80D2001E08DF80D001A688F
:1093480012018A5C8DF80E2000221C680D4801EB82
:1093580004141444257A01AC14440132082AE57235
:10936800F3D1036801A9013303600368082B04BF24
:1093780000230360054809F026FA06B0BDE831402D
:10938800854670478C280120882801200064004009
:1093980014290120F0B501388BB00F461546022379
:1093A80007282AD8DFE800F0211917110F0D0B0440
:1093B800ADF80C300B238DF81030012324E0032383
:1093C8001CE006231AE00C2318E00F22ADF80C204D
:1093D8008DF8102018E01E2310E03C23ADF80C3067
:1093E8000F238DF8103007230EE07823ADF80C30EA
:1093F8000C238DF81030032306E00823ADF80C3059
:109408000F238DF8103002238DF81130884800237F
:109418008DF80F3009F07EF84FF0007001210AF046
:109428005FF8082001210AF037F80323002401938C
:109438000820022301218DF808308DF809308DF8B5
:109448000A408DF80B400AF027F87A4801A909F07C
:1094580077FE78482146092209F0EFFE7548012178
:10946800092209F0EAFE0126714803A98DF80E4089
:109478008DF812408DF813608DF814408DF8154062
:109488008DF816608DF8176009F05EF8B7F5006F73
:109498008DF822408DF823408DF824600FDA7B0187
:1094A800ADF818304FF6FF73ADF81A40ADF81C3020
:1094B800ADF81E30ADF820408DF825600DE04FF670
:1094C800FF73ADF81840ADF81A40ADF81C30ADF890
:1094D8001E30ADF820408DF8254006A809F09FF809
:1094E800012300228DF822308DF823208DF82430B6
:1094F80095B1B5F5006F0FDA6901ADF81A204FF68E
:10950800FF72ADF81810ADF81C20ADF81E20ADF8AC
:1095180020308DF825300DE04FF6FF71ADF818209A
:10952800ADF81A20ADF81C10ADF81E10ADF82030BB
:109538008DF8252006A809F072F802238DF822304C
:109548007B13FF0047F0040700260124ADF81A70CA
:1095580006A84FF6FF77ADF818308DF823608DF820
:109568002440ADF81C70ADF81E70ADF820608DF881
:10957800254009F054F80323B5428DF822308DF8C0
:1095880023608DF8244010DD6B13ED0045F00405D1
:10959800ADF81830ADF81A50ADF81C70ADF81E7063
:1095A800ADF820408DF825400CE00423ADF8186094
:1095B800ADF81A30ADF81C70ADF81E70ADF820404B
:1095C8008DF8256006A809F02AF801240726002549
:1095D800142368468DF800308DF801608DF802502C
:1095E8008DF803400BF084F9152368468DF8003098
:1095F8008DF801608DF802508DF803400BF078F972
:10960800132368468DF800308DF801608DF80250FC
:109618008DF803400BF06CF922460548022109F049
:1096280038FA03481021224609F033FA0BB0F0BD8E
:1096380000640040000C0240F0B5437887B004464F
:10964800426833B104238DF80C3000230292019351
:1096580003E08DF80C3001920293A37803B1022342
:109668008DF80D3023788DF80E300023E11801AA0B
:109678001A44097A0133082BD172F7D1114801A98C
:1096880009F0A1F8042817D10F4F104B3D681B684B
:109698000135082D08BF00259D420FD03E680C4BB0
:1096A80003EB061694E80F0086E80F000121054831
:1096B8000A463D6009F0EDF9012000E0002007B0FE
:1096C800F0BD00BF00640040882801208C280120DC
:1096D8001429012030B50D4B0D4C054622681B6836
:1096E8009A420ED023685A1C22600A4A02EB0313DE
:1096F8000FCB85E80F002368082B04D100232360D3
:1097080001E0002030BD012030BD00BF102901203C
:1097180084280120902801202DE9F0474FF480503B
:1097280088B0012109F0E8FE464E01200024E0231C
:109738000225014601938DF80A408DF80B408DF8FB
:1097480008508DF8095009F0A7FE304601A909F024
:10975800F7FC052130460A4609F06FFD3A4F3046BE
:109768000621052209F069FD05223046072109F086
:1097780064FD01264FF4827A4FF400794FF0100807
:10978800384603A9ADF80C40ADF81040ADF81A40C2
:10979800ADF81C40ADF80EA0ADF81250ADF814604D
:1097A800ADF81690ADF8188009F0ACFF3846314690
:1097B8000AF045F831464FF4804009F091FE07F56C
:1097C80054474FF460432846314601938DF80A40C8
:1097D8008DF80B408DF808508DF8095009F05CFEA3
:1097E800384601A909F0ACFC38460D21052209F0DC
:1097F80024FD38460E21052209F01FFD05223846B2
:109808000F2109F01AFDADF80C40ADF81040ADF885
:109818001A40ADF81C400D4C03A92046ADF80EA027
:10982800ADF81250ADF81460ADF81690ADF8188088
:1098380009F068FF204631460AF001F808B0BDE893
:10984800F08700BF000002400030014000380040AF
:1098580070B50D46144628B101282AD11D4B102297
:109868005A8304E01C4B02225A831E4610E01B4810
:1098780002210AF074F80028F9D0184829460AF09D
:1098880039F8164801210AF06AF80028F9D01AE0D8
:10989800134802210AF063F80028F9D01048294635
:1098A8000AF028F80E4801210AF059F80028F9D0E2
:1098B80001E0002070BD0CB10223338308480AF090
:1098C80016F8C0B270BD14B1024B10221A830348B7
:1098D800F5E700BF000002400010024000300140E0
:1098E80000380040000000002DE9F0414FF48000EE
:1098F8009CB0012109F0D0FD4FF4807001210025B2
:1099080009F0FAFD0327332301A9514801938DF883
:1099180008708DF80B5009F013FC01A94D4801247B
:1099280001978DF808708DF80B5009F009FC01A912
:1099380049484A4E01948DF808708DF80B5009F08B
:10994800FFFB21464FF4800009F0A6FD21464FF4A5
:10995800807009F0D1FD304609F074F9404B4FF0A2
:1099680007080E933F4B30460F934FF480631393D1
:109978004FF4006314934FF4005315934FF480731E
:1099880016930DA94FF4003317930D951095CDF844
:1099980044801295189519941A951B9509F0D8F9D1
:1099A80021463046A6F5A236103E09F00CFA03A867
:1099B800039504950595069508F02AFC304607A9F5
:1099C80007958DF820408DF8214009950A950B954B
:1099D8008DF8308008F0EDFB3046214608F0E0FCB9
:1099E8003046224623460A2108F05EFC30462346CC
:1099F8000E21022208F058FC30463A4623460F2131
:109A080008F052FC304623460821042208F04CFC9A
:109A1800304623460921052208F046FC30462346F5
:109A28000B21062208F040FC4246234630462946D0
:109A380008F03AFC3046214608F0BBFC3046214687
:109A480008F000FC304608F077FC1CB0BDE8F08157
:109A58000008024000040240000002401064024076
:109A68004C200140440600200928F8B51FD008D82A
:109A7800042810D0082812D0002879D14A4B188819
:109A88000BE00B2863D05FD30C2863D0FF286FD17D
:109A9800454B988801E0444B588880B2F8BD424B4A
:109AA800588940F2712380B258430013F8BD3E4BE9
:109AB800988880B20DF0AAF90CF08CFD00223B4B7F
:109AC8000CF0DCFD2CA3D3E900230CF0D7FD0446F1
:109AD8000D4622462B4628A1D1E900010CF01AFCBC
:109AE80027A3D3E9002306460F46204629460CF053
:109AF800EFFE02460B46304639460CF0E9FE0DF003
:109B08007FF80CF067FD0022294B0CF0E1FE0DF008
:109B1800F3FF1DA3D3E900230CF0B0FD1CA3D3E988
:109B280000230CF0F9FB02460B461BA1D1E900010A
:109B38000CF0CEFE1AA3D3E900230CF0EBFB0DF0DA
:109B48005FF80DF031FBF8BD174BD88804E0164BD1
:109B5800188901E0144B988944F2740380B2584381
:109B680040F6FF7390FBF3F0A0F500503A38F8BDCB
:109B78000020F8BDAFF300806666666666660A4038
:109B88009A99999999990140C3F5285C8FA27240D6
:109B98000000000000FEAA409A999999FD6F2F4194
:109BA800C3F5285C8F127140440600200000303F46
:109BB80000002440AFF300800C4BC0EBC0001844F9
:109BC80090F800380B7090F801384B7090F8023814
:109BD8008B7090F80338CB7090F804380B7190F8BC
:109BE80005384B7190F806388B7170475406002081
:109BF80038B54FF40063254A002199540133B3F571
:109C0800804FF8D14FF40064002006210122FFF7AD
:109C18001FFE002005210246FFF71AFE002001461C
:109C28000122FFF715FE8307F3D500200221024623
:109C3800FFF70EFE0020C4F307210246FFF708FED7
:109C48000020E1B20246FFF703FE0025B5F13F0E02
:109C5800DEF100024FF0000052EB0E020146013522
:109C6800FFF7F6FD402DF1D1002005210246FFF750
:109C7800EFFD002001460122FFF7EAFDC307F3D4F8
:109C88004034B4F5804FBFD138BD00BF5406002022
:109C9800F7B5C0EBC00000F5006500200C46024691
:109CA8000321FFF7D5FD0020C5F307210246FFF782
:109CB800CFFD0020E9B20246FFF7CAFD00200146A9
:109CC8000246FFF7C5FD0746002001460246FFF79A
:109CD800BFFD0646002001460246FFF7B9FD0546CE
:109CE800002001460246FFF7B3FD8DF8030000206F
:109CF80001460246FFF7ACFD8DF80400002001463E
:109D08000246FFF7A5FD8DF8050000200146012257
:109D1800FFF79EFD23788DF80600BB420DD16378CE
:109D2800B3420AD1A378AB4207D1DDF80300D4F8D7
:109D38000330C31A5842584100E0002003B0F0BD78
:109D480038B51B4B04460D46195500200621012243
:109D5800FFF77EFD002005210246FFF779FD002070
:109D680001220146FFF774FD8207F3D50020022186
:109D78000246FFF76DFD0020C4F307210246FFF7F6
:109D880067FD0020E1B20246FFF762FD0020294688
:109D98000122FFF75DFD002005210246FFF758FD6F
:109DA800002001460122FFF753FDC307F3D438BD55
:109DB8005406002038B5C0EBC0050C4605F5006018
:109DC8000978FFF7BDFF05F601006178FFF7B8FFD6
:109DD80005F60200A178FFF7B3FF05F60300E17866
:109DE800FFF7AEFF05F604002179FFF7A9FF05F696
:109DF80005006179FFF7A4FF05F60600A179BDE823
:109E08003840FFF79DBF2DE9F041002304460F4677
:109E18001646B34205D03D4AF95C2244D154013379
:109E2800F7E7002006210122FFF712FD0020052197
:109E38000246FFF70DFD002001460122FFF708FD4D
:109E48008507F3D5002002210246FFF701FD002017
:109E5800C4F307210246FFF7FBFC0020E1B20246EB
:109E6800FFF7F6FC0025B54242D0013414F03F0854
:109E7800795D04D0721EA81A4242424100E00122D4
:109E88000020FFF7E5FCB8F1000F2FD1731E9D42AB
:109E98002CD2002005210246FFF7DAFC00200146FB
:109EA8000122FFF7D5FC10F00100F2D106210122B2
:109EB800FFF7CEFC002005210246FFF7C9FC002071
:109EC80001220146FFF7C4FC8207F3D500200221D6
:109ED8000246FFF7BDFC0020C4F307210246FFF746
:109EE800B7FC0020E1B20246FFF7B2FC0135BAE741
:109EF800002005210246FFF7ABFC002001460122A5
:109F0800FFF7A6FCC307F3D4BDE8F0815406002090
:109F1800014B185C704700BF5406002010B50023A1
:109F2800934205D0034C0444E45CCC540133F7E776
:109F380010BD00BF5406002073B50020032102465F
:109F4800FFF786FC002001460246FFF781FC00204F
:109F580001460246FFF77CFC002443F6FF72A51A6F
:109F68006A424FF000006A410146FFF771FC374B27
:109F780018550134B4F5804F1D46EED10020052157
:109F88000246FFF765FC002001460122FFF760FC4E
:109F980010F07104F2D1FEF765F90646FEF762F992
:109FA800801B0028B8BF4042B0F5FA6F07DA3CB909
:109FB80095F8FF47B4F142035C425C41EEE714B107
:109FC800234B1B78ABB340F2FF700021FFF7B8FEBC
:109FD800FFF70EFE00201F494022FFF714FF4FF441
:109FE80080701D49B422FFF70EFF40201B49202234
:109FF800FFF709FF002301934FF4C364204601A92A
:10A0080004220434FFF7FFFEB4F5FF6FF6D10023F6
:10A0180001934FF4A764204601A904220434FFF7F2
:10A02800F2FEB4F5C36FF6D140F2FF704221FFF79C
:10A0380087FE002007494022FFF770FF40200849AB
:10A048002022FFF76BFF02B070BD00BF540600204E
:10A05800C42901200400002064800108448001080C
:10A06800DC290120F8B505460C4605F085FE0646B4
:10A0780028B128462146BDE8F84005F083BE32469F
:10A08800C4F307410120FFF7E3FB0A4D07023246FC
:10A09800C4F3072101202F60FFF7DAFB38430602DB
:10A0A8000120E1B202462E60FFF7D2FB30430609D9
:10A0B8002E60F8BD5446002038B5444C0B2303FBF2
:10A0C800004203FB00431179032984BF0321117166
:10A0D8009A79032A84BF03229A710B2303FB004257
:10A0E80003FB0043117A0F2984BF0F2111725A7A9A
:10A0F800072A84BF07225A720B2303FB004203FB83
:10A108000043917A0F2984BF0F2191725A7B0F2A3D
:10A1180084BF0F225A730B2202FB004302FB00424A
:10A12800997B0F2984BF0F21997313795279DB0327
:10A1380043F4002121611AB1244943F404230B613B
:10A148000B2101FB0041C979204B19B1196941F470
:10A15800005119610B236AB903FB0043197A9A79F4
:10A16800C90141EAC22122695B7A0A4342EA031221
:10A1780022611AE003FB00431B7B144A1BB11369DD
:10A1880043F4805313610B2202FB0042917B557B01
:10A1980022690E4B42EAC51201F0070542EA051290
:10A1A800090748BF42F400621A610B2202FB004211
:10A1B800D17A064B19B9917A1A690A431A61216949
:10A1C800FFF750FF2369636138BD00BF5446002084
:10A1D80010B5114C00232361C300E218527F12B15D
:10A1E8004FF400722261E118897F0B4A19B1116995
:10A1F80041F480711161E218D17F23440F2984BF93
:10A208000F21D177D97F236919432161FFF72AFFED
:10A218002369236210BD00BF5446002038B5224C84
:10A228004FF460232361C300E21892F82B2012B187
:10A238004FF470222261E21892F8251092F8245007
:10A24800090341EA853192F826202569012A41EA65
:10A258000501216103D1144A41F480611161E118BB
:10A2680091F82750226991F8281042EA052201291D
:10A27800226103D10C4942F080020A61E11891F889
:10A288002910094A012903D1116941F040011161DE
:10A29800234493F82A10236943EA01112161FFF747
:10A2A800E1FE2369E36238BD5446002038B52A4CE4
:10A2B80043001A18224492F931103F29C4BF3F21A4
:10A2C80082F831101A18224492F931103F31BCBF7C
:10A2D800C12182F831101A18224492F832101F292D
:10A2E80084BF1F2182F832104FF4402222611A18CD
:10A2F800224492F83020012A03D1174A4FF4502102
:10A30800116104EBC00191F82B10134A51B91918C7
:10A31800114491F83150116905F07F0541EA052192
:10A3280011610CE01D18154495F8315001F0030136
:10A3380005F07C052943156945EA012515610344A3
:10A34800234493F83210236919432161FFF78AFEE9
:10A358002369636338BD00BF5446002010B58300ED
:10A36800254C1A18224492F83810012984BF01217B
:10A3780082F838101A18224492F83910032984BF39
:10A38800032182F839101A18224492F83A100F293A
:10A3980084BF0F2182F83A101A18224492F83B1011
:10A3A800032984BF032182F83B101A18224492F82B
:10A3B8003C1003440F2988BF0F21234488BF82F82B
:10A3C8003C1093F83C1093F8382041F4202141EADE
:10A3D800C23193F8392041EA423193F83A2093F890
:10A3E8003B3041EA022141EA43112161FFF73AFE7D
:10A3F8002369236410BD00BF54460020224B01206E
:10A4080010B503220024052183F8300083F82800C2
:10A41800022083F8264083F8274083F8294083F8F0
:10A428002A0083F82B4083F8384083F8394083F8B2
:10A438003A4083F83B4083F83C405C779C77DC7774
:10A4480018715C71DC719C711872DC721C735C731E
:10A4580083F8311083F8321083F8242083F82520FC
:10A468005A7299729A732046FFF778FF2046FFF7D1
:10A478001DFF2046FFF7D2FE2046FFF7A9FE204623
:10A48800BDE81040FFF718BE54460020054B0429CC
:10A4980003EBC00318BF0022D97718BF5A77FFF71C
:10A4A80097BE00BF54460020044B03EBC003597706
:10A4B80009B10422DA77FFF78BBE00BF54460020AB
:10A4C800024B03EBC0039977FFF782BE5446002086
:10A4D800024B03EBC000C07F704700BF544600200A
:10A4E800024B03EBC000407F704700BF544600207A
:10A4F800024B03EBC000807F704700BF544600202A
:10A50800034B0B2202FB00331971FFF7D5BD00BFC7
:10A5180054460020034B0B2202FB00335971FFF70E
:10A52800CBBD00BF54460020034B0B2202FB003377
:10A53800D971FFF7C1BD00BF54460020034B0B2261
:10A5480002FB00339971FFF7B7BD00BF54460020E6
:10A55800034B0B2202FB00331972FFF7ADBD00BF9E
:10A5680054460020034B0B2202FB00335972FFF7BD
:10A57800A3BD00BF54460020034B0B2202FB00334F
:10A588009972FFF799BD00BF54460020034B0B2278
:10A5980002FB00331973FFF78FBD00BF544600203C
:10A5A800034B0B2202FB00335973FFF785BD00BF35
:10A5B80054460020034B0B2202FB00339973FFF72C
:10A5C8007BBD00BF54460020024B0B2202FB00302B
:10A5D8000079704754460020024B0B2202FB0030E2
:10A5E8004079704754460020024B0B2202FB003092
:10A5F800C079704754460020024B0B2202FB003002
:10A608008079704754460020024B0B2202FB003031
:10A61800007A704754460020024B0B2202FB0030A0
:10A62800407A704754460020024B0B2202FB003050
:10A63800807A704754460020024B0B2202FB003000
:10A64800007B704754460020024B0B2202FB00306F
:10A65800407B704754460020024B0B2202FB00301F
:10A66800807B704754460020034A00EB8003134464
:10A6780083F83810FFF772BE54460020034A00EBF7
:10A688008003134483F83910FFF768BE544600204E
:10A69800034A00EB8003134483F83A10FFF75EBEC9
:10A6A80054460020034A00EB8003134483F83B1010
:10A6B800FFF754BE54460020034A00EB80031344BE
:10A6C80083F83C10FFF74ABE54460020034B00EBCA
:10A6D8008000184490F83800704700BF54460020A6
:10A6E800034B00EB8000184490F83900704700BF16
:10A6F80054460020034B00EB8000184490F83A00C1
:10A70800704700BF54460020034B00EB80001844FC
:10A7180090F83B00704700BF54460020034B00EB05
:10A728008000184490F83C00704700BF5446002051
:10A73800034A00EB4003134483F83010FFF7B6BD1B
:10A7480054460020034A00EB4003134483F83110B9
:10A75800FFF7ACBD54460020034A00EB4003134406
:10A7680083F83210FFF7A2BD54460020034B00EBDC
:10A778004000184490F83000704700BF544600204D
:10A78800034B00EB4000184490F93100704700BFBC
:10A7980054460020034B00EB4000184490F8320068
:10A7A800704700BF54460020034B03EBC00383F8F7
:10A7B8002410FFF733BD00BF54460020034B03EBC2
:10A7C800C00383F82510FFF729BD00BF54460020B9
:10A7D800034B03EBC00383F82610FFF71FBD00BF30
:10A7E80054460020034B03EBC00383F82710FFF700
:10A7F80015BD00BF54460020034B03EBC00383F88C
:10A808002810FFF70BBD00BF54460020034B03EB95
:10A81800C00383F82910FFF701BD00BF544600208C
:10A82800034B03EBC00383F82A10FFF7F7BC00BF04
:10A838005446002010B5064B044603EBC00383F8CA
:10A848002B10FFF7EBFC2046BDE81040FFF72EBDAC
:10A8580054460020024B03EBC00090F824007047D8
:10A8680054460020024B03EBC00090F825007047C7
:10A8780054460020024B03EBC00090F826007047B6
:10A8880054460020024B03EBC00090F827007047A5
:10A8980054460020024B03EBC00090F82800704794
:10A8A80054460020024B03EBC00090F82900704783
:10A8B80054460020024B03EBC00090F82A00704772
:10A8C80054460020024B03EBC00090F82B00704761
:10A8D800544600202DE9F0472E4D1E462B1893F8BC
:10A8E800443004468A469146DDF82080099F042BAF
:10A8F8001AD8DFE803F003080D121700FFF7DCFB96
:10A908002B19012212E0FFF789FC2B1902220DE016
:10A91800FFF724FD2B19032208E0FFF7C7FC2B19CA
:10A92800042203E0FFF754FC2B19002205EBC404B2
:10A9380083F8442094F82A20164B012A12D002D317
:10A94800022A14D020E0BAF1000F03D01B689B0C38
:10A958008AF80030B9F1000F16D02B689B0A89F8E5
:10A96800003011E086B11B689B0A33600CE01EB111
:10A978001B68DB0B5B013360B8F1000F04D02B6858
:10A98800C3F3842388F800300FB12B683B70BDE80F
:10A99800F08700BF54460020054B0B2202FB003312
:10A9A800DA7A1AB90122DA72FFF786BB704700BF5C
:10A9B80054460020054B0B2202FB0033DA7A1AB109
:10A9C8000022DA72FFF778BB704700BF54460020B8
:10A9D800044B0B2202FB0030C07AD0F1010038BFD3
:10A9E8000020704754460020064B40F2826203EB79
:10A9F800C00090F8290040F63B43002814BF1046D9
:10AA080018467047544600202DE9F041114AC70006
:10AA1800D31993F82A600546032E904604D00322E2
:10AA280083F82A20FFF7FAFB2846FFF7F7FBD8F848
:10AA38000040230344BF6FEA04346FEA1434032E42
:10AA480005D0474487F82A602846FFF7E7FB2046E9
:10AA5800BDE8F0815446002070B5084C9DF81060A0
:10AA68009DF8145004EBC00421766276A376E6764E
:10AA78002577BDE87040FFF7ABBB00BF5446002008
:10AA880006281AD8DFE800F004070A0D101316008C
:10AA98000A4B1B6810E0094B1B6A0DE0074B5B690A
:10AAA8000AE0064B1B6C07E0044B5B6B04E0034BAE
:10AAB800DB6A01E0014BDB7A0B60704754460020EB
:10AAC8007047704770477047704770477047122348
:10AAD8000B800148704700BF4400002004230B800E
:10AAE800004870475600002000207047002070473B
:10AAF8000020704770B5084C002223688A4207D0AE
:10AB08003F2B03D8865CE5182E7101330132F5E737
:10AB18002360002070BD00BF9C46002010B5044C87
:10AB28000A46044821460AF0EBFB204610BD00BF48
:10AB3800B33D0120C996010810B5044C0A460448E3
:10AB480021460AF0DDFB204610BD00BFB33D0120C1
:10AB5800E196010810B5044C0A46044821460AF05B
:10AB6800CFFB204610BD00BFB33D0120F996010878
:10AB780010B5044C0A46044821460AF0C1FB204699
:10AB880010BD00BFB33D01200197010810B5044C6A
:10AB98000A46044821460AF0B3FB204610BD00BF10
:10ABA800B33D01200C970108202811D0212821D17C
:10ABB800114B9A69100A0A704870100C120ECA706C
:10ABC8001A7F88700A715A7F9B7F4A718B7111E0D6
:10ABD8008A784878120442EA00220878064B024331
:10ABE800C87842EA00629A610A791A774A795A77EC
:10ABF8008A799A770020704744000020F7B5274CDF
:10AC08004FF4C053002603270093204602236946C9
:10AC18008DF804308DF805708DF806608DF80760A2
:10AC280008F08EFA20460B210A2208F006FB20467F
:10AC38000A220C2108F001FB01254FF4007320467D
:10AC4800694600938DF805708DF804608DF80650FC
:10AC58008DF8076008F074FA20460A22092108F0E6
:10AC6800ECFA4FF480632046694600938DF806504D
:10AC78008DF807508DF8057008F062FA0A210A4627
:10AC8800204608F0DAFA29464FF4804008F034FCF0
:10AC98008020294608F00CFC03B0F0BD00000240FB
:10ACA80007B54FF4C06009F019FE43238DF804304E
:10ACB8000322012301A88DF805308DF806208DF8B0
:10ACC800073009F015FE03B05DF804FB78235843FC
:10ACD8000722B0FBF2F0002301338342FCD970470E
:10ACE8004FF47A735843FFF7F1BF684620F0070125
:10ACF8008D4601B503480BF0DDF8BDE801408546F7
:10AD0800704700BF742A0120F0B500238B420ED093
:10AD1800074A084E15686C1C1460C75CB4F5006FD0
:10AD280028BF0024775528BF14600133EEE7F0BD33
:10AD380040280120B3350120074B10B51A684AB1E5
:10AD4800002305490C1D1C5DC45401339342F8D1FE
:10AD580000230B60104610BD9C460020084B1B6862
:10AD6800082B0BD90023064A111D595CC154013325
:10AD7800092BF8D100231360012070470020704789
:10AD88009C46002007B5064A064802F13C0300939A
:10AD980001212032044B09F01DFF03B05DF804FBCC
:10ADA80044000020742A01205801002001480BF0BB
:10ADB80054B800BF742A012010B5034CA378002BA7
:10ADC80040F05E8202E000BF683001206378FE2B0D
:10ADD80000F2F083DFE813F0FF00E103060113013E
:10ADE80020012D0138013C01EE03EE03EE03EE03D2
:10ADF80042014F015B01EE03EE037001EE03850192
:10AE08008B01EE03EE03EE03EE0391019701EE03CF
:10AE18009D01A301EE03EE03EE03EE03EE03EE0342
:10AE2800EE03EE03EE03EE03EE03EE03EE03EE0392
:10AE3800EE03EE03EE03EE03EE03EE03EE03EE0382
:10AE4800EE03EE03EE03EE03EE03EE03EE03EE0372
:10AE5800EE03EE03EE03EE03EE03EE03EE03EE0362
:10AE6800EE03EE03EE03EE03EE03EE03EE03EE0352
:10AE7800EE03EE03EE03EE03EE03EE03EE03EE0342
:10AE8800EE03EE03EE03EE03EE03EE03EE03EE0332
:10AE9800EE03EE03EE03EE03EE03EE03EE03EE0322
:10AEA800EE03EE03EE03EE03EE03EE03EE03EE0312
:10AEB800A701AD01B301B901BF01C501CB01D101A2
:10AEC800D701DD01E301E901EF01F501FB01EE0323
:10AED800020208020E025E02660214026D02EE030E
:10AEE8001E02EE0326022C0232023C0244024A02EF
:10AEF80077025602EE03EE03EE03EE03EE03EE03D3
:10AF0800EE03EE03EE03EE03EE03EE03EE03EE03B1
:10AF1800EE03EE03EE03EE03D502DD02E502ED02D9
:10AF2800F502070319032B0333033B0343034B03C6
:10AF3800530361036903710379038103890391034F
:10AF4800EE0399039E03B103B603EE03EE03EE038B
:10AF5800EE03EE03EE03EE03EE038E0293029B0272
:10AF6800EE03EE03BE03EE03A302D003DA03EE03FF
:10AF7800A802EE03EE03EE03EE03E103E703EE039C
:10AF8800BE02EE03C302EE03EE03EE03EE03EE038E
:10AF9800EE03EE03EE03EE03EE03EE03EE03EE0321
:10AFA800EE03EE03EE03EE03EE03EE03EE03EE0311
:10AFB800EE03EE03EE03EE03EE03EE03EE03EE0301
:10AFC800EE03EE03EE03EE03EE03EE03EE03EE03F1
:10AFD800EE03EE03C802D4F803100020BDE81040C9
:10AFE80004F084BCD4F80310D24BD34A0B449342E8
:10AFF80000F24681BDE81040002004F01BBCD4F8E4
:10B008000310CC4BCC4A0B44934200F23981BDE883
:10B018001040002004F02EBCD4F80310C54BC64ADB
:10B028000B44934200F22C81BDE81040002004F04C
:10B03800D1BCD4F80310C14B994200F22181BDE87C
:10B048001040002004F0A4BCE278BD4B5A7202E024
:10B05800E278BB4B9A720122BA4BADE2D4F80320D6
:10B06800B74B1AB95A7B42F0020202E05A7B22F02F
:10B0780002025A7310BDD4F80320B14B1AB95A7B97
:10B0880042F00102F5E75A7B22F00102F1E70020C5
:10B09800022104F0BFFCD4F8034004F069FA002C44
:10B0A800B8BF6442844200F3EB80BDE81040A64B71
:10B0B800D3F8030005F056B80020022104F0AAFCDA
:10B0C800D4F8034004F054FA002CB8BF6442844218
:10B0D80000F3D680BDE810409B4BD3F8030005F081
:10B0E800CFB8D4F80300BDE8104005F02FB8D4F865
:10B0F8000300BDE8104005F051B8D4F80300BDE8DE
:10B10800104006F05FBAD4F80300BDE8104006F01E
:10B118005FBAD4F80300BDE8104006F05FBABDE896
:10B12800104006F061BAD4F80300BDE8104004F0FE
:10B1380095BED4F80300BDE8104004F095BED4F8DD
:10B148000300BDE8104004F095BED4F80300BDE844
:10B15800104004F029BED4F80300BDE8104004F004
:10B168002FBED4F80300BDE8104004F03DBED4F86B
:10B178000300BDE8104004F03DBED4F80300BDE86C
:10B18800104004F093BFD4F80300BDE8104004F069
:10B1980037BED4F80300BDE8104004F037BED4F839
:10B1A8000300BDE8104004F037BED4F80300BDE842
:10B1B800104004F037BED4F80300BDE8104004F096
:10B1C80037BED4F80300BDE8104004F039BED4F807
:10B1D8000300BDE81040C0B204F03ABED4F8030042
:10B1E800BDE8104004F018BFD4F80300BDE81040D3
:10B1F80004F050BFD4F80300BDE8104004F018BFB5
:10B20800D4F803100020091A18BF0121BDE8104026
:10B2180004F088BDD4F80330002B00F0CE8106F08E
:10B2280085F92AE0D4F80300BDE8104004F02EBEEA
:10B23800D4F80300BDE8104004F022BED4F803009F
:10B24800A0F10A03282B1BD8BDE8104004F02EBE3D
:10B25800D4F80300002813DBBDE8104004F02CBE2E
:10B26800D4F80300BDE8104004F02CBED4F8033035
:10B27800002B00F0A28106F075F9002840F09D81AE
:10B28800042298E1D4F803000028F9DBBDE8104057
:10B2980004F074BFD4F80330022BF1D82A4BDA78C3
:10B2A8002A4B89E1D4F803100020BDE8104004F0CF
:10B2B800B1BBD4F80310264B9942E1D8BDE8104041
:10B2C800002004F0F7BA002004F076FC08B106224A
:10B2D80071E1A0781A4BE17803EB4013D97204F0BE
:10B2E800A9FBE178A078C1F10801C9B2BDE8104016
:10B2F800FFF7CCB8D4F80320114B1A7210BDD4F85C
:10B308000330134A9342BBD80D4A136010BDD4F8DA
:10B3180003300F4A9342B3D8094A536010BDD4F89A
:10B328000320074BDA7710BDD4F80320044BDA81E9
:10B3380010BD00BFFEFF8713FCFF0F277DC3C901A7
:10B34800DC290120382A012068300120E04600204D
:10B35800FFFF8713D4F80320984B5A6110BDD4F827
:10B368000320964B9A8310BDD4F80330052B87D859
:10B37800934B0020D978914B1973BDE8104004F025
:10B38800A7BCD4F803100020C9B2BDE81040FFF7ED
:10B398008BB8D4F803100020C9B2BDE81040FFF7FD
:10B3A8008FB8D4F803100020C9B2BDE81040FFF7E9
:10B3B800A7B8D4F803100020C9B2BDE81040FFF7C1
:10B3C800A9B80020FFF708F9D4F8031028B9A07825
:10B3D800C9B2BDE81040FFF7B1B8A078C9B2BDE85E
:10B3E8001040FFF7D3B80020FFF7F6F8D4F80310A1
:10B3F80028B9A078C9B2BDE81040FFF7A9B8A0786D
:10B40800C9B2BDE81040FFF7D5B80020FFF7E4F84F
:10B41800D4F8031028B9A078C9B2BDE81040FFF7E6
:10B42800A1B8A078C9B2BDE81040FFF7B9B8D4F800
:10B4380003100020C9B2BDE81040FFF79DB8D4F84A
:10B4480003100020C9B2BDE81040FFF70DB9D4F8C9
:10B4580003100020C9B2BDE81040FFF70FB9D4F8B7
:10B4680003100020C9B2BDE81040FFF711B9D4F8A5
:10B4780003100020C9B2BDE81040FFF713B9D4F893
:10B4880003100020C9B2FFF717F9A2784D4B03EB60
:10B49800C203D4F803205A7110BDD4F80310002059
:10B4A800C9B2BDE81040FFF743B9D4F80310002033
:10B4B80049B2BDE81040FFF745B9D4F803100020A1
:10B4C800C9B2BDE81040FFF76FB9D4F803100020E7
:10B4D800C9B2BDE81040FFF771B9D4F803100020D5
:10B4E800C9B2BDE81040FFF773B9D4F803100020C3
:10B4F800C9B2BDE81040FFF775B9D4F803100020B1
:10B50800C9B2BDE81040FFF781B9D4F803202B4B2E
:10B518009A6110BDD4F803002A4B186010B9597904
:10B52800FFF7CAF8A078284B1B5C012B45D1BDE872
:10B538001040234BD978FCF773BFD4F80320214B74
:10B548001A7110BDD4F803100020C9B2BDE810402C
:10B55800FEF7EABF194BD4F80300196920B141F08E
:10B5680080611961002002E021F080611961090EF3
:10B57800BDE81040FDF706B9104BE1781A690020C4
:10B5880022F07F4242EA01621A61F1E7D4F803101F
:10B598000020BDE81040FDF75BBCD4F80300BDE80F
:10B5A800104004F08FBDD4F803100020BDE810400F
:10B5B800FDF746BC0322054B1A7010BDDC2901209B
:10B5C80068300120AC2901203B2A0120DC30012011
:10B5D80070B5034D034CAB78002B40F0158403E0A5
:10B5E80068300120DC3001206B78FE2B00F2F283FA
:10B5F800DFE813F0FF00040109010E01130118012F
:10B608001D01210125012A013001430156015F0175
:10B618006401710187018B018F01FE010202F003B1
:10B62800F003F003F00306020A020E0212021602E9
:10B63800F003F003F003F003F003F003F003F0036A
:10B64800F003F003F003F003F003F003F003F0035A
:10B65800F003F003F003F003F003F003F003F0034A
:10B66800F003F003F003F003F003F003F003F0033A
:10B67800F003F003F003F003F003F003F003F0032A
:10B68800F003F003F003F003F003F003F003F0031A
:10B69800F003F003F003F003F003F003F003F0030A
:10B6A800F003F003F003F003F003F003F003F003FA
:10B6B800F003F003F003F003F003F003F003F003EA
:10B6C800F003F003F003F003F003F0031A021E0284
:10B6D800220226022A022E02320236023A023E02D2
:10B6E800420246024A024E025202560266026A02AA
:10B6F8006E02EB02EF027202F402F90277027B0299
:10B708007F02830287028B028F029302FE02970256
:10B71800F003F003F003F003F003F003F003F00389
:10B728009B029F02A402A902AE02B302B802F00370
:10B73800F003F0034B03500355035A035F036D03F3
:10B748007B0389038E03930398039D03A203A60337
:10B75800AB03B003B503BA03BF03C403C903CD03E6
:10B76800D103D503D903F003F003F003F003F0038A
:10B77800F003F003F0030C03100314031803F003A1
:10B78800F003F0031C03DE03E203F0032003F003DD
:10B79800240328033B03E703EB03F0033F03F00311
:10B7A8004303F003F003F003F003F003F003F003A6
:10B7B800F003F003F003F003F003F003F003F003E9
:10B7C800C602CA02CE02D202D602DA02DE02E202C1
:10B7D800E602F003F003F003F003F003F003F003D4
:10B7E800F003F003F003F003F003F003F003F003B9
:10B7F8004703002004F076F9606007E3002004F0B6
:10B808008BF9606002E3002004F020F96060FDE23B
:10B81800002004F033F96060F8E2002004F0AEF98B
:10B828006060F3E2002004F091F96060EEE29E4B64
:10B838005B7A6360EAE29C4B9B7A6360E6E20020F5
:10B8480004F0E4F96060E1E2984B1B69C3F38023DC
:10B858006360DBE2964B587E30B904F031FA003071
:10B8680018BF01206060D1E2002004F029FAD0F16D
:10B87800010038BF00206060C8E28D4B587E30B9A7
:10B8880004F016FA003018BF01206060BEE2002004
:10B8980004F00EFAD0F1010038BF00206060B5E274
:10B8A800814B5B7B13F0020F14BF002301236360FD
:10B8B800ACE27D4B5B7B13F0010FF5E7002004F051
:10B8C80075F9022803D004F0A1FB60609EE204F041
:10B8D8004FFC60609AE2002004F06EF918B103F0A2
:10B8E80047FE606092E2A878FFF77EF8AA786E4B70
:10B8F80003EB42135B7AFF22584390FBF2F3636039
:10B9080084E204F0C9FC606080E204F0BFFC60607F
:10B918007CE20020674E606004F078F918B1736823
:10B9280043F00103736004F0B7FC18B1636843F097
:10B938000203636004F050FA18B1636843F004032B
:10B948006360A87804F032F918B9636843F0080313
:10B958006360A87804F02AF9012803D1636843F0EA
:10B9680010036360A87804F021F9022803D1636802
:10B9780043F0200363604D4B1B69590503D5636889
:10B9880043F0400363604C4B1A69120703D56268A1
:10B9980042F0800262601B69DB0603D5636843F4EA
:10B9A8008073636002F030FF18B1636843F400737A
:10B9B800636002F023FF18B1636843F48063636037
:10B9C80002F028FF18B1636843F4006363603B4BDF
:10B9D8001B781BB1636843F48053636005F0ECFD8A
:10B9E800002800F01382636843F4005363600DE29B
:10B9F80004F0B2FB606009E204F0ECFB606005E271
:10BA080005F0C2FD606001E205F0C4FD6060FDE183
:10BA180005F0C6FD6060F9E105F0C8FD6060F5E17C
:10BA280005F0CAFD6060F1E104F0B0FA6060EDE194
:10BA380004F0B2FA6060E9E104F0B4FA6060E5E1AC
:10BA480004F0B8F96060E1E104F0C0F96060DDE19C
:10BA580004F03EFA6060D9E104F040FA6060D5E194
:10BA680004F02AFB6060D1E104F03EFA6060CDE1A9
:10BA780004F040FA6060C9E104F042FA6060C5E190
:10BA880004F044FA6060C1E104F046FA6060BDE188
:10BA980004F04CFA6060B9E104F052FA6060B5E174
:10BAA80004F056FA6060B1E1DC290120000C024084
:10BAB80004000020DC300120000402400035012091
:10BAC80004F0B0FA6060A1E104F0EAFA60609DE178
:10BAD80004F0C8FA606099E1002004F06DF8606035
:10BAE80094E105F039FD606090E104F075F960605B
:10BAF8008CE104F069FA606088E104F05FFA606044
:10BB080084E104F071FA606080E104F073FA606027
:10BB18007CE104F075FA606078E105F02FFD606063
:10BB280074E104F035FB606070E104F0DBFB6060F9
:10BB38006CE10A20FDF798FF606067E10B20FDF7D4
:10BB480093FF606062E10820FDF78EFF60605DE1B1
:10BB58000C20FDF789FF606058E10920FDF784FF9C
:10BB6800606053E10020FEF73FFFAA789B4B03EB90
:10BB780042139B7AFF22584390FBF2F3636045E13E
:10BB880004F016FA606041E104F0F4F960603DE108
:10BB980004F0F6F9606039E105F08EFC606035E18B
:10BBA80005F096FC606031E105F0A8FC60602DE1CD
:10BBB80004F0D4F9606029E1894B1B68636025E1D2
:10BBC8000B20FDF751FF606020E1864B1B78636016
:10BBD8001CE1002003F0EAFF606017E1002003F099
:10BBE8006BFF606012E1002003F060FF60600DE110
:10BBF800002003F0E1FF10B10823636006E1AA7892
:10BC0800764B03EB4213DB7A6360FFE0734B1B7ADE
:10BC18006360FBE0714B1B686360F7E06F4B5B6828
:10BC28006360F3E0704B1B686360EFE06B4BDB7F96
:10BC38006360EBE0694BDB896360E7E06B4B1B6893
:10BC48006360E3E06A4B00221978626011B16949C8
:10BC5800012048601A70684B1A781AB1626842F07D
:10BC68000202626000221A70D0E0644B1B786360A5
:10BC7800CCE05A4B5B696360C8E0584B9B8B6360B0
:10BC8800C4E0564B1B7B6360C0E00020FEF728FC35
:10BC98006060BBE00020FEF72BFC6060B6E000208F
:10BCA800FEF792FC6060B1E00020FEF795FC606052
:10BCB800ACE00020FEF790FC20B9A878FEF79CFCC9
:10BCC8006060A3E0A878FEF7B7FC60609EE0002003
:10BCD800FEF782FC20B9A878FEF796FC606095E034
:10BCE800A878FEF7B9FC606090E00020FEF774FCCD
:10BCF80020B9A878FEF790FC606087E0A878FEF786
:10BD0800A3FC606082E00020FEF78EFC60607DE0AE
:10BD18000020FEF7DBFC606078E00020FEF7E0FC26
:10BD2800606073E00020FEF7E5FC60606EE00020D4
:10BD3800FEF7EAFC606069E0314B5B79636065E0BF
:10BD48000020FEF713FD606060E00020FEF718FD9C
:10BD580060605BE00020FEF77DFD606056E000203B
:10BD6800FEF780FD606051E00020FEF783FD606013
:10BD78004CE00020FEF786FD606047E00020FEF7FB
:10BD880091FD606042E01F4B1B7863603EE0134BFF
:10BD98009B6963603AE01A4B1B68636036E0184B96
:10BDA8001B79636032E00020FEF71EFC60602DE026
:10BDB8000A4BDB7C636029E00020FDF73BF86060FC
:10BDC80024E004F0ADF9606020E00020FDF72CF8D5
:10BDD80060601BE00323237018E000BFDC2901200A
:10BDE800EC340120E04600209C290120C0290120D4
:10BDF800D8290120DC300120B5290120D9290120CA
:10BE0800AC290120A829012004232370084B1B78A2
:10BE180063B1084B62681A60074B1AB91A6842F096
:10BE2800080202E01A6822F008021A6070BD00BF1A
:10BE3800D7300120C83001207030012038B5AF4A12
:10BE480093781446022B00F01F81032B00F0238106
:10BE5800002B40F0908153784D2B00F0A88031D80A
:10BE6800452B72D018D8422B62D009D8402B5BD012
:10BE7800412B40F07E81D178A14B002019705BE006
:10BE8800432B5DD0442B40F07481D2F803309C4999
:10BE98001C2041F81C3F63E0482B66D00CD8462B89
:10BEA80058D0472B40F06581954DD2F8033029468C
:10BEB80041F8083F08209CE04B2B68D072D8492BEA
:10BEC80059D056E1552B00F0AB8017D8512B7AD0BA
:10BED80009D84F2B70D0502B40F04B81D178884B2C
:10BEE8001620997528E0532B7CD000F28C80D2F86C
:10BEF80003308349202041F8203F31E0832B00F0B4
:10BF0800B48006D8572B00F09680582B00F0998003
:10BF18002FE1852B00F0B380C0F0AC80FF2B40F000
:10BF28002881D278774B28E140F2FF70D17803E07E
:10BF3800D178734B01205970BDE83840FDF700BF38
:10BF4800D1786F4B04201971F6E7D1786C4B052036
:10BF58005971F1E7D2F8033069490C2041F80C3FD8
:10BF68000422BDE83840FDF74EBFD3786449262047
:10BF780001F8263F52E0D278614B0AB9DA7503E03E
:10BF880061490122DA754A601720D97DD4E75C4CF3
:10BF9800D1780320E170FDF7D3FEE078BDE83840A2
:10BFA800FDF7BAB8D178564B02209970C4E7D1781A
:10BFB800534B15205975BFE7D2F80310504BC9B23F
:10BFC80059761920B8E74E4B1A7D1D4612F0010F1D
:10BFD80004D0E378DB0701D4FDF70AFEE1781420EA
:10BFE8002975A9E7464DD2F80330294641F8103F94
:10BFF80010200422FDF707FF6879A9682A69BDE8BF
:10C008003840FDF7C7B9D2F80330012B00F2B380EE
:10C018003A4B3B49DB781A2001F81A3F0122A0E786
:10C02800D2F80330012B00F2A680D37834491B20C4
:10C0380001F81B3FF2E7D3783149272001F8273F61
:10C04800ECE72F4DD378294601F8283F2820012214
:10C05800FDF7D9FE95F828301BB9BDE83840FCF744
:10C06800FBBDBDE83840FCF7E4BDD2F80320274B00
:10C078005A6038BDD2F80320254B1A6038BDD2F873
:10C088000320224B9A6038BD5178224BD2F8032006
:10C0980043F8212038BD5378282B51D018D8022BCB
:10C0A80045D00CD8002B39D0012B62D11A4BD2F8CD
:10C0B80003205A60FCF7D6F8144B186138BD092BD9
:10C0C8005CD0272B55D1D2F80320134BDA6038BD4A
:10C0D8002B2B3FD008D8292B37D02A2B49D1D2F87F
:10C0E80003200D4B9A6138BD2D2B3DD037D32E2B15
:10C0F8003FD1D2F80320084B9A6238BD683001203E
:10C1080004000020D6300120DC300120E046002069
:10C11800D8300120E8300120002A0120184BD2F83D
:10C1280003201A60FCF79EF8164BD86038BD144BF4
:10C13800D2F803209A60FCF795F8124B586138BD85
:10C14800D2F803200E4B1A6138BDD2F803200C4BED
:10C158005A6138BDD2F80320094BDA6138BDD2F8EC
:10C168000320074B1A6238BDD2F80320044B5A62E9
:10C1780038BD032200E00422034B1A7038BD00BF0B
:10C18800002A0120E0460020DC300120F7B5B74E38
:10C19800B749327864230B70D6F80330222A4A70E4
:10C1A8004B6035460C4601F0E5805BD80F2A00F05D
:10C1B800698526D8072A00F0D18111D8032A00F012
:10C1C800E88007D8012A00F0B680022A00F0CC8067
:10C1D80001F062BB052A00F0B98140F2BF80B9E1E5
:10C1E8000B2A00F0D88405D8092A00F09F8340F272
:10C1F80088829FE30D2A00F0018540F2E98400F06F
:10C208001BBD192A00F0878614D8152A00F0E68588
:10C2180007D8132A00F07985142A00F0AF8501F0B9
:10C228003BBB172A934A00F05C8600F26786D3610D
:10C2380001F034BB1E2A00F0BF840CD81B2A00F082
:10C248008C86C0F079861C2A41F02683894B00220F
:10C258001A7601F023BB202A00F0E78740F2AC876A
:10C2680001F022B8812A01F00E8135D8412A01F067
:10C27800F88017D8252A01F0B88007D8232A01F0BA
:10C288008080242A01F0848001F006BB272A01F06F
:10C29800DA80C1F0B380402A41F0FE8202F038F81B
:10C2A80001F0FCBA452A01F0E58008D8432A01F0DC
:10C2B800DB8001F2DC8002F03FF801F0EFBA472A98
:10C2C80001F0DE80C1F0D980802A41F0E582694B17
:10C2D80000221A7601F0E2BA892A01F0B88114D84E
:10C2E800852A01F01C8109D8832A01F0E08001F237
:10C2F800FD80604B02221A7601F0D0BA872A01F03D
:10C308006B8141F2108101F049B98D2A01F0F38166
:10C3180006D88B2A01F0C58141F2B08101F0C6B977
:10C32800F22A01F02C82FF2A01F069828E2A41F05C
:10C33800B38201F06DBAB37893B90020012103F0FC
:10C3480069FBD6F80310B07803F074FAB3784A4959
:10C358000022CA544949CA5401F0A0BAB2783AB383
:10C368000423237001F09ABAAD78404E002DF7D11E
:10C378002846012103F04EFBD6F80310B078494255
:10C3880003F058FAB3783C4AD5543C4AD55401F0E6
:10C3980085BAB578002DE3D1284602F015FA03F0E6
:10C3A80031FFB378344AD554344AD55401F076BABB
:10C3B8002E4A5278032A00F2C580DFE802F00222F2
:10C3C80061890020FEF704FB10B9B078FEF7F2FA95
:10C3D800AB78294A0024D454284AD45403F0FCFCEE
:10C3E80020B1224B2146987803F014FBA878D5F8A1
:10C3F800031003F07BFAA878002103F00BFB01F08F
:10C408004DBA0020FEF7E4FA10B9B078FEF7D2FA78
:10C41800AB78194A0024D454184AD45403F0DCFCED
:10C4280020B1124B2146987803F0F4FAAC78114BFE
:10C438000E4E1B5D012B0AD005D3022B10D12046CE
:10C44800FCF724F906E0204603F04CFB02E0204606
:10C4580003F062FBD6F803100144204603F046FAC5
:10C46800A878002103F0D6FA01F018BA6830012044
:10C47800DC300120E0460020D8290120B529012020
:10C48800142B3FF76DAF0020FEF7A2FA10B9B07871
:10C49800FEF790FAAB78CC4A0024D454CB4AD45453
:10C4A800D5F803201344CA4A52F8236003F094FCD9
:10C4B80020B1C84B2146987803F0ACFAA8783146E9
:10C4C80003F014FAA878002103F0A4FA01F0E6B901
:10C4D800142B3FF745AF0020FEF77AFA10B9B07871
:10C4E800FEF768FAAB78B84A0024D454B74AD45453
:10C4F80003F072FC20B1B74B2146987803F08AFA12
:10C50800A878B54BB34C1B5C012B08D004D3022B85
:10C5180012D1FCF7BBF804E003F0E4FA01E003F001
:10C52800FBFAA378D4F80310A94A194452F8211049
:10C538000144184603F0DAF9A878002103F06AFAF2
:10C5480001F0ACB903230B7001F0A8B9FEF734FC75
:10C5580001F0A4B9FFF73CF801F0A0B9B3781BB11A
:10C5680004230B7001F09AB973788C2B00F08D803E
:10C5780030D80D2B18D80C2B68D2052B5AD007D8D9
:10C58800042B40F0BA80002003F05CFB01F086B970
:10C59800062B54D0072B40F0B0804A208F49012247
:10C5A800FDF731FC01F07AB91C2B5AD008D8192BA9
:10C5B80053D01A2B40F0A18005F026F801F06EB98F
:10C5C800702B52D0822B40F09880002003F044FB5F
:10C5D80001F064B9C92B7BD019D8C22B63D00BD812
:10C5E800B52B59D0C12B40F0888048207C490122C6
:10C5F800FDF709FC01F052B9C32B5BD0C82B7CD1E5
:10C608005F2078490122FDF7FEFB01F047B9D42BE2
:10C6180065D004D8CC2B54D0D22B59D06DE0D62B72
:10C6280064D0FE2B69D14C206F490122FDF7EBFB4A
:10C6380001F034B9002003F0FBFA01F02FB94920CA
:10C648006A490122FDF7DFFB01F028B94D2068494E
:10C658000122FDF7D8FB01F021B904F0CDFF01F06C
:10C668001DB904F0D9FF01F019B903F0AFFB02A915
:10C67800B37841F8080DB4205843694600F5867030
:10C688000422FDF7C0FB01F009B94B2059490122EA
:10C69800FDF7B9FB01F002B9582057490422FDF70C
:10C6A800B2FB01F0FBB8402054490422FDF7ABFB74
:10C6B80001F0F4B8442052490422FDF7A4FB01F02C
:10C6C800EDB84E204F490222FDF79DFB01F0E6B878
:10C6D80050204D490422FDF796FB01F0DFB85420A5
:10C6E8004A490422FDF78FFB01F0D8B85C2048497D
:10C6F8000222FDF788FB01F0D1B80323237001F073
:10C70800CDB8A878334E18B104230B7001F0C6B821
:10C7180073788C2B00F0BE8034D80D2B1AD80C2BD4
:10C7280080F09E80052B00F0908006D8042B40F006
:10C73800F98003F0A3FA01F0B1B8062B00F0898064
:10C74800072B40F0EF804A2024490122FDF7E6FB41
:10C7580001F0A4B81C2B00F08E8009D8192B00F02A
:10C7680086801A2B40F0DE8004F06EFF01F096B848
:10C77800702B00F08480822B40F0D48003F086FA7E
:10C7880001F08CB8C92B00F0A88043D8C22B00F068
:10C798008F800CD8B52B00F08480C12B40F0C2806C
:10C7A80048200F490122FDF7B9FB01F077B8C32BE8
:10C7B80000F08580C82B40F0B5805F200949012230
:10C7C800FDF7ACFB01F06AB8D8290120B529012092
:10C7D8007430012068300120E0460020E62901205D
:10C7E800E4290120FB290120E8290120E52901206D
:10C7F800E9290120E7290120F4290120DC29012069
:10C80800E0290120EA290120EC290120F029012052
:10C81800F8290120D42B77D004D8CC2B56D0D22B92
:10C828005BD07FE0D62B76D0FE2B7BD1AA4C4C2058
:10C8380004F10C010122FDF771FBB07804EB401400
:10C84800217B03F045FA01F029B803F00FFA01F053
:10C8580025B84920A1490122FDF760FB01F01EB867
:10C868004D209F490122FDF759FB01F017B804F04C
:10C87800E3FE01F013B804F0EFFE01F00FB84FF437
:10C88800867069460422FDF749FB009803F098FA80
:10C8980001F004B84B2093490122FDF73FFB00F05B
:10C8A800FDBF582090490422FDF738FB00F0F6BF81
:10C8B80040208E490422FDF731FB00F0EFBF4420F1
:10C8C8008B490422FDF72AFB00F0E8BF4E20894976
:10C8D8000222FDF723FB00F0E1BF7F4C042204F1A4
:10C8E80010015020FDF71AFBA87804EB4013D97CFF
:10C8F800FBF748FFA87804EB4014216921F07F4139
:10C90800FBF722FF00F0CABF54207B490422FDF741
:10C9180005FB00F0C3BF5C2078490222FDF7FEFA50
:10C9280000F0BCBF0323237000F0B8BFFFF786FAFE
:10C9380000F0B4BFB278724B022A00F0AA80032A32
:10C9480000F0AC80002A40F00E815B78512B71D04A
:10C958002CD8472B5CD014D8432B52D00BD8412B62
:10C9680049D04AD8402B40F0FC8040F2FF70FDF7D8
:10C97800CFFA6060F9E0452B624A45D046D8D369C2
:10C988003DE04C2B4DD008D8492B47D042D34B2BF8
:10C9980040F0E7805B4BDB7831E04F2B44D046D842
:10C9A8004D2B40F0DE80574B5B7D28E0812B52D029
:10C9B80013D8552B45D005D8532B524A3DD03ED8D5
:10C9C800136A1CE0582B3FD0802B41D0572B40F0E6
:10C9D800C8804C4B93F8273011E0852B45D004D8FC
:10C9E800832B3ED03FD8484BB3E0FE2B48D04AD8E3
:10C9F800F02B45D0B5E0434B43E0424B5B78636096
:10CA0800B3E0404B1B79FAE75379F8E7D368F6E7C8
:10CA18003C4B95E03B4B93F82630F0E7394BDB7DF8
:10CA280033E0384B9B78EAE7364B5B7EE7E7354BDC
:10CA38009B7DE4E7334B1B7DE1E71369DFE7937EDA
:10CA4800DDE7304BDB7EDAE72E4B93F82830D6E76C
:10CA58002D4B1B7ED3E72C4B1B7E181F43424341B3
:10CA6800CDE7294B69E0294B65E0274A28499368B7
:10CA78004B4303F540533933936023F00043BEE73B
:10CA8800244B1B78BBE7244B1B78003318BF0123CA
:10CA9800B5E75A78214B53F82230B0E75B78282B5A
:10CAA80050D00FD8022B4AD005D8002B42D0012BEA
:10CAB80057D11B4B41E0092B57D0272B51D1184B8D
:10CAC800DB689CE72B2B43D02CD8292B3DD02A2B75
:10CAD80047D1134B9B6992E7DC290120E529012006
:10CAE800E9290120E7290120F4290120DC29012076
:10CAF800E0290120EA290120F0290120F829012054
:10CB08006830012004000020E0460020D8300120D1
:10CB18006D4EC641302A0120D6300120E830012070
:10CB2800002A01202D2B19D015D32E2B19D1A14B5A
:10CB38009B6A64E79F4B1B6861E75B685FE79D4BF7
:10CB48009B685CE79B4B1B6959E79A4B5B6956E707
:10CB5800984BDB6953E7974B1B6A50E7954B5B6A29
:10CB68004DE7032300E004232370934B1B78002B2D
:10CB780000F09486914B62681A60914B2AB91A6842
:10CB880042F008021A6000F089BE1A6822F0080212
:10CB98001A6000F083BEB378022B15D17378372B57
:10CBA8000ED8884903F5A770800001EB83010422A1
:10CBB800FDF729F900F072BE7278142A40F2CB8290
:10CBC8000323237000F06ABE04230B7000F066BED6
:10CBD800B378022B0ED17C4B5B78372BF0D8794990
:10CBE80003F5A770800001EB83010422FDF796F995
:10CBF80000F054BE04230B7000F050BEB378002B35
:10CC08007FF4AEAB7378012B0DD007D3022B0FD175
:10CC1800002001F0E1FD606000F040BE002001F05E
:10CC2800CBFD00F03BBE002001F0CEFD00F036BE8B
:10CC380003230B7000F032BEB27812B1022A05D07D
:10CC48001CE01846FBF7E0FC00F028BE5E4A50786E
:10CC5800072808D81BB9FBF7E6FB00F01FBEFBF757
:10CC680007FC00F01BBEFF28AAD1591C0ABF534B72
:10CC7800D8B21878FBF720FC00F010BE04230B7024
:10CC880000F00CBEB378012B23D005D3022B24D19E
:10CC98007078FBF759FC0DE07078082802D8FBF78C
:10CCA8001CFC07E00A2801D100230BE00B2803D164
:10CCB800FBF742FD606012E00C2805D1434B1B696D
:10CCC800C3F3C00363600AE0FF2808D1FBF770FCD8
:10CCD800F0E77078FCF7C8FEECE704230B70364BDE
:10CCE8001B78002B00F0DA85344B62681A60344BED
:10CCF8002AB91A6842F008021A6000F0CFBD1A6813
:10CD080022F008021A6000F0C9BD71782B4A09297F
:10CD180025D8DFE801F005080B0E12181B1E212389
:10CD280011680B441AE01168CB1A17E011684B43DD
:10CD380014E0116891FBF3F310E0116891FBF3F034
:10CD480003FB10130AE011680B4007E011680B435E
:10CD580004E011684B4001E01368DB43136012687C
:10CD6800174B2AB91A6842F008021A6000F096BDFB
:10CD78001A6822F008021A6000F090BD0F4A126883
:10CD88009A420F4B196804DD21F0030141F00401B8
:10CD980008E00BBF21F0060121F0050141F0010177
:10CDA80041F0020119609AB91A6842F008021A6043
:10CDB80000F074BD002A0120D7300120C8300120BE
:10CDC80070300120E8300120683001200000024066
:10CDD8001A6822F008021A6000F060BD72780C2A06
:10CDE80000F25C85DFE802F0071019222B343E4779
:10CDF8005059626B7400A84A1268120740F14E85B8
:10CE0800A64AD36100F04ABDA34A1268170700F189
:10CE18004585A24AD36100F041BD9F4A1268D607F2
:10CE280040F13C859D4AD36100F038BD9A4A1268AA
:10CE3800D50700F13385994AD36100F02FBD964A92
:10CE48001268540740F12A85944AD36100F026BD40
:10CE5800914A126812F0050F00F020858F4AD361BD
:10CE680000F01CBD8C4A1268900740F117858B4A68
:10CE7800D36100F013BD884A1268910700F00E854F
:10CE8800864AD36100F00ABD834A1268D20640F18F
:10CE98000585824AD36100F001BD7F4A1268970672
:10CEA80040F1FC847D4AD36100F0F8BC7A4A1268EC
:10CEB800560640F1F384794AD36100F0EFBC764A14
:10CEC8001268150640F1EA84744AD36100F0E6BCA2
:10CED800714A1268D40540F1E184704AD36100F0C8
:10CEE800DDBC116A072900F2D984481C1062D06998
:10CEF80002EB81014862D36100F0D0BC126A674B33
:10CF0800002A00F0CB84013A1A6203EB8202526ACB
:10CF1800DA6100F0C3BC73782E2B04D8604A012173
:10CF2800D15400F0BBBCFF2B7FF44AAE5B4B01220F
:10CF380083F8442000F0B2BC73782E2B04D8584AEA
:10CF48000021D15400F0AABCFF2B7FF439AE534B1B
:10CF5800002283F8442000F0A1BC504C94F84520EE
:10CF680082B9581C4FF00A0204D14E4B1B685A4331
:10CF7800A26401E05343A364FBF774F90123E0645E
:10CF880084F845306B78042B00F28884DFE803F0DE
:10CF980003436EAE1900FBF765F9E26CA16C801AC9
:10CFA80080EAE072A2EBE0728A423C4B04D900228C
:10CFB80083F8452000F072BCDA69013ADA6100F0C2
:10CFC8006DBCA87801F008FC40B9334B84F84500E3
:10CFD8001A6822F010021A6000F060BCA36C2F4D92
:10CFE800A3B1FBF73FF9EB6CAA6CC01A80EAE073B7
:10CFF800A3EBE073934209D9002385F84530264B0B
:10D008001A6842F010021A6000F048BCE369013B5C
:10D01800E36100F043BCA87802F0F8FD064648B189
:10D02800002384F845301C4B1A6822F010021A605D
:10D0380000F034BCA36C194D9BB1FBF713F9EB6CF2
:10D04800AA6CC01A80EAE073A3EBE073934208D994
:10D05800114B85F845601A6842F010021A6000F01A
:10D068001DBCE369013BE36100F018BC0E4B5A7E1E
:10D078001E4612B1737EF3B118E0A87802F018FECC
:10D088000028F7D0002384F84530034B1A6822F0B3
:10D0980010021A6000F002BC70300120E046002047
:10D0A800442A0120C830012004000020A87802F09A
:10D0B800FFFD0028E6D0A36C9C4D9BB1FBF7D2F88E
:10D0C800EB6CAA6CC01A80EAE073A3EBE07393429E
:10D0D80008D9002385F84530954B1A6842F01002AC
:10D0E8001A60DBE3E369013BE361D7E3914B5A7EC6
:10D0F8001E4612B1737E9BB10DE0A87802F0E0FDE8
:10D108000028F7D0002384F84530894B1A6822F0AC
:10D1180010021A60C2E3A87802F0D2FD0028F1D00C
:10D12800A36C824D9BB1FBF79DF8EB6CAA6CC01AFF
:10D1380080EAE073A3EBE073934208D9002385F8F3
:10D1480045307B4B1A6842F010021A60A6E3E36987
:10D15800013BE361A2E3B17899B9774941F82230FC
:10D16800744B9B7E002B00F09983002A00F0968375
:10D1780002F2851001EB820180000422FCF743FED5
:10D188008CE3FF297FF4ECA862B94FF4C3646B49C0
:10D198002046214404220434FCF735FEB4F5CD6F53
:10D1A800F5D17BE3644902F2851001EB820180002E
:10D1B8000422FCF728FE71E37378142B3FF600ADC8
:10D1C8005F4A9278B2B95C4A52F823205D4B4A60B4
:10D1D8001B78002B00F062835B4B1A60544B22B91A
:10D1E8001A6842F008021A6058E31A6822F0080226
:10D1F8001A6053E3FF2A7FF4B3A863B94FF4C364FA
:10D208004E492046214404220434FCF787FEB4F535
:10D21800CD6FF5D142E3484903F28510800001EB58
:10D2280083010422FCF77AFE38E37678142E3FF661
:10D23800C7ACA878424F010619D5C20704D502F039
:10D248006BFC3D4B43F826003A4B9B7E002B00F0CD
:10D2580025836B78002B00F02183374903F2851072
:10D26800800001EB83010422FCF7CDFD16E30028C2
:10D278007FF476A802F050FC2E4B2F4A9B7E42F892
:10D288002600002B00F00A837B78002B00F0068331
:10D29800B97803F285100844194402EB8101800033
:10D2A8000422FCF7B0FDF9E27278274B0A2A54D819
:10D2B800DFE802F0060B11161C24292E33384E0025
:10D2C80022491A6809680A4403E020491A6809686B
:10D2D800521A1A6041E01D491A6809684A43F8E77A
:10D2E8001A491A68096892FBF1F2F2E7174A1968B5
:10D2F800126891FBF2F002FB1012EAE7134A116878
:10D308001A680A40E5E7114A11681A680A43E0E713
:10D318000E4A11681A684A40DBE70C4A1168C9438B
:10D3280011601AE01A6809490A6016E0E046002010
:10D33800703001200400002074300120602A012090
:10D3480068300120D7300120C8300120E4300120A6
:10D35800A54A18681168106019601A68A34B22B9A9
:10D368001A6842F008021A6098E21A6822F0080265
:10D378001A6093E29E4B1B68C6F80330FDF71CFD4C
:10D388008CE29B4B1B68C6F80330FEF757FD85E21D
:10D398007378052B00F28282DFE803F003090F158A
:10D3A8001B21924B1A6802F00F021A6076E28F4B2B
:10D3B8001A6822F010021A6070E28C4B1A6822F088
:10D3C80020021A606AE2894B1A6822F040021A6049
:10D3D80064E2864B1A6822F080021A605EE2834B90
:10D3E8001A6822F480721A6058E272782E2A3FF680
:10D3F800E7AB804901EB820213654FE27D4B7C4924
:10D40800D3F80C210A60D3F8102177490A60D3F8C1
:10D4180014217649DA61D3F818210A60D3F81C215F
:10D42800754983F84520D3F82021DA64D3F82421FC
:10D438009A6493F82821885C08B101208854002256
:10D4480083F82C212AE2B378002B7EF489AF737815
:10D45800142B3FF6B5AB664A1168684A42F82310A8
:10D468001CE200F05DFF19E200F067FF16E200F031
:10D4780065FF13E200F063FF10E200F061FF0DE2C8
:10D4880000F05FFF0AE2727812B1012A04D00BE0C3
:10D49800584B01221A7601E2B3F5006FBEF460AF73
:10D4A80054490A76CB61F9E103230B70F6E1514B3D
:10D4B800002183F8441083F82C114E4A4FF0FF30B6
:10D4C80002F1500343F821004B4800234354013133
:10D4D8002F29F2D11376D361136282F84530444A7A
:10D4E8001360414A1360414A1360D7E1444B1B7DE6
:10D4F8009B0711D404F0C0F810B90A232370CDE1BA
:10D50800D6F803100423B1F5006F37BF394A2370EA
:10D518001376C2F83011C1E108230B70BEE1354B18
:10D5280000221A76BAE1374A01251570344A364C7A
:10D538009178B3F5006F217026D2127D12EA0506A4
:10D5480022D118466946FCF737FB9DF80030267251
:10D5580063709DF80130A3709DF80230E3709DF868
:10D56800063023719DF8053063719DF80430A3716E
:10D578009DF80330E3712B46E15C227A01330A44BB
:10D58800082B2272F8D189E101230021E1540133EB
:10D59800082B1D4AF9D1137813727FE1737883B988
:10D5A800184A012111701649174A897811701749CC
:10D5B80008680133C11811F8011C082BD154F8D19F
:10D5C8006CE1012B40F06A810522CA714B711F2260
:10D5D8000B238A710B7161E17378032B00F25E8172
:10D5E800DFE803F016222D31E430012070300120ED
:10D5F800C8300120E0460020442A01207430012070
:10D6080004000020CC300120CD3001200000002093
:10D61800A34B1A7ECA7193F84520D3F830318A712A
:10D628001A0A4A710B7139E19D4B1A7ECA7193F837
:10D638004520DB698A711A0A4A710B712EE1994BF0
:10D648001B684B602AE1984B1B684B6026E1727897
:10D65800002A40F02381B178002940F01F8140F270
:10D66800D242934240F01A8140F2FF70FCF768FB07
:10D67800FCF7BEFA0120FBF7B3FA0FE172788B4B87
:10D6880002B101221A70EA78894B1A70844B93F818
:10D698003421884B1A70884A00231370874A137004
:10D6A800FCE07F4B012283F83521F7E06D78844E4A
:10D6B80015B1012D0FD01BE0042240F2FB70694622
:10D6C800FCF72CFC009BD6F803209A4206BF0123E6
:10D6D80063606560E2E0B3782A2B06D140F2FB7004
:10D6E800F11C0422FCF78FFBD8E003230B70D5E074
:10D6F80003230B70D2E07278032A3DD8DFE802F0EA
:10D7080008022E3966480022D0F83811054610E084
:10D71800634AD2F83811092907D8481CC2F83801D9
:10D7280002EB8102C2F83C31B8E009232370B5E06E
:10D7380001328A4200F0B2806248960050F82240D6
:10D748009C42F5D18319481E824204D25C6801329A
:10D7580043F8044BF7E7C5F838019FE0504A002327
:10D76800C2F83831574A002199500433282BF9D18F
:10D7780094E00A234B6091E003230B708EE07378EA
:10D78800812B40F08B80B2784D4B922A40F08680F6
:10D798009A79A32A40F082805A79B42A7ED11A79DC
:10D7A800C52A7BD1DB78D62B78D1474B04221A8344
:10D7B800FDF7FCFAFAF756FD0446FAF753FD001B8D
:10D7C8000028B8BF4042B0F57A7FF6DB72B6FBF7A7
:10D7D80015FA3E4B00241C6021463D4805F0F3FA3B
:10D7E8003B4805F02FFA04F0D7FC05F0C3FB4FF0D7
:10D7F800804006F049F92046FBF7F2F94EE040F286
:10D80800D24293424AD1264B012283F8642145E053
:10D81800B17831B12A4A5278033AD2B2012A3EF697
:10D828009FAD6A780A2A34D8DFE802F0060A0E1299
:10D83800171C1F23272B2F0004F032FB60602DE0FC
:10D8480004F031FB606029E004F030FB606025E003
:10D85800184604F02DFB606020E00846194604F0E5
:10D8680083FB1BE004F092FB18E004F097FB606078
:10D8780014E0184604F098FB10E004F09BFB60608D
:10D888000CE0184604F09CFB08E004F09FFB606085
:10D8980004E00323237001E00223237003B0F0BDEA
:10D8A800E0460020C8300120E4300120A0290120F2
:10D8B800BD2901203A2A0120BC290120732A012010
:10D8C800683001201C4800200010024010E000E0F1
:10D8D800106402403049002370B50B602F49304A6C
:10D8E8000B603049D36113620B6082F8453082F8CF
:10D8F800443082F82C3115462B4A4FF0FF3142F85C
:10D9080023102A4A0020D05401332F2BF4D1284B5E
:10D91800284E197B02F0DCF996F8283013B9FBF78A
:10D928009BF901E0FBF785F90023234A0021995070
:10D938000433B3F5806FF8D1B37E13B9F37E6BB1BE
:10D9480018E04FF4C3641D492046214404220434DE
:10D95800FCF7E4FAB4F5CD6FF5D1EFE74FF4A7641F
:10D9680017492046214404220434FCF7D7FAB4F5B9
:10D97800C36FF5D1337903F0EF02012A01D0212BCF
:10D9880001D1012300E0002385F86531737D03B1DF
:10D9980001232B7670BD00BFC8300120E430012080
:10D9A800E04600207030012030470020442A012042
:10D9B800DC29012004000020E8300120602A012031
:10D9C800B02B0120F7B50F4E0F4CC6F803300F4BA4
:10D9D80086460F46B270002294E803001A708DE85C
:10D9E800030086F800E07770FEF7D0FB21786368C3
:10D9F800074A82F866119DE8030084E80300184688
:10DA080003B0F0BD68300120DC300120D7300120A0
:10DA1800E0460020014B93F866017047E04600207D
:10DA2800F7B51F4E024653780C4696E803008DE87A
:10DA380003001C4900270B7093786D464B70D37810
:10DA48008B7013798B7153794B7193790B71D379EF
:10DA5800CB70154B1F70FEF799FB144B19783346A2
:10DA680071B9217032786170A2707278E270F279BF
:10DA78002271B27962717279A2713279E27109E028
:10DA8800012907D13A460A4911444978A15401327B
:10DA9800082AF8D195E8030083E8030003B0F0BD35
:10DAA800DC30012068300120D7300120CC30012043
:10DAB800CD3001202DE9F04FAF4B95B01B78AF4C1E
:10DAC80013B994F8673163B1AD4B1B78062B08D0B6
:10DAD8000A2B06D003F0EF030F2B1CBF002384F89A
:10DAE800343194F83431A54A591EC9B20129A54EDA
:10DAF8003BD8A549012BCA6814BF082307238DF812
:10DB0800303094F868310D9232788DF83130002336
:10DB18008DF83230C2B98B688DF83F208DF83830D7
:10DB28009A4B19788DF8391059788DF83A10D979B7
:10DB38008DF83B1099798DF83C1059791B798DF83F
:10DB48003D108DF83E3009E0012A07D19049013394
:10DB58000CAA595C1A44082BD171F7D10CA8FBF711
:10DB68006BFD002800F0A683ACE0032B2AD192F8C5
:10DB780065511DBB33788BB9834F844DB87897F8BE
:10DB880001802A78804490446A789044EA799044E5
:10DB9800AA7990446A7990442A7920E0012B40F0D0
:10DBA80091807B4B585D0135FBF784FA092DF8D13C
:10DBB80088E0072B63D192F8653173B3734801F09D
:10DBC800AFFB7FE0042BF4D16F4F704DB87897F816
:10DBD8000180002301226B702A706B60804490449E
:10DBE800FBF768FA7878FBF765FA2878FBF762FAAA
:10DBF8006878FBF75FFAE879FBF75CFAA879FBF736
:10DC080059FA6879FBF756FA5FFA88F82879FBF72A
:10DC180051FA4046FBF74EFA54E032782ABB5A4B89
:10DC280093F802E093F801C0584B8DF818E01F787C
:10DC38005D78E644D8798DF81A70774499798DF82B
:10DC48001B503D445A798DF81C0028441B798DF8E7
:10DC58001D1001448DF81E200A448DF81F3013440E
:10DC68008DF819C08DF8203028E0012A26D1484ABD
:10DC780006A99A5CCA540133092BF8D11EE0082B77
:10DC880020D1424A002301205370107053603E4A4D
:10DC98008DF81A00917852788DF818108DF819209F
:10DCA8000A4402448DF81B308DF81C308DF81D3065
:10DCB8008DF81E308DF81F308DF8202006A8092118
:10DCC800FDF722F8334B1A789846002A00F08C802A
:10DCD800314B324D1B78013B062B00F28180DFE887
:10DCE80003F00404257F7F7F5F00274A2978936823
:10DCF8008DF84E108DF8483080238DF849308A23EE
:10DD08008DF84A3000238DF84B308DF84C308DF863
:10DD18004D308DF841308DF84230D368072110A876
:10DD28008DF840101193FBF787FC59E0164F2A78BD
:10DD3800B87897F80190814409F10A099144FBF7F2
:10DD4800B9F97878FBF7B6F98020FBF7B3F98A20A0
:10DD5800FBF7B0F90020FBF7ADF90020FBF7AAF9B3
:10DD68000020FBF7A7F95FFA89F92878FBF7A2F9F1
:10DD78004846FBF79FF933E0D6300120E046002003
:10DD880068300120CC30012004000020DC30012064
:10DD9800CD300120732A01203A2A0120BC29012014
:10DDA800B54B2A789878597880238DF82510014446
:10DDB8000A318DF826308A238DF824008DF8273013
:10DDC8008DF82B2000230A4409A809218DF8283052
:10DDD8008DF829308DF82A308DF82C20FCF794FF27
:10DDE80000232B7088F80030002384F83431337016
:10DDF80084F8673194F8643113B10120FAF7F0FE22
:10DE080094F835219D4B52B193F86521D2F1010266
:10DE180038BF002283F86521002283F835210CA839
:10DE2800FBF758FC002840D09DF83030062B3CD931
:10DE3800934B9DF838201A709DF839205A709DF838
:10DE48003A209A709DF83B209A719DF83C205A71AF
:10DE58009DF83D201A719DF83E20DA709DF831300A
:10DE680084F86831844B1A690D9B934203D1834B24
:10DE7800012283F86721FAF7F5F9824B002218602E
:10DE8800814B1A709DF83030227E072B0CBF01237E
:10DE9800022384F83431531EDBB2012B7B4B02D9A9
:10DEA800052A40F0CB800022E3E094F86551002D6C
:10DEB80071D109A8FBF718F900286CD0FBF732F9E3
:10DEC80010B16E4B83F8695194F869119DF82400DC
:10DED8004A1CD2B22144092A684B84F8692181F886
:10DEE8006A0140F0DB80002283F86921624A93F8D6
:10DEF8006A315178994207D092F82710002900F02A
:10DF0800CD808B4240F0CA8092F827209A4204BF05
:10DF1800012384F8673100231A46584D05F5B57179
:10DF2800595C01330A44082BD2B2F6D195F8723104
:10DF380093422CD1524B95F86B211A7095F86C21AD
:10DF48005A7095F86D219A7095F86E219A7195F826
:10DF58006F215A7195F870211A7195F87121DA704C
:10DF6800FAF780F94A4B4B4A1860297E0023137050
:10DF7800032285F834214A1ED2B2012A85F8693174
:10DF8800424A02D9052918BF0123137086E00423E9
:10DF980085F8343182E094F86531384D7BB13848E2
:10DFA80001F071F858B1FAF75DF9394B394A186040
:10DFB80000231370032285F834212A7E36E094F872
:10DFC8006561002E41D110AD2846FCF7C7FE002838
:10DFD8003BD033463246E95C01330A44082BD2B2BF
:10DFE800F9D19DF8481091422CD1254B9DF841203C
:10DFF8001A709DF842205A709DF843209A709DF837
:10E0080044209A719DF845205A719DF846201A714E
:10E018009DF84720DA70FAF725F91D4B1D4A18605C
:10E0280000231370072284F83421227E511EC9B2BE
:10E0380001291946154B03D9052A01D0012218E0F8
:10E0480019702BE084F8343128E0237E0B4D013B16
:10E05800DBB2012B22D8E869B0F5006F1CD2431C53
:10E068000749EB61FBF7A8FD092385F83431074B15
:10E0780001221A7012E000BF04000020E0460020D0
:10E08800683001202C2A012098290120D73001204E
:10E09800342A0120392A012000232B76237E874D3C
:10E0A800042B04D1864E3278130640F1D98094F8B7
:10E0B800343113F0FB0F05D0082B03D0062B01D009
:10E0C800FEF764F894F83431092B0BD07B4B93F8A6
:10E0D8003401092840F0AA801A7E022A04BF0522CA
:10E0E8001A76A3E0FAF7BEF8744A764DD2682B6820
:10E0F800801A80EAE072A2EBE0729A4208D9724B69
:10E108001A78012A04BF02221A70FAF7ABF8E06005
:10E11800FAF7A8F823696A68C01A80EAE073A3EBE3
:10E12800E073934208D9684B5A78012A04BF022247
:10E138005A70FAF797F82061FAF794F86369AA68B1
:10E14800C01A80EAE073A3EBE073934208D95E4BF0
:10E158009A78012A04BF02229A70FAF783F860615C
:10E1680094F84420554B002AB0D093F82C21002A6B
:10E17800ACD15649DC6C0968049401915449D3F830
:10E188001C410968D3F80C9102915249D3F81081C7
:10E198000968D8690391996CD3F814C10591D3F82B
:10E1A800187193F845100094D3F82061D3F82451DE
:10E1B80093F828411346DFF810A11AF803B0BBF111
:10E1C800020F18D1DFF814B15BF823B0BBF1FF3FA1
:10E1D8000DD000918446DCB2059D049E039F5846ED
:10E1E800DDF80880DDF804900122002103E04FF0FB
:10E1F800000B0AF803B001332F2BDCD12F4B83F827
:10E2080045100099C3F80C91C3F81081D861C3F880
:10E2180014C1C3F81871C3F81C11C3F82061C3F8FE
:10E22800245183F8284183F82C214FE7D3F838216B
:10E238002249002A3ED009283CD10B7E012B39D136
:10E24800C86900231D4901F59E7454F82340A04273
:10E2580002D105230B762DE001339342F2D129E058
:10E2680095F8343113F0FB0F24D0082B22D0062B5D
:10E2780020D0D5F83001184CD6F80330B0F5006F2F
:10E288006270636012D23146FBF794FDD5F8300115
:10E298003146FBF7FDFC30B1D5F830310133C5F814
:10E2A8003031652300E00723237003E00723237040
:10E2B80000232B7615B0BDE8F08F00BFE0460020A4
:10E2C80068300120002A0120442A0120C83001209A
:10E2D800E430012070300120DC300120304700207C
:10E2E800704710B5F9F7BEFF074C2368C01AB0F5A0
:10E2F800FA7F07D9054B5A6982F040025A61F9F74B
:10E30800B1FF206010BD00BFE834012000100240BA
:10E3180008B5FAF749FC014B586008BDDC3001200C
:10E32800044BD3F8030008B9FAF79DBD0020FAF7AB
:10E3380097BD00BF6830012070477047704770472D
:10E34800704770472DE9F047B74B04465B7E6BB9C1
:10E3580001F0AEFC10F10009204618BF4FF001098A
:10E3680001F0AEFC003018BF01200DE001F0A0FC68
:10E37800D0F10109204638BF4FF0000901F0A0FC98
:10E38800D0F1010038BF0020A84E650173191B7A2F
:10E3980013F0800F03F07F08A54B1B6914BF83F4AB
:10E3A800806AC3F3802A08F1FF33DBB218BFCAF3CF
:10E3B800802A092B00F2FC81012202FA03F313F4EC
:10E3C800407F40F0AF8113F0F00F40F0C7801B078B
:10E3D80000F0EE81974F3B5D013B0E2B00F2E88188
:10E3E800DFE813F00F00F0002B00120135003E00AB
:10E3F800460056007C0095009A00E601B20096019E
:10E40800B900204601F0BAFB35446B7B07EB840763
:10E41800786001212046BB6001F0FCFAA8F10208EF
:10E428005FFA88F8B8F1010FDFF8089294BF022369
:10E43800042309F80430BDE8F087002800F0B8810B
:10E44800204601F069FB7C4B43F8240090E1B9F1C8
:10E45800000F00F0AD81204601F020FC0623A6E164
:10E46800354400226A732046696801F0E3F9F7E051
:10E47800B9F1000F40F09C8120464946354401F02F
:10E48800D9F969682046494201F0D4F908238EE198
:10E49800B9F1000F00F08C81204601F03DFB00210E
:10E4A8008046204601F0C6F9634B354453F82420D2
:10E4B8004FF00009C8EB02022046696885F80D9004
:10E4C80043F8242001F086FA2046414601F00EFA6E
:10E4D8002046494601F09EFA092368E1204601F0EA
:10E4E80095FB002800F06481A8F1030801F08AFE7A
:10E4F8005FFA88F8002001F0E5FDB8F1010F00F29D
:10E5080047812046012101F085FA3544BBE0B9F185
:10E51800000F00F04D81C7E0B9F1000F40F04881CD
:10E52800204601F0F9FA49468046204601F082F972
:10E5380035440221204698FBF1F185F80D9001F051
:10E54800D5F920464946CBE0204601F05FFB00287C
:10E5580000F02E811CE101F055FE19E1354F3B5DBD
:10E56800013B0E2B00F22481DFE813F00F00290095
:10E578003B004B00680022017C002201220194002C
:10E58800A0008600BD00D200C900204601F0F6FABE
:10E59800354407EB84036A7B5860012120469A6062
:10E5A80001F038FAB8F1060F00F0DD80B8F1080F75
:10E5B80000F0D9801F4B04221A55BDE8F087B8F146
:10E5C800060F02D17319022204E0B8F1080F02D134
:10E5D800731900225A732046715901F02BF903234D
:10E5E800E5E0A8F10503DBB2012B04D818B1B8F1B6
:10E5F800060F2FD1BCE0BAF1000F00F0D9800C2330
:10E60800D5E0B8F1050F02D17319012204E0B8F181
:10E61800070F02D1731900225A73715920464942D3
:10E6280001F008F90523C2E004000020DC290120DC
:10E63800000C0240544800209C290120A8F1050341
:10E64800DBB2012B08D8B9F1000F05D0B8F1050FDE
:10E6580000F089800F23AAE0BAF1000F00F0A8802B
:10E668000723A4E0BAF1000F40F0A280354402234A
:10E678006B732046696809E0BAF1000F40F0988092
:10E68800354401236B7369682046494201F0D2F88A
:10E698000A238CE0BAF1000F00F08A80204601F0CE
:10E6A8003BFA07EB8403D8600B2380E0BAF1000F34
:10E6B8007ED1204601F030FA35448046696820460C
:10E6C80085F80DA001F086F907EB8403DB680221C9
:10E6D8009844204698FBF1F101F008F9204651468C
:10E6E80001F098F94EE0204601F090FA00285FD03A
:10E6F8000E233B550020BDE8F04701F0E3BC20465F
:10E70800012101F087F92046002101F093F83FE04C
:10E7180007EB84039A6835446A732046596801F008
:10E7280059F943E0234F3B5D013B0E2B40D8DFE80E
:10E7380003F008213F243F3F3F3F3F3F3F3F2B3DF2
:10E74800310020460121354401F064F9E97C204676
:10E7580041F00401FAF716F820460121FAF762F8A9
:10E76800B8F1090F01D1022321E0B8F10A0F1FD136
:10E7780004231CE02046715902E0715920464942A1
:10E7880001F058F80D2312E0204601F077F978B926
:10E798000E230CE02046002101F04CF80E233B55D7
:10E7A80020460021BDE8F047FAF73CB800233B5566
:10E7B800BDE8F08754480020024B1A5C0AB90122D0
:10E7C8001A54704754480020024B1A5C0AB10F22B1
:10E7D8001A54704754480020014B185C704700BF1A
:10E7E80054480020034B00201870034B997AF9F71E
:10E7F80017BE00BF3B2A0120DC290120014B1878F5
:10E80800704700BF64480020014B5878704700BF2C
:10E8180064480020014B9878704700BF6448002086
:10E828002DE9F743974CE37823B96FF00043636011
:10E838000123E370257A944F4DB9E8B2F9F74DFEFC
:10E8480078550135082DF8D18E4B01221A722725EB
:10E858000026F0B2F9F741FEBB5D83421BD08A4B1C
:10E868008A4AF054B31C02EB83035B68022B05D081
:10E87800032B0AD0012B0ED168B106E058B9844A9F
:10E88800515D012907D1535505E0814B5A5D012A95
:10E8980004BF02225A550136082E05F10105D8D1C8
:10E8A8007C4D6B7E13B16B7EC3B107E0607C01F0D9
:10E8B800FFF90028F7D0A37C33B111E0607C01F0A8
:10E8C800F7F90028F7D009E06E4B01229A74704BD3
:10E8D800DA7E012A04D10222DA7601E00023A37449
:10E8E8006B7E13B16B7EC3B107E0607C01F0E8F981
:10E8F8000028F7D0E37C33B111E0607C01F0E0F947
:10E908000028F7D009E05F4B0122DA74604B1A7FC8
:10E91800012A04D102221A7701E00023E374EB698B
:10E92800A3B15D4E37788FB9F9F79CFC5B4B594A18
:10E938001B68D269C01A80EAE073A3EBE0739342C4
:10E9480004D9384601F0AAF9012333702B6AA3B120
:10E95800534D2E788EB9F9F785FC524B4D4A1B68FA
:10E96800126AC01A80EAE073A3EBE073934204D9F9
:10E97800304601F093F901232B700820FBF774F857
:10E98800632801D8012305E00820FBF76DF8692802
:10E9980001D9002363700820FBF766F840F21223C0
:10E9A800984201D9012306E00820FBF75DF8B0F58D
:10E9B800027F01D2002323700920FBF755F878283D
:10E9C80001D9012305E00920FBF74EF8592801D8A1
:10E9D8000023A37062782B4B334F1AB91A780AB9FF
:10E9E8009B7813B104233B8301E004237B8302F06B
:10E9F80051FE607C01F0E0F80146224E607C2B4D10
:10EA080000295FD02A4B02221A54FBF7C3FE737CFD
:10EA180005EB4315697AB0EBD10F02D01846F9F728
:10EA2800FFFC0023607C237501F0F0F870B1154BF2
:10EA380017495B7CDA1C885C012804BF02208854D3
:10EA4800012202FA03F3227D1343237519491A4A56
:10EA58000B783BB1207D034204D11370174B1B7810
:10EA680003B90B70137833B1227D1A409A4202D150
:10EA7800134B01221A70002003B0BDE8F043FFF7E2
:10EA880061BC00BF644800206D480020002A0120B6
:10EA9800442A012004000020392A0120342A0120B8
:10EAA800982901202C2A012000100240DC2901208D
:10EAB8003B2A0120BD290120BC290120A0290120D1
:10EAC800732A012005EB401393F80CC0DFF874E2B9
:10EAD8008300974ADFF87082BCF1000F00F0D28003
:10EAE8000244009208EB0002019273440A46FBF7C5
:10EAF800F1FE707C4201AB181B7B013B042B00F23A
:10EB08002D82DFE803F0033A9A3A9A00894B8A4E3D
:10EB18001B6913F0080F04EB00035B7D10D0022B78
:10EB280003D1335C002B00F019821544697AF9F798
:10EB380077FC607CFBF73EFF637C02221C4418E0F4
:10EB4800012B03D1335C002B00F008822A44917A10
:10EB5800F9F766FC607C05EB4015AB7A13B9FBF757
:10EB68001BFF03E0335C0BB1FBF724FF637C01223E
:10EB78001C4462750022F254F0E118F900306E4E20
:10EB8800002B19DB23185B7D022B01D1335C63B1A9
:10EB98002A44517AF9F744FC607CFBF70BFF637C4D
:10EBA8000221E21851750022F254667CF9F75AFBEB
:10EBB80004EB8603586034E02044437DDFF880810D
:10EBC800012B03D1637CF35C9BB92AE0F9F74AFB7C
:10EBD80098F811300A2108EB830205EB43139B8B4D
:10EBE80052684B43801A80EAE072A2EBE0729A42C4
:10EBF800E8DD607C05EB4013997AF9F711FC607C3D
:10EC080005EB40139B7A13B9FBF7C6FE03E0335CB0
:10EC18000BB1FBF7CFFE637C0121E218517500228E
:10EC2800F254637C05EB43152B7B042B40F0968153
:10EC3800404A126912F0080F20E023185B7D3E4E0F
:10EC4800022B01D1335C63B12A44517AF9F7E8FB0E
:10EC5800607CFBF7AFFE637C0221E218517500224D
:10EC6800F254637C05EB43152B7B052B40F0768132
:10EC7800304B1B6913F0080F4FF0040314BF7B835C
:10EC88003B836BE10EEB0301024408EB000300F049
:10EC9800ABFF707C00F0F2FE10BBF9F7E3FA737C6F
:10ECA80006EB830672680A26801A5A01A918898B0E
:10ECB8000028B8BF4042714388425DDD1F491E4E9F
:10ECC800C85C0F4610B9F15C002955D02A44184693
:10ECD800917AF9F7A5FB637C0022FA54F2544BE0D1
:10ECE800707C164F4301EA18D27FDFF84C806AB374
:10ECF80000F0C4FE8146707C00F0A8FE8145707C5F
:10ED08003B5C0CD0032B02D118F800305BB305EB49
:10ED18004013D97FF9F784FB637C032222E0022B9E
:10ED280002D118F80030F3B105EB401315E000BF2D
:10ED3800A829012000000240382A01203B2A01208E
:10ED480064480020C0290120D92901203A5C022A00
:10ED580002D118F8002032B12B44597AF9F760FB38
:10ED6800637C0222FA54667C002308F80630F9F71F
:10ED780079FA04EB86067060607C7A4E05EB4013E6
:10ED88009B69EBB1F9F778FCD0B1707C00F076FEA6
:10ED9800737C754A0028B8BF404202EB431292695F
:10EDA80090420DD9184600F079FF737C6F4A012113
:10EDB800D1546F4A0F33D15C012904BF0221D154C9
:10EDC8000023607C237500F021FF70B1654B684912
:10EDD8005B7CDA1C885C012804BF0220885401226D
:10EDE80002FA03F3227D134323756249624A0B78C2
:10EDF8003BB1207D034204D11370604B1B7803B9EB
:10EE08000B70137833B1227D1A409A4202D15C4BC1
:10EE180001221A70607C00F031FE20B1667C594BEB
:10EE28009B5D33B92AE04F4B587C00F00FFE002859
:10EE3800F4D1637C05EB4312D28912B9514AD35CF1
:10EE480013B3F9F70FFA637C04EB8302926905EBBD
:10EE58004311801AC98980EAE072A2EBE0720A20A5
:10EE680041438A4210DD484EF25C6AB91846FBF706
:10EE780093FD3C4B01225B7CF25405E0F9F7F2F973
:10EE8800384B03EB8606B061607C00F0F7FD3F4E1F
:10EE9800637C0028B8BF404256F83320314F904277
:10EEA80018460AD2FBF73AFC7B7C06EBC30672795C
:10EEB80082420DD11846002108E0FBF72FFC7B7C2D
:10EEC80006EBC3067179884202D01846FBF7F4FBBB
:10EED800F9F7C8F9E369234EC01A80EAE073A3EB97
:10EEE800E0730A2B3ADD707CFFF72CFA707C00F097
:10EEF800C5FD68B3707C1C4F05EB40156B693BB3CF
:10EF080000F00AFE0546707CF9F7C0FB737C281AEE
:10EF180007EB4312526980EAE075A5EBE075002A19
:10EF2800B8BF5242954213DD184600F0B7FE7B6920
:10EF3800002B02DA0020F9F796FF637C144A0121BE
:10EF4800D1540B4A1533D15C012904BF0221D15495
:10EF5800044B00225A74F9F785F9E06103B0BDE863
:10EF6800F08300BF64480020DC290120D829012053
:10EF7800442A0120BD290120BC290120A029012003
:10EF8800732A01203C2A01203D2A0120AC290120B6
:10EF9800B5290120074B10B518681C4601460A78A8
:10EFA8000B4601311AB12C2AF9D100221A7001330B
:10EFB800236010BD8448002070B50646FAF794F81F
:10EFC8000D4C054618B100232371012070BDA368BC
:10EFD800E268934207D25A1C23441B7C01203370F9
:10EFE8002071A26070BD04F11000FBF7A5FEA560BA
:10EFF800E060284670BD00BF8448002010B50D4C65
:10F00800024623791BB9BDE81040FAF753B8206DC2
:10F018000D2A00F101032044236580F8542002D012
:10F028003F2B00D829B919460348FBF76DFE00238A
:10F03800236510BD84480020D848002070B5012100
:10F04800044686B02020FFF7D9FF002C04DA2D20D3
:10F058000121FFF7D3FF644200230A2194FBF1F258
:10F0680001FB124101AE30311D469955144601335A
:10F07800002AF2D1705D0121FFF7C0FF15F1FF35BD
:10F08800F8D206B070BD2DE9F34105460DF1070031
:10F09800FFF792FF974C002800F0C88094F894304E
:10F0A8009DF80700944E03BB7378403398420DD106
:10F0B800D4F89830002B40F0B9803179012331F031
:10F0C800010184F8943040F0B180ADE00D2801D002
:10F0D8001B2801D1002305E0D4F898307E2B00F2DC
:10F0E800A5800133C4F89830A0E0317931F00101EE
:10F0F80001D1FFF783FF9DF807301F2B0CD9D4F8F7
:10F1080098207C497E2A00F28280501C0A44C1F86B
:10F11800980082F89C307AE0082B08D1D4F898300F
:10F12800002B74D0734A013BC2F898306FE00D2B66
:10F138006DD1D4F89830002B69D03379112B16D1C2
:10F148006D4B0121587800274030C0B2FFF756FFB9
:10F15800D4F898309F4206D2684B0121D85DFFF75A
:10F168004DFF0137F4E70D200121FFF747FF00238A
:10F17800D4F898802768C4F81C311A4619464245C5
:10F1880037D0012911D002D3022925D02FE0DFF88A
:10F1980064C10CF19C00105C202828D00CEB030102
:10F1A80081F820010133012121E0524800F19C0C33
:10F1B80012F80CC0BCF1200F0AD1012B04D9184455
:10F1C800002180F8201101334D4F02211F440EE029
:10F1D800184480F820C109E0DFF818C10CF19C0040
:10F1E800105C202803D09C448CF8200101330132A4
:10F1F800C5E70022C4F81C31234483F820210123E9
:10F20800276084F89F3184F89420C4F898209DF8EA
:10F2180007301B2B0AD133790021012BC4F8981031
:10F2280084F8941002D10D20FFF7E8FE94F89F01AE
:10F23800002600285AD02F4B83F89F61F7B2DFF8D9
:10F24800DC80C7EBC70708EB07042D48214608F008
:10F258001FFB28B9A6796379F1072B7036D506E02C
:10F2680018F807300136002BE8D12B703DE0FFF786
:10F2780091FE2B780446042B14D1224908F008FB90
:10F2880008B900230CE020461F4908F001FB08B923
:10F29800012305E01D49204608F0FAFA90B9022337
:10F2A8006B7013E00D2B0ED1194908F0F1FA002804
:10F2B800E7D02046174908F0EBFA0028E8D02046A6
:10F2C8001549E9E7204608F0DFFA6870B20704D567
:10F2D800FFF760FE08F0D8FAA870730705D5FFF7A6
:10F2E80059FE08F0D1FAC5F80300012002B0BDE8C4
:10F2F800F08100BF8448002004000020204900203D
:10F30800A44900201A9701081E97010822970108AE
:10F31800289701082E9701083397010818810108DA
:10F3280038B50D4D0446A87801214030C0B2FFF72A
:10F3380065FE687801214030C0B2FFF75FFE207893
:10F34800FFF77CFE6068FFF779FEBDE838400D20C6
:10F358000121FFF753BE00BF040000200000000099
:10F36800B0F5803F53DBB0F1807F2ADBB0F1805FDE
:10F3780011DBB0F1804F08DB3D4B984244DC3D4B3C
:10F38800021653F822301B0212E03A4B821553F84A
:10F398002230DB010CE0B0F1806F364B04DB021544
:10F3A80053F822309B0103E0821453F822305B01AA
:10F3B8005A1C90FBF3F31A445210531C90FBF2F2C0
:10F3C8001FE0B0F5801F2B4B0CDBB0F5800F04DB82
:10F3D800021453F822301B0110E0821353F8223034
:10F3E800DB000BE0B0F5802F04DB021353F822306A
:10F3F8009B0003E0821253F822305B005A1C90FBFA
:10F40800F3F313445B1021E04FF6FF707047FF28B9
:10F4180022DDB0F5805F174B0BDBB0F5804F03DBC7
:10F42800021253F8223010E0821153F822305B1098
:10F438000BE0B0F5806F04DB021153F822309B100B
:10F4480003E0821053F82230DB10013303FB03F290
:10F45800824208DD581E7047002806DB054B53F82A
:10F46800200000117047184670474FF0FF30704772
:10F478000080FE7FF88101081C4B5A7E1C4BC2B9E4
:10F48800597BCB0709D51B4B1B69180705D51A4BA8
:10F4980018680028BCBF1A605A608B0724D5154B22
:10F4A8001B69D80620D5144B1A68002A1CDD0022D7
:10F4B80018E05A7BD1070AD50E4B196911F00801DB
:10F4C80005D10D4B18680028BCBF19605960930717
:10F4D8000AD5084B1A6912F0100205D1064B1968B3
:10F4E800002901DD1A605A60704700BF040000203F
:10F4F800DC29012000040240244A0020184B10B5E2
:10F508001A7A044662B1FBF755FA164B2046597A27
:10F51800F8F786FF144A00231370144A137010BDBD
:10F528005A7A02F0FF0112B1012912D010BD1A68EF
:10F53800A2B9DA681B699A4210D02046FBF73AFA5A
:10F54800084B2046597AF8F76BFF074B00221A70D0
:10F5580010BD1A6812B95B69002BEED110BD00BF4F
:10F56800244A0020DC2901203D2A01200035012001
:10F5780008B50020FBF796F940B9FBF70BF9013005
:10F5880007F016F80EA3D3E9002308E00020FBF7E4
:10F5980001F9013007F00CF80BA3D3E9002307F0B9
:10F5A8006DF80BA3D3E9002307F092F900220A4B68
:10F5B80007F064F807F0FCFA08BD00BFAFF300805D
:10F5C80049922449924CB14024499224496AA24064
:10F5D8001B0DE02D90A0F63F0000A03F684620F0EC
:10F5E80007018D4631B5194DAB6973B11848012132
:10F5F80004F0B5F90028F9D01548AC6904F077F99A
:10F60800C4F10304C0B22C442077AB690F4C022B21
:10F618000BD8A3690E485A1CC3F10203A2611C440B
:10F6280094F8201004F066F90CE0002208487121D3
:10F6380004F086F9074B10221A83002384F824303B
:10F6480084F82530BDE8314085467047244A0020BB
:10F6580000300140000002401D4B30B50028B8BF03
:10F668004042DD6A40430135DD629A6A1D6B0A211A
:10F67800B2FBF1F490FBF1F1294419636422D96AD1
:10F68800B4FBF2F4A14222DB586B996B03EB8101C6
:10F69800C96B411A5963996B1C6B4FF47A70B4FBB0
:10F6A800F0F003EB8101C863596B986B03EB8000A2
:10F6B800C06B01445963996B01319963996B91FB54
:10F6C800F2F002FB10129A630022DA621A6330BD6C
:10F6D800244A00202DE9F0414D4B1B78002B40F0C7
:10F6E80087804C4A4C4D566AA2F57042526A4B4C80
:10F6F8002A604B4A1360B4F800802A6842F21073FB
:10F708009A421FFA88F807DD23889BB2082B03D991
:10F718002388C3F34E0323802B68B3F57A7F0ADA74
:10F7280022883E4B92B2B2F5804F04D21A8892B228
:10F73800520092B21A80374F0821384604F029FE49
:10F7480088B12B6838465B4208212B6004F02CFEF8
:10F75800238801229BB2F31AFB6323889BB23344AC
:10F768003B64304B9A822B4F1021384604F011FE2F
:10F7780070B13846102104F017FE238801229BB28D
:10F78800F31AFB6323889BB21E44264B3E649A827D
:10F79800404607F03FFB06F01DFF1BA3D3E90023FB
:10F7A80006F06CFF2E68044630460D4607F032FB23
:10F7B80006F010FF02460B462046294607F088F857
:10F7C800194B044618680D4606F004FF02460B461E
:10F7D8002046294606F052FF07F0EAF9134A144B6F
:10F7E8001278186072B11A6852421A60BDE8F08146
:10F7F8000848082104F0D8FDBDE8F041054810216B
:10F8080004F0D2BDBDE8F08100000000006AF840B5
:10F818007628012000040140F83401200E3501202B
:10F82800FC34012000140040702801206C280120BD
:10F83800F434012010B50446084607F0EBFA06F048
:10F84800C9FE09A3D3E9002306F018FF07F0B0F9B1
:10F85800074B58615A692046BDE81040C3F8CC21CF
:10F86800FFF74CBEAFF300802D431CEBE2361A4085
:10F87800244A002010B50446084607F0CBFA06F0E3
:10F88800A9FE09A3D3E9002306F0F8FE07F090F9D2
:10F89800074B18601A682046BDE810405A60FFF709
:10F8A8002DBE00BFAFF300802D431CEBE2361A409B
:10F8B800244A002008B581EAE170A0EBE17007F066
:10F8C800A9FA06F087FE06A3D3E9002306F0D6FEC0
:10F8D80007F06EF9044BC3F8D00108BDAFF3008000
:10F8E8002D431CEBE2361A40244A002070B50E4B1B
:10F8F8000E4C00221A70237A054673B10C4B084649
:10F908001E6807F087FA0B4B53F8251007F0D6FA54
:10F9180007F024FC801BE06000E0E1602846BDE8B9
:10F928007040FFF7EBBD00BF00350120244A0020DE
:10F93800183501207028012038B5114B05461A7A70
:10F948000C46BAB1084607F065FA0E4B53F8251075
:10F9580007F0B4FA07F002FC05460020F8F796FE17
:10F96800094B281A18600020F8F7AAFE074B201A3E
:10F97800186038BD1961BDE83840FFF7BFBD00BF4A
:10F98800244A00207028012018350120083501205C
:10F9980010B5044681EAE170A0EBE17007F03AFA8D
:10F9A80006F018FE08A3D3E9002306F067FE07F067
:10F9B800FFF8074BC3F8D4012046BDE81040FFF715
:10F9C8009DBD00BFAFF300803A8C30E28E79454090
:10F9D800244A002010B5044681EAE170A0EBE170EA
:10F9E80007F018FA06F0F6FD07A3D3E9002306F09E
:10F9F80045FE07F0DDF8064BC3F8D8012046BDE800
:10FA08001040FFF77BBD00BF2D431CEBE2361A40C8
:10FA1800244A0020022902D8024BC9B25972FFF7C2
:10FA28006DBD00BF244A0020014B83F8DC117047EC
:10FA3800244A0020082904D8034BC1F10801C3F85F
:10FA4800E011F8F7F5BE00BF244A002008B50A4BBC
:10FA5800586907F0DFF906F0BDFD05A3D3E90023D7
:10FA680006F036FF07F0A4F808BD00BFAFF300802A
:10FA78002D431CEBE2361A40244A002008B50A4BF5
:10FA8800186807F0C7F906F0A5FD05A3D3E9002318
:10FA980006F01EFF07F08CF808BD00BFAFF300802A
:10FAA8002D431CEBE2361A40244A0020014BD3F8C0
:10FAB800E4017047244A002008B5094BD3F8D00167
:10FAC80007F0A8F906F086FD03A3D3E9002306F0A2
:10FAD800FFFE07F06DF808BD2D431CEBE2361A4017
:10FAE800244A0020094B10B51A7A0446D86862B136
:10FAF800074B1B68184407F08DF9064B53F8241080
:10FB080007F090FA07F02AFB10BD10BD244A002028
:10FB18001835012070280120094B10B51A7A0446BF
:10FB2800186962B1074B1B68184407F073F9064B54
:10FB380053F8241007F076FA07F010FB10BD10BD3B
:10FB4800244A0020183501207028012008B50A4BE6
:10FB5800D3F8D40107F05EF906F03CFD04A3D3E91D
:10FB6800002306F0B5FE07F023F808BDAFF30080C8
:10FB78003A8C30E28E794540244A002008B50A4B79
:10FB8800D3F8D80107F046F906F024FD04A3D3E919
:10FB9800002306F09DFE07F00BF808BDAFF30080C8
:10FBA8002D431CEBE2361A40244A0020014B587AB8
:10FBB800704700BF244A0020024B187A003018BF53
:10FBC80001207047244A0020014B93F8DC0170475C
:10FBD800244A0020034BD3F8E001C0F10800C0B26A
:10FBE800704700BF244A002010B50748C46920099F
:10FBF80011B1E40C64010C6012B1C0F384211170DE
:10FC080003B1187010BD00BF244A0020064B1A7AB1
:10FC1800032A05D01869DB68C31A5842584170474F
:10FC2800024B1878C0B27047244A00200C350120D6
:10FC3800B4235843024900F580700422FAF7E3B868
:10FC4800F84B0020B4235843024900F5827004227F
:10FC5800FAF7D9B8FC4B0020B4235843024900F501
:10FC680084700422FAF7CFB8F44B00204FF4807068
:10FC780001490422FAF752B9F84B00204FF4827078
:10FC880001490422FAF74AB9FC4B00204FF484706A
:10FC980001490422FAF742B9F44B0020034B012230
:10FCA8005A7200225A611A60704700BF244A002025
:10FCB800024B186900F00800704700BF00040240BA
:10FCC800024B186900F01000704700BF00040240A2
:10FCD800134B70B51C7A06460D46BCB959B14FF0A6
:10FCE80080400121224604F03FFB30462146BDE812
:10FCF8007040FAF781BD0121FAF77EFDBDE870403A
:10FD080001214FF080400A4604F02EBB19B1FFF7DD
:10FD1800E9FEF8F739FF2846BDE87040F8F7BABFA2
:10FD2800244A002070B50846114C51B1207AE8B930
:10FD3800104B1B7B13B10146FFF7CAFF0123237247
:10FD480070BD237A032B11D10A4E337B0BB1FFF719
:10FD5800BFFF0025F17A28462572FFF76BFE317B3D
:10FD680021B12846BDE87040FFF7B2BF70BD00BFA3
:10FD7800244A0020DC2901204FF08043988900F0B4
:10FD880001007047074B93F82420002AFAD101227A
:10FD9800C3F8E81183F8242093F82420002AFBD123
:10FDA800704700BF244A0020014BC3F8EC0170479C
:10FDB800244A0020014BD3F8EC017047244A002064
:10FDC800014BC3F8F0017047244A0020014BD3F8D7
:10FDD800F0017047244A0020024B187AC31E58428B
:10FDE80058417047244A0020014BC3F8F40170477A
:10FDF800244A0020014BC3F8F8017047244A002028
:10FE0800014BC3F8FC017047244A0020014BC3F89A
:10FE180000027047244A0020014BC3F804027047CF
:10FE2800244A0020014BC3F808027047244A0020E6
:10FE380032235843014AC2F80C027047244A002072
:10FE480032235843014AC2F810027047244A00205E
:10FE5800014BC3F814027047244A0020014BC3F831
:10FE680018027047244A0020014BC3F81C0270474F
:10FE7800244A0020014BC3F820027047244A00207E
:10FE8800014B1860704700BF0435012008B506F023
:10FE9800C1FF044B196807F011F807F05FF9024B2E
:10FEA800186008BD7028012010350120014B18602A
:10FEB800704700BF20350120014B1860704700BF14
:10FEC8001C350120014B1860704700BF1435012014
:10FED800014BD3F8F4017047244A0020014BD3F8B2
:10FEE800F8017047244A0020014BD3F8FC01704701
:10FEF800244A0020014BD3F800027047244A00200E
:10FF0800014BD3F804027047244A0020014BD3F870
:10FF180008027047244A0020034BD3F80C0232230E
:10FF280090FBF3F0704700BF244A0020034BD3F83E
:10FF38001002322390FBF3F0704700BF244A0020E0
:10FF4800024BD3F81402C0B2704700BF244A002005
:10FF5800014BD3F824027047244A0020014BD3F800
:10FF680028027047244A0020014BD3F82C0270471E
:10FF7800244A0020014BD3F830027047244A00205D
:10FF8800014BD3F834027047244A0020014BD3F8C0
:10FF980018027047244A0020014BD3F81C0270470E
:10FFA800244A0020014BD3F820027047244A00203D
:10FFB800014BD3F838027047244A0020014B1868D7
:10FFC800704700BF0435012008B5054B186806F0D6
:10FFD80021FF044B196807F025F807F0BFF808BDA2
:10FFE8001035012070280120014B1868704700BFA8
:08FFF80020350120014B1868BF
:020000040801F1
:10000000704700BF1C350120014B1868704700BFC6
:1000100014350120014BD3F83C027047244A0020DC
:10002000014BC3F840027047244A0020014BD3F82B
:1000300040027047244A002008B50028B8BF40425B
:1000400006F0ECFE06F0CAFA05A3D3E9002306F099
:1000500019FB06F0B1FD044BC3F8440208BD00BF14
:100060002D431CEBE2361A40244A002008B50A4B07
:10007000D3F8440206F0D2FE06F0B0FA04A3D3E9A6
:10008000002306F029FC06F097FD08BDAFF30080C1
:100090002D431CEBE2361A40244A0020014BC3F8E2
:1000A00048027047244A0020014BD3F848027047A9
:1000B000244A0020014BC3F84C027047244A002018
:1000C000014BD3F84C027047244A002038B5124B3C
:1000D00004461D7AB5B11D6906F0A0FE0F4B1968E4
:1000E00006F0F0FE07F03EF80D4B401B18600020B4
:1000F000F8F7EAFA0B4B201A18602046BDE83840A2
:10010000F8F746BD28462146FFF71AFC2846214647
:10011000BDE83840F8F7E0BA244A002070280120F2
:10012000183501200835012008B5074B187A20B191
:100130000020F8F7C9FA054B02E0F8F7ABFA044BD8
:100140001B68184408BD00BF244A00200835012060
:1001500018350120014BC3F850027047244A002093
:10016000014BD3F850027047244A0020014BC3F8DA
:1001700054027047244A0020014BD3F854027047C0
:10018000244A0020034BD3F85822002AA8BFC3F802
:1001900058027047244A0020014BD3F85802704798
:1001A000244A002008B50028B8BF404206F036FEB9
:1001B00006F014FA06A3D3E9002306F063FA06F06A
:1001C000FBFC054BC3F85C0208BD00BFAFF3008029
:1001D0003A8C30E28E794540244A002008B50A4B1B
:1001E000D3F85C0206F01AFE06F0F8F904A3D3E98E
:1001F000002306F071FB06F0DFFC08BDAFF30080C2
:100200003A8C30E28E794540244A002010B51C4CCF
:10021000237A032B05D0012300206372FFF772F9C4
:1002200024E0637ADBB2012B20D002D3022B23D04F
:1002300010BD20682368D4F8D42180FB0301D317B4
:1002400006F0D6FFCB0FC018236841F1000149101A
:100250004FEA3000002B0B4BD4F860221B6813448C
:10026000CCBFC018C0EB0300E06010BD0020014609
:10027000BDE81040FFF7E2BA0023C4F8543210BDC5
:10028000244A002018350120014BC3F8640270474E
:10029000244A0020014BD3F864027047244A00200E
:1002A00038B5114C237A032B16D10020FFF7D2FB6F
:1002B000D4F86422D4F8E431801A984212DC002089
:1002C000D4F8E451FFF7C6FBD4F8643218448542F1
:1002D000CCBF0020012038BD20686369C31A584292
:1002E000584138BD002038BD244A002010B50A20EE
:1002F000F9F7BEFB04460B20F9F7BAFB404304FBB9
:100300000400BDE81040FFF72FB8684620F0070151
:100310008D462DE9F14F012188B04FF0804004F067
:100320003CF8002801F0B880B64C4FF08040012125
:1003300004F03EF8D4F86832082B0AD9012384F877
:100340006C320023C4F86832AF4B1A6801321A606D
:1003500004E0D4F868320133C4F868320025D4F8D8
:1003600070322846012384F87432C4F87052F8F7CA
:100370004DFBF8F7D9FB2846F8F78CF90590059B5B
:10038000C4F87832A14B1A781E461AB1F7F76EFFFF
:100390009F4B186094F86C329A4D002B70D03378D4
:1003A0009C4E002B55D0059AD5F87C32D31A002BE1
:1003B000B8BF5B42202B964B30DD1968D5F8802200
:1003C00091422BD0059AC5F884221B68C5F8883263
:1003D000D5F88402D5F87C32D5F88882C01A06F0A8
:1003E0001DFDD5F880728146C7EB080006F012FDAE
:1003F0000146484606F01AFE06F0F0F8864B002249
:1004000006F040F906F0D8FB3060D5F88432C5F824
:100410007C32D5F88832C5F880320DE01A68D4F8FD
:100420008032D31A002BB8BF5B42642B04DD754ABF
:1004300000233360C2F8E431D4F8E421D4F8E411A5
:100440003368CB1A802193FBF1F3D31AC4F8E4315B
:1004500016E06D4A1268642A06DD3360C5F8E4319F
:100460006E4B08221A800BE0D5F8E421D5F8E41190
:100470003368CB1A102193FBF1F3D31AC5F8E4319A
:10048000237A604D032B00F02D8195F87422002A09
:1004900000F06087022B00F05D876B7A002B42D161
:1004A000EA682B69D31AC5F88C3295F8DC3123B988
:1004B000D5F8D831C5F8903210E0E8682B69C01A39
:1004C0000028B8BF4042FEF74FFF0646D5F8D401DA
:1004D0004000FEF749FF7043C5F89002E1682269C9
:1004E000484B91420BDDD3F89012D3F8D8219142BA
:1004F000B4BFD3F89022D3F8D8215A6117E0D96855
:100500001A6991420BDAD3F89012D3F8D8219142AC
:10051000B4BFD3F89022D3F8D8215242EDE700229D
:100520005A611A6003E06FF00043C5F88C3221680D
:100530006269344B914200F08E80D3F89412D3F864
:10054000D4210A44C3F89422D3F894221214C3F895
:100550009822D3F89412D3F89822A1EB0242C3F860
:10056000942293F8DC210AB95A691A6021686269F9
:10057000244B91420BDA1868D3F898125A69014457
:10058000914214DA1A68D3F89832134410E01968CB
:100590005A6991420DDD1868D3F898125A69411AC8
:1005A000914204DD1A68D3F89832D31A00E05B69EF
:1005B0002360D4F8D021134B002A51DD5A6942B987
:1005C0001868D3F8D0110028B8BF4042884247DAF3
:1005D00035E05A69002A23DD1A68002A04DD19680B
:1005E000D3F8D021914209DB2268064B002A37DA82
:1005F0001968D3F8D0215242914231DDD3F8D0218D
:100600001DE000BF244A0020FC3401207628012090
:10061000F8340120F434012000408F400E350120D1
:100620005A69002A1CDA1A68002A0ADA1968D3F80B
:10063000D0215242914204DDD3F8D02152421A60B7
:100640000EE02268BE4B002A0ADD1968D3F8D021DB
:10065000914205DAF0E70022C3F89422C3F8982209
:10066000D4F89C122268B64B0A44C4F89C22D4F8F1
:100670009C22B34D1214C4F8A022D4F8A012D4F8CE
:100680008C220029B8BF4942002AB8BF5242914289
:10069000C4BFD3F88C22C3F8A022D4F89C22D4F88B
:1006A000A032A2EB0343C4F89C322269D4F8A032F2
:1006B00013442361FEF7E4FED4F8E031062B08D89A
:1006C000D5F8A422D5F8A012D5F8E03101FA03F349
:1006D00003E0D5F8A432D5F8A0221344C5F8A4321B
:1006E00000F038BE0020FAF777F9002800F01586F0
:1006F00095F86C32002B41D0D5F8E421D5F81832AA
:10070000002AB8BF52429A4235DDD5F82002D5F80A
:10071000E431D5F81862002BB8BF5B429B1B434302
:10072000D5F81C12D5F818228A1A93FBF2F3C5F8F3
:100730003832D5F8E431002B04DAD5F838325B4290
:10074000C5F83832D4F83812D4F820227C4B9142C4
:10075000C4BFD3F82022C3F83822D4F83812D4F812
:100760002022774B5242914208DAD3F8202252429B
:10077000C3F8382202E00023C5F8383294F8743206
:100780006F4F704D002B00F03A846F4E337B8BB16E
:100790006E4B18686E4BD3F8008006F03FFB6D4B34
:1007A000196806F08FFB06F0DDFC0023C8EB0000A3
:1007B000F8607B722B7803F0FF02002B40F0CA83B5
:1007C000617A5F4B022900F0B582D3F8A812D3F802
:1007D0006022891A604A11605B68002B134602DAB6
:1007E000126852421A60716931B3186881EAE17285
:1007F000A2EBE1720028B8BF404290421CDD00220B
:1008000062612260C4F8CC216260D4F860220029C1
:10081000C4F8A822D4F86022B8BF49494F48E26022
:100820004FF00102B8BF81F8AC2202704C4A517DF2
:10083000012904BF02215175D4F84412D4F8D821FB
:10084000914226DD1A68002A02DA434A002111602B
:100850001968D4F84822914202DA3F4A0021116017
:100860001868D4F8403280FB0301002871F10003BE
:1008700002DAFF3041F10001020A42EA0162D4F8D3
:100880004472D4F8D8117F1ABA4203DC22EAE27724
:1008900000E00027637A2A4E002B63D1F268D6F875
:1008A0006032D31AC6F88C3296F8DC312BB9D6F800
:1008B000D8313B44C6F8903212E0F068D6F8603286
:1008C000C01A0028B8BF4042FEF74EFD8046D6F859
:1008D000D4014000FEF748FD00FB08F0C6F8900286
:1008E000E168D4F86022164B91420DDDD3F89012E6
:1008F000D3F8D8213A44914202DAD3F8902212E098
:10090000D3F8D821174414E0D968D3F86022914273
:1009100011DAD3F89012D3F8D8213A44914204DA8C
:10092000D3F8902252425A6120E0D3F8D8211744DC
:100930007F425F611AE000225A611A6016E000BF30
:10094000244A002000350120DC2901205C280120F8
:100950001835012070280120EC340120B529012030
:10096000442A01206FF00043C6F88C322168626986
:10097000AE4B91427ED0D3F89412D3F8D4210A44DE
:10098000C3F89422D3F894221214C3F89822D3F80F
:100990009412D3F89822A1EB0242C3F8942293F860
:1009A000DC210AB95A691A60216862699F4B914239
:1009B0000BDA1868D3F898125A690144914214DA94
:1009C0001A68D3F89832134410E019685A699142B2
:1009D0000DDD1868D3F898125A69411A914204DD66
:1009E0001A68D3F89832D31A00E05B692360D4F810
:1009F000D0218E4B002A42DD5A6942B91868D3F8DB
:100A0000D0110028B8BF4042884238DA26E05A693F
:100A1000002A14DD1A68002A04DD1968D3F8D021F1
:100A2000914209DB2268814B002A28DA1968D3F841
:100A3000D0215242914222DDD3F8D0210EE05A69F2
:100A4000002A1CDA1A68002A0ADA1968D3F8D021B9
:100A50005242914204DDD3F8D02152421A600EE096
:100A60002268724B002A0ADD1968D3F8D02191421E
:100A700005DAF0E70022C3F89422C3F89822D4F8EC
:100A80009C122268694B0A44C4F89C22D4F89C2228
:100A9000664E1214C4F8A022D4F8A012D4F88C2206
:100AA0000029B8BF4942002AB8BF52429142C4BF90
:100AB000D3F88C22C3F8A022D4F89C22D4F8A03218
:100AC000A2EB0343C4F89C32D4F86022D4F8A032DD
:100AD0001344C4F86032637A002B48D1F268D6F828
:100AE000A832D31AC6F8B03296F8DC3123B9D6F85A
:100AF000D831C6F8B43211E0F068D6F8A832C01A7E
:100B00000028B8BF4042FEF72FFC0746D6F8D401B4
:100B10004000FEF729FC7843C6F8B402E168D4F837
:100B2000A822424B91420CDDD3F8B412D3F8D8215D
:100B30009142B4BFD3F8B422D3F8D821C3F8CC2162
:100B400019E0D968D3F8A82291420BDAD3F8B4128D
:100B5000D3F8D8219142B4BFD3F8B422D3F8D82126
:100B60005242EBE70022C3F8CC215A6003E06FF059
:100B70000043C6F8B0326168D4F8CC212B4B9142C7
:100B800000F08B80D3F8B812D3F8D4210A44C3F80C
:100B9000B822D3F8B8221214C3F8BC22D3F8B81282
:100BA000D3F8BC22A1EB0242C3F8B82293F8DC21AF
:100BB00012B9D3F8CC215A606168D4F8CC211B4B10
:100BC00091420CDA5868D3F8BC12D3F8CC21014416
:100BD000914216DA5A68D3F8BC32134413E05968CC
:100BE000D3F8CC2191420FDD5868D3F8BC12D3F86A
:100BF000CC21411A914204DD5A68D3F8BC32D31A91
:100C000001E0D3F8CC316360D4F8D021074B002A3F
:100C100048DDD3F8CC215AB95868D3F8D011002850
:100C2000B8BF404288423DDA2BE000BF244A002092
:100C3000D3F8CC21002A14DD5A68002A04DD596853
:100C4000D3F8D021914209DB6268A44B002A29DA4B
:100C50005968D3F8D0215242914223DDD3F8D021F4
:100C60000FE0D3F8CC21002A1CDA5A68002A0ADAED
:100C70005968D3F8D0215242914204DDD3F8D021F3
:100C800052425A600EE06268944B002A0ADD5968AD
:100C9000D3F8D021914205DAF0E70022C3F8B82258
:100CA000C3F8BC22D4F8C01262688C4B0A44C4F862
:100CB000C022D4F8C0221214C4F8C422D4F8C4123A
:100CC000D4F8B0220029B8BF4942002AB8BF524226
:100CD0009142C4BFD3F8B022C3F8C422D4F8C022D2
:100CE000D4F8C432A2EB0343C4F8C032D4F8A8222B
:100CF000D4F8C4321344C4F8A832FEF7C1FBD4F8C8
:100D000060222369D31AC4F83C322269D4F83C32F9
:100D10001344236122690599059BFF339A4204DC41
:100D2000A1F1FF039342B8BF134623612369C4F8BE
:100D3000603225E1D3F85012002901DDFF2205E0E1
:100D4000D3F850120029B8BF6FF0FE02C3F83C225E
:100D5000D4F85012D4F85422604B914200F099809C
:100D6000D3F8C812D3F85C220A44C3F8C822D3F8D7
:100D7000C8221214C3F8CC22D3F8C812D3F8CC225C
:100D8000A1EB0242C3F8C82293F8DC211AB9D3F8C8
:100D90005422C3F85022D4F85012D4F854224F4BA6
:100DA00091420EDAD3F85002D3F8CC12D3F8542281
:100DB000014491421ADAD3F85022D3F8CC321344CA
:100DC00016E0D3F85012D3F85422914212DDD3F832
:100DD0005002D3F8CC12D3F85422411A914205DDC7
:100DE000D3F85022D3F8CC32D31A01E0D3F85432DE
:100DF000C4F85032D4F85822384B002A4EDDD3F8CC
:100E000054224AB9D3F85002D3F858120028B8BF78
:100E10004042884242DA39E0D3F85422002A18DDF1
:100E2000D3F85022002A05DDD3F85012D3F8582207
:100E300091420BDBD4F85022284B002A2EDAD3F84B
:100E40005012D3F858225242914227DDD3F858224B
:100E50001CE0D3F85422002A20DAD3F85022002ACA
:100E600006DAD3F85012D3F85822524291420ADCE3
:100E7000D4F85022194B002A10DDD3F85012D3F8C1
:100E8000582291420ADAD3F858225242C3F850222B
:100E900004E00022C3F8C822C3F8CC22104B5A7ECB
:100EA000737B0ABBDF070AD50E4909690E0706D511
:100EB000D4F850120029BCBF0849C1F83C22980759
:100EC0002ED5084B1B69D9062AD5D4F85032002BF1
:100ED00026DD024B0022C3F83C2221E0244A0020F8
:100EE0000400002000040240DA070BD5AC4A126966
:100EF00012F0080206D1D4F850120029BCBFA9494B
:100F0000C1F83C229B070BD5A54B1B6913F01003BE
:100F100006D1D4F85022002AC4BFA24AC2F83C32FB
:100F20002269D4F83C321344236122690599059B58
:100F3000FF339A4204DCA1F1FF039342B8BF13468A
:100F400023612369E3602369C4F860322369C4F82C
:100F5000A83215E0002363612360C4F8CC316360DC
:100F6000D4F86032C4F8A832E2680599059BFF33D3
:100F70009A4204DCA1F1FF039342B8BF13462361F8
:100F80008949E6680868059B301A9842854A874B6C
:100F900016DA0598D66809683144884210DA19686B
:100FA000002903DD1A68013A1A600FE08049012325
:100FB0000B70D2F86012D268914207D12B7005E015
:100FC0007C4A12681A607A4B00221A707A4B059993
:100FD000E0681A68821A914206DB7249059AC9686C
:100FE0001B680B449A4201DD00232B70637A012BAE
:100FF00003D06C4B5B7A022B01D100232B70059A36
:101000002369C4F8D0322B7803F0FF0123B16B4B76
:1010100018686B4B196800E00A20D4F8D062D4F845
:10102000F051604B3544AD1AC4F82C52D4F82C5210
:10103000C4F8D452D4F82C62D4F8EC51002EB8BFC6
:101040007642AE423DDCD3F82C525DB3D3F82C721D
:10105000D3F82C627843D3F8D8520A2790FBF7F0E4
:10106000751B01FB0501C3F8D412D3F8D402D3F8E1
:10107000EC118842C4BFD3F8EC11C3F8D412D4F8F1
:10108000D402D4F8EC11474B4942884204DAD3F831
:10109000EC114942C3F8D412D4F8D4321A44C4F83B
:1010A000302204E0D3F82C120A44C3F83022D4F8DA
:1010B0003022D4F838321344C3F30903C4F834326D
:1010C0001EE0D3F82C02D3F8EC114942884203DA2F
:1010D000D3F8EC11521A08E0D3F82C02D3F8EC1133
:1010E00088420DDDD3F8EC110A44C3F83022D3F85E
:1010F0003012D3F838220A44C2F30902C3F834226A
:10110000D4F82C32274DC4F8D832D4F83432C4F88D
:10111000A432637A022B30D1FEF72EFAD5F8503282
:1011200006468342C8BFC5F85002D4F85022434255
:101130009A42BCBF1B4AC2F85032D4F85002002871
:10114000B8BF404205F06AFE0546304605F066FE2F
:101150000146284605F06AFF05F040FA0EA3D3E9E0
:10116000002305F08FFA05F027FDFF28A8BFFF2018
:10117000C4F82802C4F82402ECE0D5F81432002B9D
:1011800000F0C680D5F84C32D5F8F401D5F8042229
:10119000C3B1D5F8D43217E00000000000E06F4082
:1011A00000040240244A002010350120F0340120C0
:1011B0000C35012004350120143501202035012093
:1011C0001C350120D5F82C320130801AD5F8FC717D
:1011D000D5F8F8B1D5F8F4A1D5F80092D5F8FC818E
:1011E000019305F01BFE019B064683EAE370A0EB2A
:1011F000E370C01B05F012FE0746CAEB0B0005F0BA
:101200000DFE8246C8EB090005F008FE0146504677
:1012100005F00CFF0146384605F054FE0146304605
:1012200005F048FD05F09EFFC5F82802D4F8281205
:10123000D4F8F4219B4B9142BCBFD3F8F421C3F8FE
:101240002822D4F82812D4F8F821964B9142C4BF32
:10125000D3F8F821C3F82822D4F8DC22914B002AD5
:1012600004DDD3F8DC22013AC3F8DC22D4F8E02212
:101270008C4B002A04DDD3F8E022013AC3F8E022C7
:10128000D4F82812D4F82422864B91421CDDD3F8DE
:101290000C2212B3D3F8DC22002A5BD1D3F824123B
:1012A000D3F804220A44C3F82422D3F82412D3F832
:1012B000F8219142C4BFD3F8F821C3F82422D4F80E
:1012C0000C32C4F8DC3245E0D3F82812D3F82422DB
:1012D00091423FDAD3F8102222B9D3F82822C3F87A
:1012E000242237E0D3F8E022002A33D1D3F82402B5
:1012F000D3F80812884204DBD3F82412D3F808226A
:101300008A1AC3F82422D4F81032C4F8E03221E05B
:10131000D5F8F831C5F824321CE068612860C5F8BA
:10132000CC016860059B2B61059BEB60059BC5F8B4
:101330006032059BC5F8A8325B4B05981B681844C2
:1013400005F06CFD594B196805F070FE05F00AFFB9
:10135000F7F71EFC0598D4F8E411D4F85022514D4B
:1013600000F03EFE00F01EFE30B300F027FE012824
:1013700006D00AD3022817D1EB680693059B15E027
:101380006B690693D5F8E43110E06B7A022B05D136
:10139000D5F850320693D5F8503207E0D5F83C32F4
:1013A0000693D5F83C3201E000230693079308AB7F
:1013B00013E9030000F0B2FDFEF798FFFEF750F9C5
:1013C00094F82520374B002A61D193F8E422002AB3
:1013D0005DD193F82420002A4AD1D3F8E021062ACF
:1013E00001D91A7A52B1D4F8A432314AC3F30903AD
:1013F00002EB8303D3F8003423620FE0D3F8E0213B
:10140000D3F8A412072A2B4A01F00F0102EB810244
:101410000CBFD2F80823D2F848231A62227A214B53
:10142000032A28D193F82020D2B203920399D3F84B
:1014300024225143FF22B1FBF2F10391196A4908BA
:10144000196293F82110C9B204910498D3F82412B8
:101450004143B1FBF2F20492049AD2B283F8212004
:101460001A6A52001A62039AD2B283F8202002E06C
:10147000D3F8E8211A62104B10225A830F48012238
:101480000023712184F82520A36102F05DFA002376
:1014900084F86C3284F8743208B0BDE8F14F8546A8
:1014A000704700BF244A0020183501207028012011
:1014B000F8810108F092010800000240003001406C
:1014C000034BD3F8A802034B1B681844704700BFB6
:1014D000244A00201835012008B5094BD3F8CC0167
:1014E00005F09CFC05F07AF803A3D3E9002305F08E
:1014F000F3F905F061FB08BD2D431CEBE2361A4001
:10150000244A002008B50A4B586805F087FC05F00E
:1015100065F805A3D3E9002305F0DEF905F04CFBDF
:1015200008BD00BFAFF300802D431CEBE2361A402C
:10153000244A0020094B1A7A2AB983F8E5220422AA
:101540001A7201207047032A05D10120042283F872
:10155000E5021A7270470020704700BF244A00203D
:10156000014B93F8E6027047244A0020044B1A7A94
:10157000032A03D1012083F8E70270470020704757
:10158000244A0020014B93F8E8027047244A0020C7
:10159000014B986A704700BF244A0020014BD3F8E2
:1015A000EC027047244A0020014B586B704700BF83
:1015B000244A0020014BD3F8F0027047244A00204F
:1015C000014B93F8F4027047244A0020014B9862C3
:1015D000704700BF244A0020014BC3F8EC0270475B
:1015E000244A0020014BC3F8F0027047244A00202F
:1015F000024B012283F8F522704700BF244A0020E5
:101600004FF4887001490422F8F701BC4C4A0020CD
:101610004FF48A7001490422F8F7F9BB104D0020FD
:101620004FF48C7001490422F8F7F1BB144D0020EF
:101630004FF48E7001490122F8F7E9BB184D0020E4
:101640004FF4887001490422F8F76CBC4C4A002022
:101650004FF48A7001490422F8F764BC104D002051
:101660004FF48C7001490422F8F75CBC144D002043
:101670004FF48E7001490122F8F754BC184D002038
:10168000054B1A682AB95869D0F1010038BF00200B
:1016900070470020704700BF244A002070B5BB4C43
:1016A000237A013B052B00F20881DFE803F00319E0
:1016B000465383AF00252846C4F8E051F7F7BCF83D
:1016C0002846FEF7EFFA28462561E560FDF71AFF88
:1016D000F6F7CCFDC4F8A452C4F8F80202232AE0BD
:1016E000F6F7C4FDD4F8F832A84DC01A80EAE073CA
:1016F000A3EBE073B3F5FA7F40F3DF8000200146EF
:10170000F6F7EAFF0020F6F7C5FF28612B690020F5
:10171000EB60EB68C5F86032EB68C5F8A8329C4B0B
:1017200018609C4B18609C4B197B09B1FEF7D4FAEA
:101730000023637203232372BFE094F8AC32002BC2
:1017400000F0BB800020F9F72BF9904B002283F8C2
:10175000AC22B2E000252846C4F8E051F7F76CF857
:101760002846FEF70FFAC4F8FC022846FEF7F2F905
:101770008A4BC4F800032846C4F8D831FDF7C2FEEE
:10178000874B2846C4F8D431FDF7BCFE2846FEF747
:1017900089FA7F4BC4F8A4522561E5601D607D4B3A
:1017A0001D60012384F8E632F6F760FD0523C4F8D6
:1017B000F802C0E7F6F75AFDD4F8F832734EC01AB3
:1017C00080EAE073A3EBE073FA2B76DD724B002521
:1017D0001969284621F02F411961724B090E1D70BD
:1017E000F6F7D4FF28464FF48031F6F7B1FF2846CC
:1017F0002946F6F771FF6C4B28461B681B02F36005
:101800007572FDF77FFE0623337256E00020FEF767
:1018100001FA002851D00020F6F73CFF051E08DA37
:1018200000200121F6F7B2FF5B4B1A6942F080728B
:101830001A615E4B85EAE570A0EBE57053F8041F72
:101840004A1C11D06FF0C70291FBF2F20A448242A7
:10185000F4DCC82291FBF2F20A449042EEDC002054
:10186000F7F7F2FA022303E0002384F8E5320323BA
:101870000025002084F8E632FEF714FA28462946AF
:101880002561E560F6F728FF94F8E5323F4E002B1E
:1018900000F00182012333720020D4F8FC1284F896
:1018A000E552FEF79BF80020D4F80013FEF774F819
:1018B000394B0020D97AFEF7C1F894F8E732013BA2
:1018C0000B2B00F28481DFE813F00C001D002F00C9
:1018D0004E007300D600F0001E01E00038015E01EA
:1018E0007A01012300200225C4F8F00184F8E832CF
:1018F0006572FDF707FEFDF73FFE84F8E752C4F876
:10190000540264E1D4F85022D4F854321F4D9A4264
:1019100040F05D81032385F8E732F6F7A7FCD5F8A0
:10192000E431C5F8040314E0F6F7A0FCD4F804335E
:10193000164DC01A80EAE073A3EBE073B3F5FA6FBB
:101940000ADAD5F8E421D5F808331344022293FBD0
:10195000F2F3C5F808333AE1FDF70EFE4042C5F850
:101960005402042384E0D4F85022D4F85432074DB2
:101970009A4240F02C81052385F8E732F6F776FC91
:10198000D5F8E431C5F8040327E000BF244A00205D
:101990001835012008350120DC290120B81E05007A
:1019A000EF8D210075280120682801207496010818
:1019B000F6F75CFCD4F80433B84DC01A80EAE07343
:1019C000A3EBE073B3F5FA6F0ADAD5F8E421D5F8A2
:1019D0000C331344022293FBF2F3C5F80C33F6E008
:1019E0000023C5F85432D5F80C3383EAE372A2EB36
:1019F000E372D5F808339A4218DAD5F8F031013B92
:101A0000C5F8F031FDF7B8FDD5F80C33C5F8540230
:101A100083EAE372A2EBE372D5F808339B1A002B3A
:101A2000B8BF5B42C5F81033062321E01FDDD5F8AF
:101A3000F0310133C5F8F031FDF79EFDD5F80C33D8
:101A4000404283EAE372A2EBE372D5F80833C5F8AB
:101A500054029B1A002BB8BF5B42C5F81033092310
:101A600006E04EDDD5F8F0310133C5F8F0310C2336
:101A700085F8E732ABE0D4F85022D4F85432874DE1
:101A80009A4240F0A480082308E0D4F85022D4F809
:101A90005432824D9A4240F09A800B2385F8E73207
:101AA000F6F7E4FBC5F8040391E0D4F80C337B4D62
:101AB00083EAE372A2EBE372D4F808339B1A83EA59
:101AC000E372A2EBE372D4F810339A42C9DAD5F884
:101AD000F031013BC5F8F031F6F7C8FBD5F80C231F
:101AE000D5F8E431002AB8BF5242C5F808339B1A32
:101AF000002BB8BF5B42C5F81033C5F804030823B8
:101B0000B6E70C2361E0F6F7B1FBD4F80423634B8E
:101B1000801A80EAE072A2EBE072B2F57A7F0ADA0C
:101B2000D3F8E411D3F808230A44022192FBF1F21E
:101B3000C3F808234BE007223EE0D4F80C33574D9E
:101B400083EAE372A2EBE372D4F808339B1A83EAC8
:101B5000E372A2EBE372D4F810339A420EDAD5F8AE
:101B6000F0310133C5F8F031F6F780FBD5F8E431F8
:101B7000C5F80403C5F80C330B2379E7C1DDD5F8AC
:101B8000F031013B71E7F6F771FBD4F80423434BC6
:101B9000801A80EAE072A2EBE072B2F57A7F0ADA8C
:101BA000D3F8E411D3F80C230A44022192FBF1F29A
:101BB000C3F80C230BE00A2283F8E72207E0022394
:101BC00084F8E8320023C4F8543284F8E732D4F8B9
:101BD000EC32324D2BB36A6B9A4222D9F6F746FBB0
:101BE000D5F81433C01A80EAE073A3EBE073B3F5C1
:101BF0007A7F16DD95F8F4327BB9012385F8F4324B
:101C0000F6F734FBD5F8F032C5F818030133C5F800
:101C1000F032FFF70DFDFFF703FDF6F727FBC4F8E1
:101C20001403F6F723FBD4F81823A16A801A80EA7C
:101C3000E072A2EBE0728A42184B10D993F8F422BA
:101C400082B193F8F5226AB1002583F8F45283F843
:101C5000F552FFF7EDFC2846F7F706F902E00022FF
:101C600083F8F52294F8F43223B10020BDE87040E7
:101C7000F7F7FDB80A4B1B7B012B03D0043BDBB20B
:101C8000012B0AD8074B1B691B07EED5BDE8704036
:101C90000020F7F7E9B83572FEE570BD244A002050
:101CA000DC290120000002407FB5244D244C082689
:101CB0002E80616A2B8820469BB2C91A02F057F920
:101CC000636A2988204689B2194402F052F92046F5
:101CD0003146012202F04CFB01222046102102F085
:101CE00047FB2E230124174D8DF800306846022350
:101CF0008DF801308DF802408DF8034002F0FCFDB4
:101D00002146202001F0F0FB284601F0C1FE4FF6ED
:101D1000FF7302934FF41673ADF804302846002386
:101D200001A9ADF80C30ADF8063001F05BFF284694
:101D3000214601F0ECFF04B070BD00BF0E3501205C
:101D400000040140001400407FB500204C4CFDF71A
:101D500091FF0020FDF796FF0020FDF79BFF04F5A3
:101D6000F8714FF486700422F8F7DCF8FFF768FC8E
:101D7000FFF76EFCFFF774FCFFF77AFCFF230F22DE
:101D80004049C4F8EC310125C4F824220026C4F8E7
:101D9000F4210A22C4F8F831C4F8FC61C4F8003216
:101DA000C4F80452C4F80852C4F80C62C4F81062B3
:101DB000C4F81452C4F84C5284F8DC510A60324919
:101DC00064200E6031490B60314908603149284672
:101DD0000A604FF4FA62C4F840224B22C4F8482249
:101DE0002D4A2946C4F84422C4F820322B4BC4F8AB
:101DF00018322B4BC4F81C324FF4FA73C4F8643217
:101E00004AF2C573C4F85C3201F06EFB4FF08040BB
:101E100001F03EFE41F2707301A94FF08040029341
:101E2000ADF80460ADF80C60ADF8066001F0DAFEC4
:101E30002A4629464FF0804002F09AFA29464FF090
:101E4000804001F064FFFFF72FFF1C2368468DF8E8
:101E500000308DF801508DF802508DF8035002F0DB
:101E60004BFD232368468DF800308DF801608DF816
:101E700002508DF8035002F03FFD04B070BD00BF6A
:101E8000244A0020203501201C3501201435012072
:101E90001035012004350120703D0A0020A1070003
:101EA000804F1200AFF300804DF6C020704741F61E
:101EB000583070470220704741F65733984210B5AA
:101EC00021D801291FD8144B1A681C46012A08D0B2
:101ED00001D3022A17D101EB400104EB81014868CC
:101EE00010BDC000184461B9406804F097FF04F0C9
:101EF00075FB07A3D3E9002304F0EEFC04F05CFEBD
:101F000010BD806810BD002010BD00BFAFF3008081
:101F10002D431CEBE2361A40544D002013B5124BF2
:101F20008DE80300D3F8241F41F65730814216D8BC
:101F3000D3F8280F78B90D4C481CD3F82C2F04EB9C
:101F4000C1010C1DC3F8240FC3F8282F9DE803001E
:101F500084E8030006E00138C3F8280F02E00022FD
:101F600083F8302F02B010BDF4180120544D00202A
:101F7000074B002283F8302FC3F8242FC3F8282FF3
:101F8000012283F8310FC3F8341F83F8382F7047CC
:101F9000F4180120024B002283F8302F704700BF55
:101FA000F4180120014B93F8300F7047F41801200A
:101FB000014B1860704700BF544D0020014B18685A
:101FC000704700BF544D0020014BC3F82C0F7047E1
:101FD000F4180120014BD3F82C0F7047F41801209E
:101FE00030B51B4B93F8384F84B393F8304F6CBB2C
:101FF00093F8314F062C22D8DFE804F008040C10C7
:1020000014191D00D3F8342F904218DA012283F8F6
:10201000302F14E0D3F8342F904206E0D3F8342F59
:102020009142F2E7D3F8342F9142EFDC07E0D3F886
:10203000341F8A42E9E7D3F8341F8A42F5E793F860
:10204000303F1BB1024B002283F8382F30BD00BF58
:10205000F4180120AFF300807047FEE7FEE7FEE7CB
:10206000FEE7704770477047704700002F4B82B003
:102070001A6842F001021A6000229A60196821F081
:10208000847121F48031196029495960196821F45B
:1020900080211960DA60009201921A6842F480325D
:1020A0001A60224B1A6802F400320192009A01323F
:1020B0000092019A1AB9009AB2F5A06FF1D11B688B
:1020C00013F4003318BF01230193019B012B04D0AB
:1020D000184B194A9A6002B07047144B9A689A607C
:1020E0009A6842F400429A609A6842F4A0529A6058
:1020F000124A5A601A6842F080721A6019680B4AD4
:102100008901FBD50E4B40F203711960936823F0EF
:1021100003039360936843F002039360034B9B684F
:1021200003F00C03082BF9D1D2E700BF00380240BE
:102130001030002400ED00E000800008081E40057B
:10214000003C0240134A10B59068134B00F00C009D
:102150000428124913D0082811D1546850685268D5
:1021600000F03F00C2F38812B1FBF0F15143094A7D
:102170005268C2F3014201325200B1FBF2F1054A4A
:1021800019609268C2F303121A4411791A68CA409E
:102190001A6010BD00380240BC0000200024F4008A
:1021A00008B54FF48070012101F0E6F9BDE8084060
:1021B0004FF48070002101F0DFB943680A6823F012
:1021C000407323F4807313430A7910B543EA022362
:1021D0004360CA680B6984681A438B681A43084BCA
:1021E000234013434A7943EA420383600B7DC26A6A
:1021F000013B22F47002DBB242EA0353C36210BD1A
:10220000FDF7FFC000230360037143718360C36067
:102210000361012303757047074A084B516810B5E5
:102220000B4090E812000C438168C06821430143D1
:102230000B43536010BD00BF00230140E030FCFFA2
:102240000023036043608360C3607047836811B1FB
:1022500043F0010301E023F001038360704743680A
:1022600023F4400323F40073194341607047416233
:1022700082627047436823F01F031943416070472F
:10228000044B5A6810B142F4000201E022F400024B
:102290005A60704700230140044B5A6810B142F461
:1022A000800201E022F480025A607047002301405E
:1022B000092970B50DD9A1F10A0404EB44040725DE
:1022C000A540A340C66826EA050545EA0304C460A4
:1022D0000BE001EB41040725A54003FA04F406696D
:1022E00026EA050545EA04030361062A0CD8013AEB
:1022F00002EB82021F23934001FA02F2446B24EAAC
:1023000003031A43426370BD0C2A0CD8073A02EB50
:1023100082021F23934001FA02F2046B24EA0303B2
:102320001A43026370BD0D3A02EB82021F239340F1
:1023300001FA02F2C46A24EA03031A43C26270BDBE
:10234000836843F08043836070478068C0F38050A7
:102350007047836811B143F4806301E023F4806324
:1023600083607047836811B143F0020301E023F0FA
:102370000203836070474368013923F4604343EAF2
:10238000413343607047436811B143F4006301E097
:1023900023F4006343607047C06C80B27047014B08
:1023A0001868704708230140836811B143F48073B3
:1023B00001E023F4807383607047836811B143F4B4
:1023C000007301E023F4007383607047044B5A6884
:1023D00010B142F4005201E022F400525A607047FA
:1023E00000230140092970B50DD9A1F10A0404EBBD
:1023F00044040725A540A340C66826EA050545EA2A
:102400000304C4600BE001EB41040725A54003FA77
:1024100004F4066926EA050545EA04030361846BB2
:10242000931CC4F301555B1BDBB203EB83031F2238
:102430009A40994024EA020444EA0103836370BD90
:10244000836B013923F4401343EA015383637047DC
:1024500082B0002301930190019B19440191019BDB
:102460001A6002B07047836823F4702319438160B7
:102470007047836823F44013194381607047836871
:1024800043F48003836070478068C0F380507047D6
:10249000436811B143F4806301E023F48063436037
:1024A0007047436811B143F4805301E023F4805333
:1024B0004360704782B0002301930190019B283351
:1024C00019440191019B186880B202B07047012342
:1024D000C9B203FA01F143680AB1194301E023EAE2
:1024E000010141607047036819420CBF00200120C0
:1024F0007047C943016070474368006810EA1120C3
:1025000007D0C9B2012202FA01F119420CBF002022
:10251000012070476FEA11210160704708B50B4B2D
:10252000984207D14FF00070012101F019F84FF0E7
:10253000007006E04FF08060012101F011F84FF0CB
:1025400080600021BDE8084001F00AB80064004046
:10255000036823F002030360036843F00103036090
:102560004FF480334268D20701D4013BFAD143686B
:1025700013F0010355D08B79012B03680CBF43F096
:10258000800323F080030360CB79012B03680CBF29
:1025900043F0400323F0400303600B7A012B0368F0
:1025A0000CBF43F0200323F0200303604B7A012B80
:1025B00003680CBF43F0100323F0100303608B7A11
:1025C000012B03680CBF43F0080323F008030360EA
:1025D000CB7A012B03680CBF43F0040323F0040300
:1025E00003608B78CA789B0743EA02630A7943EA5F
:1025F00002434A7943EA02530A88013A1343C3610A
:10260000036823F0010303604FF480334268D2076C
:1026100001D5013BFAD1406800F0010080F00100D3
:10262000704718467047837A01219940344B70B542
:10263000D3F80022CC4342F00102C3F80022D3F8C1
:102640001C222240C3F81C22027BA2B9D3F80C2220
:10265000C6882240C3F80C22827A4588483245EA6F
:10266000064543F8325003888288857A43EA02425D
:10267000244BED005A51037B012B15D1204B0688CA
:10268000D3F80C2245880A43C3F80C22827A45EA23
:102690000645483243F83250C3888288857A43EA37
:1026A0000242184BED005A51C37A154A1BB9D2F8B1
:1026B0000432234002E0D2F804320B430589C2F809
:1026C00004320F4B2DB9D2F814522C40C2F81442E8
:1026D00006E0012D04D1D3F814220A43C3F81422D2
:1026E000427B012A04D1D3F81C221143C3F81C12E7
:1026F000D3F8002222F00102C3F8002270BD00BF0F
:10270000006400404466004000238371C37103727B
:1027100043728372C3728370C370032303710223F5
:1027200043710123038070470D4BD3F8002242F020
:102730000102C3F80022D3F8002222F47C5222F0D6
:102740000E02C3F80022D3F8002242EA0020C3F8A8
:102750000002D3F8002222F00102C3F800227047E1
:1027600000640040036811B143F4803301E023F4B6
:10277000803303607047036899B143F080030360BE
:10278000D0F8843143F48073C0F88431D0F89431A8
:1027900043F48073C0F89431D0F8A43143F48073CB
:1027A00012E023F080030360D0F8843123F48073B7
:1027B000C0F88431D0F8943123F48073C0F8943198
:1027C000D0F8A43123F48073C0F8A4317047836833
:1027D000F0B55C01024607D48368180106D49368FB
:1027E000DB0005D40420F0BD002002E0012000E061
:1027F000022005015319D3F8804104F00104C3F805
:1028000080410C7A4E7A44B90C68D3F8807146EA5C
:1028100044543C43C3F8804109E04F68D3F880C179
:1028200044EAC70444EA0C042643C3F880618C7A66
:102830002A4404F00F048C72D3F8844124F00F046E
:10284000C3F884418E7AD3F884413443C3F8844179
:102850004E7B8C7B360446EA0466CC7A26430C7B9E
:1028600046EA0426C2F8886102F5C4744A7C8D7C6D
:10287000120442EA0562CD7B097C2A4342EA012226
:102880006260D3F8802142F00102C3F88021F0BDDC
:10289000012908D004D3022916D182680C4B04E028
:1028A00082680C4B01E082680B4B1340094A93424B
:1028B00008D001D853B907E0074A934202D0044A2E
:1028C000934203D1012070470220704700207047D7
:1028D000000003100300000400030008012907D0D2
:1028E00002D3022908D07047836843F0800306E0D2
:1028F000836843F4004302E0836843F40003836089
:10290000704730B50C010319D3F8B05105F0040538
:10291000EDB2157225B9D3F8B0516D0D156003E015
:10292000D3F8B051ED085560D3F8B05105F0020569
:102930005572D3F8B45105F00F059572D3F8B43140
:102940001B0AD3740319D3F8B85103F5DC74D5729C
:10295000D3F8B8512D0A1573D3F8B8512D0C55730F
:10296000D3F8B8311B0E93736368D37363681B0A83
:10297000137463681B0C537463681B0E937421B942
:10298000C36843F02003C36030BD036943F02003F4
:10299000036130BD21B9C36843F02003C3607047B1
:1029A000036943F020030361704709B9C06802E07E
:1029B000012903D1006900F003007047002070472F
:1029C00099B9036823F0030343F0010303604FF454
:1029D0008033426802F00302012A01D0013BF8D1A2
:1029E000406800F00300012828E0012911D10368A4
:1029F00023F0030303604FF480334268920701D051
:102A0000013BFAD1436813F0030F14BF00200120EB
:102A10007047022916D1036823F0030343F0020331
:102A200003604FF48033426802F00302022A01D0AF
:102A3000013BF8D1406800F00300022814BF0020D9
:102A40000120704700207047036823F0030343F020
:102A500002030360406800F00300831E584258419F
:102A60007047036823F0020303604FF48033426829
:102A7000920701D5013BFAD1406880F00200C0F313
:102A800040007047806900F0700070478069000E58
:102A900070478069C0F30740704743690AB1194322
:102AA00001E023EA01014161704711F4700F01D088
:102AB00083690BE0CB0101D5436807E00A0101D52A
:102AC000836803E08B014CBFC3680369C3F313033E
:102AD0000B420CBF0020012070470A4B994202D1E3
:102AE0000023836170478A01C1F3130301D5C360DA
:102AF00070474A0101D5036170470A014CBF8360EA
:102B0000436070477000F03043690B405CD040294F
:102B100042D010D8042933D005D8012927D0022962
:102B200054D1C0682FE010292CD0202930D008299A
:102B30004CD1C06835E0B1F5006F3BD00CD8B1F591
:102B4000007F31D0B1F5806F32D0B1F5807F3DD1BB
:102B5000806900F001007047B1F5803F1ED0B1F5EB
:102B6000003F1DD0B1F5004F30D1406829E08068AA
:102B700000F0013020F08070003018BF0120704755
:102B8000C06806E0006910F0030018BF012070471C
:102B90000069C0F3C0007047006902E04068F8E7D0
:102BA0004068C0F3001070478069C0F34000704770
:102BB000806906E0836913F0700F0CBF00200120CC
:102BC0007047C0F380007047184670470020704778
:102BD000B1F5807F35D00CD8082924D004D801293C
:102BE0001CD004291DD0704720291FD040291FD098
:102BF0007047B1F5006F22D006D8B1F5007F20D024
:102C0000B1F5806F1DD07047B1F5803F13D0B1F59D
:102C1000003F12D0B1F5004F15D110E00A4B836090
:102C20007047082300E01023C3607047082300E0CA
:102C3000102303617047082304E0102302E00023FF
:102C4000836104234360704701010100036823F09E
:102C5000010303600023036043608360C36003617A
:102C600021234361294B984217D0294B98421BD00E
:102C7000284B984220D0284B984225D0274B984289
:102C80002AD0274B98422ED0264B984232D0264B42
:102C9000984236D0254B984203D13D2243F8082C68
:102CA0007047234B984204D14FF4746243F8202CB0
:102CB0007047204B984204D14FF4741243F8382CDB
:102CC00070471D4B984204D14FF0746243F8502C6A
:102CD00070471A4B984203D1194A43F8642C704745
:102CE000184B984203D1184A43F87C2C7047174B75
:102CF000984203D1164A43F8942C7047154B9842DA
:102D000003D14FF03D5243F8AC2C704710600240A5
:102D100028600240406002405860024070600240FB
:102D200088600240A0600240B86002401064024027
:102D300028640240406402405864024070640240CB
:102D40003D00002088640240400F0020A064024043
:102D500000003D20B86402400268134B10B51340D8
:102D6000CC680A6814434A6914438A691443CA69DF
:102D700014430A6A14434A6A14438A6A14434A6B26
:102D800014438A6B22431343036044690A6BCB6A82
:102D900024F007041343234343610B6943604B68EA
:102DA00083608B68C36010BD3F801CF0002303600C
:102DB00043608360C360036143618361C3610362F5
:102DC00043628362C3620363436383637047036840
:102DD00011B143F0010301E023F0010303607047E8
:102DE000036811B143F4004301E023F4004303609E
:102DF0007047036811B143F0200301E023F0200382
:102E00000360704741607047406880B27047036854
:102E100012B143F4002301E023F4002303600161B5
:102E20007047036811B143F4802301E023F4802349
:102E3000036070470AB101617047C1607047006864
:102E4000C0F3C0407047006800F00100704740695F
:102E500000F0380070470A4B10B50A4A0A4CA042ED
:102E60008CBF104618468B004CBF4368036821F0A6
:102E7000F02121F0821119420CBF0020012010BD69
:102E800000600240006402400F64024010B5084B2D
:102E9000084A094CA0428CBF1046184611F0005F4A
:102EA00021F0F02121F0821114BFC160816010BDBA
:102EB00000600240006402400F6402400B0611D51E
:102EC00043694AB143F080038029436114D0036809
:102ED00001F01E0119430EE023F0800380294361B5
:102EE00004D17047802907D0002AF0D1036801F08F
:102EF0001E0123EA01010160704730B5104B114AF1
:102F0000114D21F0F024A8428CBF15461D4624F037
:102F1000C3132BB1026802F01E0202EAD12202E0C2
:102F2000426902F080028B004CBF6B682B6824F072
:102F30008210184002D0101C18BF012030BD00BF05
:102F400000600240006402400F64024010B5084B6C
:102F5000084A094CA0428CBF1046184611F0005F89
:102F600021F0F02121F0821114BFC160816010BDF9
:102F700000600240006402400F640240044B0022E3
:102F80001A605A609A60DA60024A5A61704700BF5C
:102F9000003C0140FFFF7F00837930B50168027972
:102FA00043B3194BCC431D6802F1804225401D609C
:102FB0005D6802F59E322C405C601468214311600C
:102FC00002689C68D1430C409C60DC682140D96059
:102FD0004179102906D1996811439960D9680A434B
:102FE000DA6030BD01F1804303F59E3319680A436E
:102FF0001A6030BD02F1804303F59E331A6822EA5D
:103000000101196030BD00BF003C014000230C22CB
:1030100003600371427183717047024B1A69104358
:1030200018617047003C0140034B5B6918420CBFBC
:1030300000200120704700BF003C0140014B586157
:10304000704700BF003C0140054B1A685B690340B4
:1030500004D010420CBF0020012070471846704772
:10306000003C0140014B5861704700BF003C0140EB
:1030700008B52C4B984205D10120014600F04CFACE
:10308000012048E0284B984205D10220012100F0A0
:1030900043FA02203FE0254B984205D1042001214C
:1030A00000F03AFA042036E0214B984205D108207E
:1030B000012100F031FA08202DE01E4B984205D185
:1030C0001020012100F028FA102024E01A4B984229
:1030D00005D12020012100F01FFA20201BE0174B12
:1030E000984205D14020012100F016FA402012E05C
:1030F000134B984205D18020012100F00DFA802069
:1031000009E0104B98420BD14FF48070012100F080
:1031100003FA4FF480700021BDE8084000F0FCB9CC
:1031200008BD00BF00000240000402400008024049
:10313000000C02400010024000140240001802403F
:10314000001C0240002002402DE9F0410F680023DE
:1031500001229A4002EA0705954231D15A00032420
:1031600094400668E443264006600E79D0F800C01B
:1031700006FA02F8013EF6B248EA0C0C012EC0F83D
:1031800000C014D891F805C086680CFA02FC2640ED
:10319000866086684CEA06068660466826EA05056B
:1031A00045608D7946689D40ADB235434560C56840
:1031B0002C40CD79C46005FA02F2C4682243C26093
:1031C0000133102BC4D1BDE8F0814FF6FF730360CB
:1031D0000023037143718371C371704782B04FF450
:1031E00080330193019B0B430193019BC361C16138
:1031F000019BC361C3690193C369019302B0704726
:10320000036919420CBF002001207047006980B299
:103210007047436919420CBF002001207047406984
:1032200080B2704701837047418370470AB10183C0
:10323000704741837047416170474369594041611C
:10324000704701F00703C90800EB81009B000F21C4
:1032500099409A4010B5046A24EA01010162016AAA
:103260001143016210BD00BF0A4B00211A6842F0F1
:1032700001021A6099601A6822F0847222F4803286
:103280001A60054A5A601A6822F480221A60D960CE
:10329000704700BF0038024010300024024B00226B
:1032A0001A701870704700BF02380240034B1A684A
:1032B00022F0F80242EAC00018607047003802406D
:1032C000014B1860704700BF00004742064B0022C8
:1032D00001281A701A7002D0042802D070471870A2
:1032E000704705221A70704770380240014B186011
:1032F000704700BF800E474210B5029C5B0840EA51
:1033000004600143013B41EA821242EA0344014B5B
:103310005C6010BD00380240014B1860704700BF70
:10332000600047420907034B41EA8010C3F884005C
:10333000704700BF00380240014B1860704700BF63
:1033400068004742014B1860704700BF4C0047427D
:10335000034B9A6822F0EC6211430843986070476F
:1033600000380240034B9A6822F078421143084328
:103370009860704700380240034B9A6822F00302BD
:1033800010439860704700BF00380240024B9868B5
:1033900000F00C00704700BF00380240034B9A68F1
:1033A00022F0F00210439860704700BF00380240DE
:1033B000034B9A6822F4E05210439860704700BFB4
:1033C00000380240034B9A6822F4604242EAC0008F
:1033D0009860704700380240194B10B59968194A37
:1033E00001F00C01042913D0082911D15C68596837
:1033F0005B6801F03F01C3F38813B2FBF1F25A435B
:103400000F4B5B68C3F3014301335B00B2FBF3F284
:103410000B4902608B680C4AC3F30313D45C036846
:10342000E34043608C68C4F38224145D23FA04F4FF
:1034300084608968C1F34231525CD340C36010BDDF
:10344000003802400024F400D000002000F4407353
:10345000B3F5407F084B08D1996820F0704221F401
:10346000F81122F440720A439A601A6FC0F30B00FD
:1034700010431867704700BF00380240014B1860C6
:10348000704700BF3C0E4742014B1860704700BFB9
:10349000400E4742014B1860704700BF5C01474235
:1034A000044B1A6B09B1104301E022EA00001863D3
:1034B000704700BF00380240044B5A6B09B11043FB
:1034C00001E022EA00005863704700BF0038024064
:1034D000044B9A6B09B1104301E022EA00009863A3
:1034E000704700BF00380240044B1A6C09B110430A
:1034F00001E022EA00001864704700BF0038024073
:10350000044B5A6C09B1104301E022EA00005864F0
:10351000704700BF00380240044B1A6909B11043DC
:1035200001E022EA00001861704700BF0038024045
:10353000044B5A6909B1104301E022EA00005861C6
:10354000704700BF00380240044B9A6909B110432C
:1035500001E022EA00009861704700BF0038024095
:10356000044B1A6A09B1104301E022EA0000186214
:10357000704700BF00380240044B5A6A09B110433B
:1035800001E022EA00005862704700BF00380240A4
:10359000044B1A6D09B1104301E022EA00001865DE
:1035A000704700BF00380240044B5A6D09B1104308
:1035B00001E022EA00005865704700BF0038024071
:1035C000044B9A6D09B1104301E022EA00009865AE
:1035D000704700BF00380240044B1A6E09B1104317
:1035E00001E022EA00001866704700BF0038024080
:1035F000044B5A6E09B1104301E022EA00005866FC
:10360000704700BF00380240044B1A7809B11043DC
:1036100001E022EA00001870704700BF0D38024038
:103620004309012B074A01D1136803E0022B0CBFA9
:10363000136F536F00F01F0023FA00F000F0010039
:10364000704700BF0038024007B5002301933120C6
:10365000FFF7E6FF019B01330193019BB3F5A06FD8
:1036600001D00028F3D03120FFF7DAFF003018BF77
:10367000012003B05DF804FB024B5A6F42F08072E8
:103680005A67704700380240034BDB6818420CBF92
:1036900000200120704700BF00380240014B187025
:1036A000704700BF0E38024008B5154B98420BD149
:1036B0004FF480500121FFF75FFFBDE808404FF451
:1036C00080500021FFF758BF0E4B984207D14FF4AE
:1036D00080400121FFF744FF4FF4804009E00A4B8E
:1036E00098420BD14FF400400121FFF739FF4FF40E
:1036F00000400021BDE80840FFF732BF08BD00BF11
:103700000030014000380040003C00400B8810B5FC
:103710004C88028823438C8802F441522343CC888E
:1037200023430C8923434C8923438C892343CC892D
:10373000234313439BB20380838B23F400631B0456
:103740001B0C83830B8A038210BD838BF0B523F49B
:103750007B6323F00F031B041B0C8383022303846E
:103760008B68858B022BADB238D08A88002A294A13
:1037700014BF022601269468240203D5946824F419
:1037800000049460D2F88440D2F884705268DFF864
:1037900088C002F03F02BCFBF2F2C4F38814544329
:1037A000C7F30272B4FBF2F4CA88B2F5007F18BF07
:1037B00076014FF00A020CBF240AB4FBF6F4624310
:1037C000B2FBF3F305330A229BB2B3FBF2F303F02F
:1037D00001021202C3F34F0392B200E000229C1ECA
:1037E000A4B2FE2C28BF0022CC8828BF022313439A
:1037F00023430A889BB2038445EA02034A8843F4C0
:10380000006313438A8813438A8913439BB28383DB
:10381000F0BD00BF003802400024F4000023038004
:1038200043808380C380038143818381C3810723D5
:103830000382704700230222038043808380C38079
:10384000826083817047038819B19BB243F04003C3
:1038500003E023F040031B041B0C03807047838BA1
:1038600019B19BB243F4806303E023F480631B042B
:103870001B0C83837047038823F400631B041B0C19
:10388000038003889BB2194301807047B1F5804FD4
:10389000038803D19BB243F4804303E023F48043C5
:1038A0001B041B0C038070474FF6FF63994203888B
:1038B00003D09BB243F4807303E023F480731B04B2
:1038C0001B0C03807047838819B19BB243F004033B
:1038D00003E023F004031B041B0C838070478388E0
:1038E00019B19BB243F0100303E023F010031B0453
:1038F0001B0C83807047808980B27047818170473C
:10390000038819B19BB243F4005303E023F400533E
:103910001B041B0C0380704703889BB243F4805345
:1039200003807047012914BF008B808A80B27047E2
:10393000008A80B2704783889BB20AB1194301E0C4
:1039400023EA010181807047090901238B409BB262
:103950001AB1828892B2134303E0828892B222EABB
:10396000030383807047038919420CBF00200120A4
:103970007047C94389B20181704701F00F020123EA
:1039800003FA02F210B584880089A4B280B2104014
:1039900005D009098B401C420CBF0020012010BD3E
:1039A00001F00F0101238B40DB439BB20381704781
:1039B00008B54FF480400121FFF7DEFDBDE8084067
:1039C0004FF480400021FFF7D7BD014B18607047CE
:1039D0000038014001F003039B000F229A409840F9
:1039E00001F0FC0101F1804101F59C3110B58C68BA
:1039F00024EA02028A608A6802438A6010BD014B91
:103A000018607047DC002742014B1860704700BF08
:103A100000042742024B186AC0F30020704700BF21
:103A20000038014030B5048C24F001042404240C37
:103A30000484058B048CADB225F0F305A4B22A43AF
:103A400024F00A0442EA031344F001049DB2214326
:103A50000583018430BD30B5048C24F010042404A7
:103A6000240C0484058B048C25F44075A4B22D0528
:103A70002D0D24F0A00444F0100445EA022242EA8D
:103A8000033344EA01119BB28CB20383048430BD3A
:103A900008B5474B984205D101200146FFF76CFD60
:103AA00001203DE0B0F1804F05D101200146FFF734
:103AB00057FD012076E03F4B984205D102200121BD
:103AC000FFF74EFD02206DE03B4B984205D10420EC
:103AD0000121FFF745FD042064E0384B984205D1F1
:103AE00008200121FFF73CFD08205BE0344B9842A1
:103AF00005D110200121FFF733FD102052E0314B9A
:103B0000984205D120200121FFF72AFD202049E01D
:103B10002D4B984209D102200121FFF72DFD0220F3
:103B20000021BDE80840FFF727BD284B984207D188
:103B30004FF480300121FFF71FFD4FF48030EFE795
:103B4000234B984207D14FF400300121FFF714FDB9
:103B50004FF40030E4E71F4B984207D14FF4802028
:103B60000121FFF709FD4FF48020D9E71A4B984255
:103B700005D140200121FFF7F3FC402012E0174B54
:103B8000984205D180200121FFF7EAFC802009E05E
:103B9000134B98420BD14FF480700121FFF7E0FCEA
:103BA0004FF480700021BDE80840FFF7D9BC08BD84
:103BB000000001400004004000080040000C0040EC
:103BC000001000400014004000040140004001408B
:103BD000004401400048014000180040001C004023
:103BE000002000401C4A038890429BB212D002F58C
:103BF000806290420ED0B0F1804F0BD0A2F580329F
:103C0000904207D002F58062904203D002F58062B4
:103C1000904203D14A8823F0700313430F4A904225
:103C200008D002F58062904204D023F440730A89E0
:103C30009BB2134303804B68C3620B880385064B1A
:103C4000984203D003F58063984201D18B7A0386B2
:103C500001238382704700BF000001400010004034
:103C60004FF0FF334360002303800381438083725E
:103C70007047018582827047038823F070031B041C
:103C80001B0C19430180704741627047C162704745
:103C9000406A7047008D80B27047038819B19BB2AB
:103CA00043F0020303E023F002031B041B0C038018
:103CB0007047038819B19BB243F0040303E023F07B
:103CC00004031B041B0C03807047038819B19BB2CB
:103CD00043F0800303E023F080031B041B0C0380EC
:103CE0007047038823F008031B041B0C0380038820
:103CF0009BB2194301807047038823F440731B046F
:103D00001B0C038003889BB2194301807047038812
:103D100019B19BB243F0010303E023F001031B043C
:103D20001B0C03807047038C70B523F001031B0448
:103D30001B0C0384038C8488028B0D8822F0730291
:103D40001204120C2A434E888D8923F002031B04AF
:103D50003543ADB21B0C2B430E4DA4B2A84203D089
:103D600005F58065A8420ED1CD8923F008032B43C9
:103D70008D8823F004032B434E8A0D8A24F440746B
:103D80003543ADB22C43848002838A684263038446
:103D900070BD00BF00000140038C30B523F010035C
:103DA0001B041B0C0384038C8288048B0D8824F471
:103DB000E6442404240C23F0200344EA05241B04D5
:103DC0008D891B0C43EA05134D8892B243EA051313
:103DD000124DA4B2A8429BB203D005F58065A8425B
:103DE00015D1CD8923F080039BB243EA05134FF62A
:103DF000BF751D408B8822F4406245EA03130D8A8B
:103E00009BB242EA85024D8A42EA850292B28280E2
:103E10008A6804838263038430BD00BF00000140D0
:103E2000038C30B523F480731B041B0C0384038CB8
:103E30008288848B0D8824F073042404240C23F4DA
:103E400000732C431B048D891B0C43EA05234D880A
:103E500092B243EA0523124D9BB2A84203D005F566
:103E60008065A84215D1CD8923F400639BB243EA53
:103E700005234FF6FF351D408B8822F4405245EA5A
:103E800003230D8A9BB242EA05124D8A42EA0512CB
:103E900092B282808A688483C263038430BD00BF8B
:103EA00000000140038C30B523F480531B041B0C2D
:103EB0000384038C8488828B0D8822F4E6421204EA
:103EC000120C23F4005342EA05221B048D891B0CBB
:103ED00043EA05334D88A4B243EA05330A4D92B252
:103EE000A8429BB203D005F58065A84205D10D8A92
:103EF00024F4804444EA8514A4B2848082838A68CE
:103F00000264038430BD00BF000001400023038031
:103F10004380838083608381C381038243827047AF
:103F200030B501248C40058C00F11803ADB225EAB0
:103F30000404048421F0080038B949085C584FF69D
:103F40008F702040585058580AE00439C1F34E0190
:103F5000CC5848F6FF702040C8501202C85892B2A0
:103F60000243CA5030BD4163704781637047C163EB
:103F7000704701647047038B23F070031B041B0C14
:103F8000194301837047038B23F4E0431B041B0C8C
:103F900043EA01218BB203837047838B23F07003C4
:103FA0001B041B0C194381837047838B23F4E0436C
:103FB0001B041B0C43EA01218BB283837047038BE4
:103FC00023F008031B041B0C194301837047038B68
:103FD00023F400631B041B0C43EA01218BB203830F
:103FE0007047838B23F008031B041B0C1943818348
:103FF0007047838B23F400631B041B0C43EA0121ED
:104000008BB283837047038B23F004031B041B0CC8
:10401000194301837047038B23F480631B041B0C3B
:1040200043EA01218BB203837047838B23F004039F
:104030001B041B0C194381837047838B23F480631B
:104040001B041B0C43EA01218BB283837047038B53
:1040500023F080031B041B0C194301837047038B5F
:10406000C3F30E0343EA01218BB203837047838BB2
:1040700023F080031B041B0C194381837047838B3F
:10408000C3F30E0343EA01218BB283837047038C91
:1040900023F002031B041B0C194301847047038C9B
:1040A00023F008031B041B0C194301847047038C85
:1040B00023F020031B041B0C43EA01118BB2038481
:1040C0007047038C23F080031B041B0C43EA01118F
:1040D0008BB203847047038C23F400731B041B0C06
:1040E00043EA01218BB203847047038C23F40063FD
:1040F0001B041B0C43EA01218BB203847047038C21
:1041000023F400531B041B0C43EA01318BB20384DC
:10411000704701238B408A4010B5048CA4B224EA76
:1041200003030384038C13439BB2038410BD042355
:104130008B408A4010B5048CA4B224EA03030384A4
:10414000038C13439BB2038410BD00230122038020
:1041500043808280C38003817047406B7047806BCF
:104160007047C06B7047006C7047038B23F00C03E3
:104170001B041B0C0383038B9BB219430183704701
:10418000038B23F440631B041B0C0383038B9BB240
:1041900043EA01218BB203837047F8B50C46498886
:1041A000A2880029B4F800E014BF00270227012AE2
:1041B000054614BF012602262389BEF1000F11D146
:1041C000FFF730FC2846E188FFF7CFFF2846394645
:1041D00032462389FFF73FFC2846E188BDE8F840D6
:1041E000FFF7CEBFFFF737FC2846E188FFF7C8FF8F
:1041F0002846394632462389FFF714FC2846E188D1
:10420000BDE8F840FFF7B1BF838B23F00C031B041C
:104210001B0C8383838B9BB2194381837047838BF1
:1042200023F440631B041B0C8383838B9BB243EA00
:1042300001218BB283837047F8B50E880D46044682
:104240004988AA882B893EB9FFF7ECFB2046E9880C
:10425000BDE8F840FFF789BF042E07D1FFF7FBFB4D
:104260002046E988BDE8F840FFF78ABF082EB5F878
:1042700006C0078C1CD127F480773F043F0C0784CD
:10428000868B058CB6B2ADB226F0F30625F4206518
:1042900046EA031345EA01219BB289B21A4341F46D
:1042A00080718283BDE8F84001846146FFF7ACBFAE
:1042B00027F480573F043F0C0784868B058C26F437
:1042C000407625F4005536056D046D0C360D46EA32
:1042D000022645EA013146EA033389B29BB241F432
:1042E000805183830184BDE8F8406146FFF797BFA2
:1042F0004A880B8813438A881343CA8813430A8960
:1043000013434A8913438A8913439BB2A0F844306C
:1043100070470023038043808380C38003814381EF
:1043200083817047B0F8443029B16FEA43436FEAA4
:1043300053439BB201E0C3F30E03A0F8443070472F
:10434000838819B19BB243F0040303E023F0040314
:104350001B041B0C83807047838819B19BB243F008
:10436000010303E023F001031B041B0C838070474F
:1043700083899BB20AB1194301E023EA01018181DB
:10438000704781827047038A19420CBF00200120C8
:104390007047C94389B201827047038A828911EA52
:1043A000030092B203D011420CBF002001207047DD
:1043B000C94389B2018270470A43A0F84820704778
:1043C00083899BB20AB1194301E023EA010181818B
:1043D0007047838819B19BB243F0080303E023F0D0
:1043E00008031B041B0C83807047038923F0070319
:1043F0001B041B0C03817047038923F070031B040B
:104400001B0C1943018103899BB243F0070303810D
:10441000704738B50D46602D114604464FF0010235
:1044200002D1FFF718FB01E0FFF7FCFA238923F024
:1044300070031B041B0C2B43238123899BB243F085
:104440000703238138BD038923F070031B041B0C71
:10445000194301817047838823F070031B041B0CF0
:10446000838083889BB2194381807047038923F03E
:1044700007031B041B0C038103899BB219430181B1
:104480007047038923F080031B041B0C03810389FD
:104490009BB219430181704710B50489E4B22143EE
:1044A0000A4342EA03239CB2048110BD10B50446BE
:1044B000FFF7F2FF238923F077031B041B0C43F063
:1044C0007703238110BD10B50446FFF7E5FF23896C
:1044D0009BB243F48043238110BD70B50589048BE2
:1044E000068C24F44074B6B224F0030426F02206AD
:1044F00025F00705240432432D04240C2D0C44F42C
:10450000807442EA0313294344F001049EB20181FE
:104510000483068470BD838819B19BB243F0800385
:1045200003E023F080031B041B0C83807047A0F87A
:104530005010704708B5234B984205D11020012137
:10454000FFF71AF8102037E01F4B984207D14FF4BD
:1045500000300121FFF704F84FF4003009E01B4B55
:1045600098420BD14FF480200121FEF7F9FF4FF460
:1045700080200021BDE80840FEF7F2BF144B9842AE
:1045800007D14FF400200121FEF7EAFF4FF400208D
:10459000EFE7104B984207D14FF480100121FEF74E
:1045A000DFFF4FF48010E4E70B4B984209D1202045
:1045B0000121FEF7E1FF20200021BDE80840FEF7C1
:1045C000DBBF08BD0010014000440040004800402F
:1045D000004C00400050004000140140038ACA888B
:1045E0009BB223F4405330B513430D46038209892F
:1045F000AB8882890B43698992B20B4322F4B05293
:1046000022F00C029BB213438381838AAA899BB256
:1046100023F44073134385B0838204466846FEF753
:10462000DBFE194B9C4203D003F580639C4201D111
:10463000039B00E0029BA289192112B25943002A70
:104640002A684FF06403B4BF52009200B1FBF2F14C
:10465000B1FBF3F21201100903FB1011A08900B2A3
:10466000002806DAC9003231B1FBF3F303F0070387
:1046700005E009013231B1FBF3F303F00F031A43F4
:1046800092B2228105B030BD001001404FF41653A4
:1046900003600C2200238380C380038142818381D5
:1046A00070470B8810B54C88028A23438C88C988D0
:1046B000234392B20B4322F470629BB213430382F2
:1046C00010BD0023038043808380C38070478389AB
:1046D00019B19BB243F4005303E023F400531B04CD
:1046E0001B0C83817047038B03F47F430383038B8D
:1046F0009BB2194301837047838929B16FEA434311
:104700006FEA53439BB201E0C3F30E03838170470A
:10471000838A19B19BB243F4006303E023F400637E
:104720001B041B0C83827047C1F308018180704712
:104730008088C0F308007047038A23F00F031B042E
:104740001B0C0382038A9BB2194301827047838941
:1047500019B19BB243F0020303E023F002031B04F0
:104760001B0C83817047838923F400631B041B0C9B
:10477000838183899BB2194381817047038A23F027
:1047800020031B041B0C0382038A9BB21943018282
:104790007047038A19B19BB243F4804303E023F4CA
:1047A00080431B041B0C0382704783899BB243F038
:1047B000010383817047838A19B19BB243F00803D8
:1047C00003E023F008031B041B0C83827047038B58
:1047D000DBB20383038B9BB243EA01210183704761
:1047E000838A19B19BB243F0200303E023F0200336
:1047F0001B041B0C83827047838A19B19BB243F060
:10480000100303E023F010031B041B0C838270478A
:10481000838A23F004031B041B0C8382838A9BB2CC
:10482000194381827047838A19B19BB243F0020316
:1048300003E023F002031B041B0C83827047838A6E
:104840009BB20AB1194301E023EA0101818270475A
:10485000C1F3421310B5012401F01F01A34204FA71
:1048600001F101D10C3003E0022B0CBF10301430E9
:1048700003680AB1194301E023EA0101016010BD98
:10488000038819420CBF002001207047C94389B238
:104890000180704710B5C1F3421401F01F030122DB
:1048A000012C02FA03F201D1838903E0022C0CBF30
:1048B000038A838A9BB21340028892B243B10123D8
:1048C000090A03FA01F111420CBF0020012010BDBA
:1048D000184610BD090A01238B40DB439BB20380BD
:1048E000704700BF40F0BF60024B40F40030D8601A
:1048F000704700BF00ED00E0C27810B503780AB33E
:10490000164A4478D26803F16043D243C2F30222CC
:10491000C2F10401C9B204FA01F10F2444FA02F20F
:104920008478C9B222400A431201D2B203F561432E
:1049300083F8002303780122590903F01F0302FAC8
:1049400003F306E05909012203F01F0302FA03F3FF
:104950002031034A42F8213010BD00BF00ED00E0D5
:1049600000E100E021F0604121F07F01014B0843AC
:104970009860704700ED00E0044B1A6909B11043DC
:1049800001E022EA00001861704700BF00ED00E07E
:10499000044B04281A680CBF42F0040222F00402FF
:1049A0001A60704710E000E010B5D0F8E835044612
:1049B0001B699847032384F81231002010BD08B505
:1049C00090F8123180F81331042380F81231D0F8B6
:1049D000E835DB689847002008BD08B5D0F8E43515
:1049E000DB6903B19847002008BD08B5D0F8E4356D
:1049F0001B6A9847002008BD08B5D0F8E4355B6A0B
:104A00009847002008BD10B5D0F8E83504465B692A
:104A10009847012384F81531002010BDD0F8E835FF
:104A200010B59B6904469847D4F8E43520465B6886
:104A300000219847002084F8150110BD002110B511
:104A40000B460446402201F04FF9802140222046C7
:104A5000002301F049F9012384F81231D4F8E83534
:104A6000A0785B689847002010BD13B569460446DE
:104A700000F074FA9DF8001001F01F03012B0CD018
:104A800006D3022B0ED12046694600F0DBFB0EE078
:104A90002046694600F092FA09E02046694600F097
:104AA000B9FB04E0204601F0800101F08AF9002002
:104AB00002B010BD70B50446002947D190F81131FD
:104AC000022B37D1D0F83821D0F824319A4211D9AD
:104AD000C178D21A0129C0F8382104D1D0F82811A0
:104AE0000B44C0F828312046D4F8281192B200F0C7
:104AF000EEF91FE0D0F83C51B5FBF3F603FB165678
:104B00005EB99D4209D3D0F840319D4205D232466C
:104B100000F0DDF9C4F840610CE0D4F8E435DB685E
:104B20002BB194F81221032A01D120469847204640
:104B300000F0FFF994F81631012B10D1094A2369CE
:104B400012685A60002384F8163108E0D0F8E43582
:104B50005B6923B190F81221032A00D19847002005
:104B600070BD00BF2435012010B5044659BB90F834
:104B70001131032B30D1D0F89023D0F87C339A42F6
:104B800014D9C178D21A0129C0F8902304D1D0F8E1
:104B900080131944C0F880139A4228BF1A46204651
:104BA000D4F8801392B200F0ACF915E0D0F8E435F7
:104BB0001B6923B190F81221032A00D1984720469F
:104BC00000F0A8F908E0D0F8E4359B6923B190F82B
:104BD0001221032A00D19847002010BD2DE9F04191
:104BE000069F0446164698460D46F6F70BF82046F3
:104BF0002946C4F8E485C4F8E875C4F8EC6501F00A
:104C000027F8D4F8E8351B6898472046BDE8F041FE
:104C1000F6F74AB800207047D0F8E43510B51B68A5
:104C200004469847D4F8E8359B689847002010BDA3
:104C300008B5D0F8E4355B689847002008BD00BF90
:104C400010B5074C2068FF2807D0064B064A9B6822
:104C5000064912689847FF232360002010BD00BF5B
:104C600010010020A800002030280120AB350120D1
:104C700043230B8000487047140100201B4970B586
:104C80004B685A1C052B4A602ED10A7A0023012A50
:104C90004B6029D0CA68B2F5006F08BFCB60CC6802
:104CA0000A69124B944202D100221A721CE08CBF96
:104CB000C4F50062C4EB02025A614E690B4D402EEE
:104CC000A2B205D94034403EEC606E61402304E05E
:104CD0003444EC600024B3B26C6101240C72044CC7
:104CE0008121224401F054F8002070BD30280120B9
:104CF000B335012038B5282303FB0101074C084BCD
:104D000005461B692046B1F88C13984728460121B7
:104D10002246402301F021F8002038BD6B350120E8
:104D2000A800002070B50B78064613F060050C460D
:104D300027D0202D21D1CD884A78BDB11B060BD5B7
:104D4000214B10469B682A462049984730461F4908
:104D5000E28800F0ABF807E01D4B1C491A601D4BC0
:104D60002A461D6000F0BCF800252BE0164B1046CB
:104D70009B6829462A46984724E000F011F902254D
:104D800020E04B780A2B11D00B2B14D0062B19D115
:104D90004B881B0A212B05D1CA880F493A2A28BF04
:104DA0003A2201E00D493A22304601E00C49012245
:104DB00000F07CF806E08B7813B9064B9D6101E0AA
:104DC00000F0EEF8284670BDA8000020AB350120A9
:104DD0001001002030280120260100201D010020A4
:104DE0004828012010B58121044600F09EFF20468E
:104DF000012100F09AFF8221204600F096FF024B2D
:104E00005B689847002010BDA800002038B58121BC
:104E100004464022022300F067FF20460121402281
:104E2000022300F061FF822120460822032300F0C4
:104E30005BFF084B022200251A715D71064B1B684F
:104E4000984720460121054A402300F086FF284666
:104E500038BD00BF44000020A80000206B350120B1
:104E600038B510490B7A012B19D14C690CB90C7269
:104E700015E0402C07D9CB68403C9AB24033CB6058
:104E80004C61402306E0CD68A3B22C44CC600024E2
:104E9000AAB24C61044C8121224400F079FF002029
:104EA00038BD00BF30280120B335012038B5044695
:104EB000C4F83C21C4F838210D461346022280F87C
:104EC000112100212A4600F063FF002038BD10B5F3
:104ED0000C4613460021224600F05AFF002010BD68
:104EE00038B50446C4F89423C4F890230D461346FD
:104EF000032280F8112100212A4600F02EFF002015
:104F000038BD10B50C4613460021224600F025FF9F
:104F1000002010BD10B50021042304460A4680F885
:104F200011310B4600F034FF204600F0C6FD002092
:104F300010BD10B50021052304460A4680F8113142
:104F40000B4600F00AFF204600F0B7FD002010BD20
:104F5000282303FB0101B1F88C03704790F8CC358E
:104F60000B7090F8CD354B7090F8CF2590F8CE357A
:104F700003EB02234B8090F8D12590F8D03503EB5A
:104F800002238B8090F8D32590F8D23503EB0223CF
:104F90009BB2CB80C0F84031012380F811317047BB
:104FA00010B58021044600F00CFF2046002100F0DF
:104FB00008FF2046BDE8104000F07FBD73B54B7878
:104FC00004460D46092B00F21681DFE813F0C700F6
:104FD00002011401DA0014016E000A001401B90084
:104FE0008D006B881A0A013A062A00F20481DFE874
:104FF00012F007001A00270002010201020102015B
:10500000D0F8EC350DF106011B6880789847EB88E5
:105010000146402B03D094F81231012B35D10823DF
:10502000ADF8063031E0D0F8E4350DF106019B6AA9
:1050300080789847022343700146C4F8F00524E0C5
:10504000DBB2052B00F2D780DFE803F003070B0F7C
:105050001317D0F8EC355B6812E0D0F8EC359B689C
:105060000EE0D0F8EC35DB680AE0D0F8EC351B69CF
:1050700006E0D0F8EC355B6902E0D0F8EC359B69CE
:105080000DF10601A07898470146BDF80630002BC7
:1050900000F0B580EA88002A00F0B1809A4228BF6B
:1050A0001A46ADF80620204668E0AB88002B40F099
:1050B000A280EB88002B40F09E8090F81231AE78F1
:1050C000032B06F07F0600F0968080F814613146CD
:1050D00000F0B7FE2046FFF71DFF0EB1022300E0EF
:1050E000012384F812318AE0A978464E01293170F3
:1050F00000F2818090F81231022B02D0032B09D0EC
:1051000079E0002961D00121032380F8101180F893
:10511000123111E039B9022380F8123180F81011F0
:10512000FFF786FD51E090F8101101294DD0FFF7EF
:105130007FFD317884F810112046FFF76DFD44E0C3
:10514000EA88012A57D190F81231022B04D0032BA0
:1051500051D100F5887111E02B490FE090F8123120
:10516000023B012B47D8274B01229A60D0F8182127
:105170000AB103229A60254920460222FFF796FED3
:105180003DE06B88012B2DD0022B38D1AA8812F07C
:10519000FF0F34D10369120A013A5B68042A0FD861
:1051A000DFE802F0030507090B00012206E00222F6
:1051B00004E0032202E0042200E0052262F3061369
:1051C000134A1360012384F816312046FFF7A2FE2C
:1051D00015E090F81231023B012B0CD86B88012BA3
:1051E0000DD10023C4F81831D4F8E43520469B686B
:1051F00029469847E9E720462946FFF7D1FE0020D7
:1052000002B070BD4C2801205028012054280120F4
:105210002435012038B590F812310446032B0D4691
:105220000CD10B79012B09D8D0F8E4359B6898474D
:10523000EB882BB92046FFF76DFE01E0FFF7B0FECB
:10524000002038BD70B54E788A88012E04460D4680
:10525000D3B210D027D3032E50D190F81221022AB6
:1052600028D0032A48D14A889AB95E0611D0194637
:1052700000F0A7FD0DE090F81221022A1AD0032AAF
:105280003AD14A88002A39D1590608D0194600F087
:10529000B2FDD4F8E43520469B682946984720465D
:1052A000FFF738FE2AE090F81251022D02D0032DAC
:1052B00006D021E05A0621D0194600F082FD1DE0FB
:1052C00012F0800F4FF028010D4A10D003F07F0339
:1052D00001FB030191F81E310BB1012300E0002313
:1052E000D360204607490222FFF7E0FD06E001FBFC
:1052F000030393F87633EFE7FFF752FE002070BD0B
:105300004C2801205828012030B5D0B10023DCB250
:105310000133C51815F8015C002DF8D1631C5B0042
:1053200013800B7003234B700138022310F8012FF8
:105330003AB15C1CCA54E4B202330022DBB20A5513
:10534000F4E730BD37B50023104C05460193032028
:10535000F5F7C0FC2B68013C1A69019213D0019A41
:10536000002AF4DA019A42F001020192019A1A61CC
:10537000064A1969013A019102D00199C907F8D486
:105380000320F5F7A7FC002003B030BD410D03005A
:1053900030B5C4786CB900EB82000333D0F8D0503C
:1053A0009B1022469A4204D051F822000132286014
:1053B000F8E7002030BD10B50332D0F8D04092108D
:1053C000002393424FEA830004D0206841F8230071
:1053D0000133F6E7084410BD0122F0B500238270C6
:1053E00001294FF04002C37082800CD10823037062
:1053F000042343704FF4A073C38002230372C1726D
:105400004FF0A04309E041B90C2303700623437019
:105410004FF4A063C380234BC17203F5006245784B
:105420000261C360024619460024AC4201F1200625
:1054300002F1040208D201F5106701F5306111652F
:10544000576101343146F0E7047803F58062426128
:1054500003EB441503F58862C0F8CC2005F5A06580
:1054600003F5A0620146AA4201F1040103D0C1F88C
:105470008C202032F7E703EB043403F5805204F567
:1054800080540146A24201F1040104D0C1F8CC20AD
:1054900002F58052F6E703F56063C0F80C31002096
:1054A000F0BD00BF0000044038B5037A0546012B6B
:1054B0004FF0000450F80C2F1ED1936B697A64F3FF
:1054C000104309B143F480139363D3686FF38613D9
:1054D0006FF396536FF351436FF3D343D360FFF7EA
:1054E00031FFEB78012B19D1052363F34404EB68FA
:1054F00044F020049C6011E0D36843F04003D36083
:10550000FFF720FF6B7AEA68002B0CBF4FF45023A3
:105510004FF4E81393631420F5F7E6FBEB78012BC7
:1055200007D1EB6805229C6862F3440444F0200430
:105530009C60002038BDC36800209A6842F00102D8
:105540009A607047C36800209A6822F001029A604E
:10555000704707B500230193019B43F0200301939B
:10556000019B61F38A130193019BC2681361074B8E
:105570001169013B019102D001998906F8D40320F9
:10558000F5F7A8FB002003B05DF804FB410D030014
:1055900007B500230193019B43F010030193019B86
:1055A000C2681361074B1169013B019102D0019957
:1055B000C906F8D40320F5F78DFB002003B05DF891
:1055C00004FB00BF410D0300C26808B5D368012980
:1055D0006FF35D736FF39E7302D143F0005302E0EB
:1055E00009B943F08043D3603220F5F77DFB0020FA
:1055F00008BDC368586900F001007047C368586966
:1056000000F0010080F001007047C368586900F0A5
:1056100001007047C3685A69986910407047C368B1
:105620005868704703691A6861F301021A6070478D
:1056300010B5C26800236FF080414FF0FF349361D2
:1056400051615460516109499161C17800209942CA
:1056500008BF102343F0804343F47013916943F46F
:10566000605343F00C030B43936110BD00080080AE
:1056700038B5D0F80C3100221A60036915461A6853
:10568000044665F3CC221A60C37A012B21D1032191
:10569000FFF7C8FFE36880214FF4001261F30F02A7
:1056A00059629A62A02262F30F0561F31F454FF41D
:1056B0009072C3F8045162F30F05C0F220054FF455
:1056C000A072C3F8085162F30F056FF31F45C3F8CA
:1056D0000C5110212046FFF73CFF2046FFF758FFF2
:1056E000236900224FF0FF311A615A619961DA6132
:1056F00061788A420FD204EB82018969013208681D
:105700000028ACBF00204FF09040086000200861E6
:10571000FF208860ECE7002261788A420FD204EB18
:105720008201496D013208680028ACBF00204FF0AB
:105730009040086000200861FF208860ECE71A694B
:1057400042F480721A61E278012A04D1044A4021AD
:1057500061F359421A632046FFF76AFF002038BD03
:105760000301010003699B68C3F34103022B05D0C9
:10577000032B05D0012B03D0032070470120704775
:1057800002207047036910B59C688169C4F3410029
:105790000A68022806BF032060F30A026FF30A02B8
:1057A0000A605A68002042F480725A6010BD30B519
:1057B0004D780B78012D4FF0000200EB830405D1EA
:1057C00005FA03F3A46963F30F0205E0012505FA66
:1057D00003F3646D63F31F4223681D040DD48D68C9
:1057E00065F30A03CD78C98865F3934361F3995350
:1057F00043F0805343F40043236003690020D969D8
:105800000A43DA6130BD30B54D780B780024012DA4
:10581000224600EB830105D105FA03F3896963F39E
:105820000F0205E0012505FA03F3496D63F31F42FA
:1058300003696FF3CF340C60D969002021EA0202BA
:10584000DA6130BDF8B54E780A460978012E536901
:1058500000EB810145D18D6929682C6963F312043D
:1058600013B966F3DC440BE096689F19013FB7FB60
:10587000F6F666F3DC44D678012E08BF66F35E7454
:105880002C61C4781578012C05D100EB8505AD6934
:1058900014696C610AE0D478012C07D033B1012778
:1058A00007FA05F50469666B35436563D478012C06
:1058B00007D10469A468E40554BF41F0005141F0E8
:1058C0008051147841F0044100EB8404A469216004
:1058D000D178012936D1D1689BB21278FFF758FDF3
:1058E00030E04E6D9568316834692BB965F3120468
:1058F000012363F3DC440AE02B44013BB3FBF5F3E3
:1059000063F3DC44C3F309035D4365F312043461BC
:10591000C378012B05D1137800EB83035C6D136909
:105920006361D378012B06D1537913B141F0005153
:1059300001E041F08051137841F0044100EB830015
:10594000436D19600020F8BDF7B591F801C04A69B0
:10595000BCF1010F3DD18469236826690096F5B238
:10596000C6F3074742B962F306056CF3C4078DF826
:1059700000508DF802700FE08E68B2428ABF66F365
:10598000060562F306054E6101223E4662F3C40637
:105990008DF800508DF80260009A2261C278012AC9
:1059A00005D10A7800EB820295690A696A6143F0C1
:1059B00004432360C378002B3FD14B69002B3CD0BC
:1059C0000A78012101FA02F20369586B02435A6313
:1059D00033E00B7800EB83035C6D23682569009549
:1059E000EFB2C5F307468D684AB9012265F3060791
:1059F00062F3C4068DF800708DF802600BE03A4641
:105A000065F306024D618DF800203546012262F3F0
:105A1000C4058DF80250009A2261C278012A05D18E
:105A20000A7800EB8202546D0A6962610A7843F0D9
:105A3000044300EB8200426D1360002003B0F0BD10
:105A40004B78012B0B7800EB830006D18269136839
:105A5000002B04DA43F0804301E0426D136843F405
:105A600000131360002070474B78012B0B78C97826
:105A700000EB83000CBF8269426D02391368C9B222
:105A80006FF35553012998BF43F0805313600020F2
:105A9000704703699A69D8691040000C704700EBA1
:105AA00081014B6D02699B6850691840704703691A
:105AB0009869DB69184080B2704782B00023009378
:105AC000C0238DF8033001224FF0000362F3C403BA
:105AD0008DF8023018238DF80030009A436D1A615A
:105AE000C278012A06D100F2CC5058611A684FF0F2
:105AF00080221A6002B07047D0F8183110B5044601
:105B0000D3B103699A68D20716D5827A42B1D0F828
:105B10000C21D0F80C116FF341026FF300020A6000
:105B20005A68052042F001025A60F5F7DDF8236952
:105B30005A6822F001025A6010BD837A63B103698A
:105B40009B68DB0708D5D0F80C31D0F80C216FF337
:105B500041036FF3000313607047012310B5002267
:105B600080F8123104460346617804338A4206D233
:105B70005869FF218160186D01328160F4E7236963
:105B800000221A615A61DA614FF0FF3220469A61B1
:105B9000FFF7FEFC20461021BDE81040FFF7D9BCFE
:105BA0004B78012B0B7800EB830009D183691B68CC
:105BB000990211D413F4003F0CBF3020202070470D
:105BC000436D1B689A0209D413F4003F0CBF4FF4D5
:105BD00040504FF400507047102070474FF48050F1
:105BE000704730B54D780C46012D0D7800EB8503DC
:105BF0000BD19D69102A2B6803D1BDE83040FFF717
:105C00001FBF202A0CD0302A0FE05D6DB2F5805FF7
:105C10002B6802D143F4001318E0B2F5005F02D103
:105C200043F0006312E0B2F5405F0CD19A0205D553
:105C300000236371BDE83040FFF716BF43F0044313
:105C400043F4004302E00AB962F3CF332B6030BD66
:105C500010B50446FFF7C0FB0123002284F812317F
:105C600084F814212346617828338A4212D2012114
:105C700083F8F5104020002183F8F420A3F8FA20DF
:105C800083F8F710C3F8FC00C3F80011C3F808113B
:105C90000132E8E723460022617828338A4211D294
:105CA0000021402083F84C23A3F8522383F84D139E
:105CB00083F84F13C3F85403C3F85813C3F86013A1
:105CC0000132E9E72046FFF73DFC2046FFF7ECFBF9
:105CD00020460021FFF778FC2046FFF7C9FC20464C
:105CE000BDE81040FFF727BC70B5CDB215F0800FAE
:105CF00001F07F044FF0280615BF06FB040106FBE8
:105D0000010101F58E7101F55D71E4B2ED090C70D0
:105D10004D708A60CB7005B1CC80022B04BF00238C
:105D20000B71FFF744FD002070BDCBB213F0800F64
:105D300001F07F0210B54FF0280415BF04FB0201EB
:105D400004FB010101F58E7101F55D71DB090A703B
:105D50004B70FFF758FD002010BD38B501F07F04EF
:105D6000282505FB040505F55D714B610023CA601C
:105D70008B614B7085F87443C378012B08BF0A61AF
:105D800014B9FFF7E1FD01E0FFF75CFD002038BD2D
:105D900070B501F07F04282505FB0405012605F5F3
:105DA0008E714E7085F81C41CA600A6100228A61BA
:105DB0004B6114B9FFF7C8FD01E0FFF743FD002078
:105DC00070BDCBB213F0800F01F07F0210B54FF021
:105DD000280415BF04FB020104FB010101F58E71CB
:105DE00001F55D71DB0901248C700A704B70FFF7BF
:105DF00027FE002010BDCBB213F0800F01F07F0210
:105E000010B54FF0280415BF04FB020104FB01018B
:105E100001F58E7101F55D710024DB098C700A704B
:105E20004B70FFF721FE204610BD08B50B0604D5C8
:105E300001F07F01FFF78DFB01E0FFF7A9FB0020D8
:105E400008BD0269002361F30A1311680B43136054
:105E50007047036903205A686FF341025A60F4F7F0
:105E600043BF036903205A6842F002025A60F4F704
:105E70003BBF11F0800F4FF0280306D001F07F01E7
:105E800003FB010101F58E7103E003FB010101F544
:105E90005D71FFF785BE11F0800F4FF0280306D02B
:105EA00001F07F0103FB010101F58E7103E003FBAB
:105EB000010101F55D71FFF794BE00002DE9F04F7F
:105EC00085B00446FFF79AFB08B900201DE2204682
:105ED000FFF7A0FB06460028F7D0C0F3C04000281B
:105EE0004FD02046FFF7D5FD27468046A1464FF00C
:105EF000000AB8F1000F43D018F0010F38D05FFA54
:105F00008AFB59462046FFF7CAFDC107054620D542
:105F10007B6D01259D60E278AA4207D11A69D9F804
:105F20007C33C2F312029B1AC9F88C33A64B20466D
:105F30001B6859461B689847E378012B09D1BAF1D1
:105F4000000F06D194F81131052B02D12046FFF73E
:105F5000B4FDAA0702D57B6D02259D602B0707D5EE
:105F6000994B20461B6808259B6898477B6D9D6070
:105F70000AF1010A4FEA5808043709F12809B8E77D
:105F80000120750340F1A3802046FFF790FDA04655
:105F9000824627464FF00009BAF1000F00F09680C4
:105FA0001AF0010F00F08A8023695FFA89FB1969F2
:105FB0005D6B04EB8B0225FA0BF59269ED0192689B
:105FC000EDB20D431540E8071CD5012505FA09F18E
:105FD0005A6B204622EA01025A63D8F81830594613
:105FE0009D60794B1B685B689847E378AB4209D1A9
:105FF000B9F1000F06D194F81131042B02D12046DB
:10600000FFF75BFD290703D5D8F8183008259D60F8
:10601000EA0603D5D8F8183010259D606B0603D525
:10602000D8F8183040259D60A80703D5D8F8183057
:1060300002259D60290641D5D7F83431D7F83021A3
:10604000D21AD7F824319A4238BF134603F1030C11
:10605000D8F818304FEA9C0C9B699BB2634529D94C
:10606000D7F83451D7F830319D4223D213B3D7F843
:1060700024215D1B954228BF154605F1030C4FEA0C
:106080009C0CABB2D7F8281120465A46CDF804C074
:10609000FFF77EF9D7F828312B44C7F82831D7F815
:1060A00034311D44C7F83451D8F81830DDF804C035
:1060B0009B69D2E7D8F8183080259D6009F1010965
:1060C0004FEA5A0A08F10408283765E70120B207A9
:1060D00002D5E36802225A61002E19DAA37A43B18D
:1060E000D4F80C31D4F80C216FF341036FF30003A3
:1060F0001360236920465A6822F001025A60324B2D
:106100001B689B699847E3684FF000425A61012081
:1061100033052DD500238DF80F3094F81231204629
:106120008DF80F30284B1B685B69984723694FF443
:1061300000619A68E3685961A37AC3B1D70716D59D
:1061400094F81531012B12D19DF80F30032B0ED18D
:10615000D4F80C311A6842F001021A601A6842F051
:1061600003021A60194B1A6942F006021A610120F3
:10617000350708D5144B20461B68DB689847E36851
:1061800008225A610120F10636D5E36828259A696C
:1061900022F010029A611F6A07F00F0305FB034506
:1061A000C7F34343022B05F55D7511D0062B1DD1B6
:1061B000204604F2CC510822FFF7FDF8AB69C7F383
:1061C0000A173B44AB6111E0E000002000ED00E065
:1061D000C7F30A1757B13A462046E968FFF7EBF8CC
:1061E000EB683B44EB60AB691F44AF61E36801209F
:1061F0009A6942F010029A61F20434D523690025AD
:106200005A68204622F001025A602946FFF7A1F998
:1062100023462A46617804338A4206D25869FF2110
:106220008160186D01328160F4E7236901274FF026
:10623000FF3267F30F059A6167F31F450B22DD619B
:106240005A611A611A6820466FF30A121A60FFF742
:1062500034FCE3684FF480525A612D4B20461B6892
:106260001B6998473846B3041DD52046FFF78AFAC4
:10627000E3682046DD68FFF775FA032806D100239E
:10628000A3704FF40073A380092304E00123A370DB
:106290004023A380052363F38D25E3684FF4005268
:1062A000DD6001205A61F70209D5194B20461B68B1
:1062B000DB699847E3684FF480125A610120B50208
:1062C00009D5134B20461B681B6A9847E3684FF4B7
:1062D00000125A610120710009D50D4B20461B6840
:1062E0005B6A9847E3684FF080425A610120720769
:1062F0000BD5E3685D686B0704D5054B20461B682A
:106300009B6A9847E36801205D6005B0BDE8F08FA7
:10631000E000002081F0004102E000BF83F0004374
:1063200030B54FEA41044FEA430594EA050F08BF30
:1063300090EA020F1FBF54EA000C55EA020C7FEAF4
:10634000645C7FEA655C00F0E2804FEA5454D4EB71
:106350005555B8BF6D420CDD2C4480EA020281EA3B
:10636000030382EA000083EA010180EA020281EA73
:106370000303362D88BF30BD11F0004F4FEA0131C5
:106380004FF4801C4CEA113102D0404261EB4101D4
:1063900013F0004F4FEA03334CEA133302D052425A
:1063A00063EB430394EA050F00F0A780A4F1010416
:1063B000D5F1200E0DDB02FA0EFC22FA05F2801850
:1063C00041F1000103FA0EF2801843FA05F3594136
:1063D0000EE0A5F120050EF1200E012A03FA0EFCB5
:1063E00028BF4CF0020C43FA05F3C01851EBE371DF
:1063F00001F0004507D54FF0000EDCF1000C7EEBFC
:1064000000006EEB0101B1F5801F1BD3B1F5001F39
:106410000CD349085FEA30004FEA3C0C04F1010458
:106420004FEA445212F5800F80F09A80BCF1004F81
:1064300008BF5FEA500C50F1000041EB045141EA03
:10644000050130BD5FEA4C0C404141EB010111F404
:10645000801FA4F10104E9D191F0000F04BF0146AF
:106460000020B1FA81F308BF2033A3F10B03B3F18D
:1064700020020CDA0C3208DD02F1140CC2F10C021D
:1064800001FA0CF021FA02F10CE002F11402D8BF7B
:10649000C2F1200C01FA02F120FA0CFCDCBF41EA47
:1064A0000C019040E41AA2BF01EB0451294330BD16
:1064B0006FEA04041F3C1CDA0C340EDC04F11404F3
:1064C000C4F1200220FA04F001FA02F340EA0300CA
:1064D00021FA04F345EA030130BDC4F10C04C4F110
:1064E000200220FA02F001FA04F340EA03002946F0
:1064F00030BD21FA04F0294630BD94F0000F83F43A
:10650000801306BF81F480110134013D4EE77FEA1C
:10651000645C18BF7FEA655C29D094EA050F08BF68
:1065200090EA020F05D054EA000C04BF1946104649
:1065300030BD91EA030F1EBF0021002030BD5FEA8D
:10654000545C05D14000494128BF41F0004130BDB5
:1065500014F580043CBF01F5801130BD01F0004509
:1065600045F0FE4141F470014FF0000030BD7FEA7C
:10657000645C1ABF194610467FEA655C1CBF0B4677
:10658000024650EA013406BF52EA033591EA030F8E
:1065900041F4002130BD00BF90F0000F04BF002186
:1065A000704730B54FF4806404F132044FF00005B9
:1065B0004FF0000150E700BF90F0000F04BF002132
:1065C000704730B54FF4806404F1320410F0004598
:1065D00048BF40424FF000013EE700BF42004FEA93
:1065E000E2014FEA31014FEA02701FBF12F07F4310
:1065F00093F07F4F81F06051704792F0000F14BF0D
:1066000093F07F4F704730B54FF4607401F0004550
:1066100021F0004120E700BF50EA010208BF7047A7
:1066200030B54FF000050AE050EA010208BF70479C
:1066300030B511F0004502D5404261EB41014FF405
:10664000806404F132045FEA915C3FF4DCAE4FF009
:1066500003025FEADC0C18BF03325FEADC0C18BFF0
:10666000033202EBDC02C2F1200300FA03FC20FA41
:1066700002F001FA03FE40EA0E0021FA02F114448E
:10668000C1E600BF70B54FF0FF0C4CF4E06C1CEAA3
:1066900011541DBF1CEA135594EA0C0F95EA0C0F18
:1066A00000F0DEF82C4481EA030621EA4C5123EA8B
:1066B0004C5350EA013518BF52EA033541F48011BA
:1066C00043F4801338D0A0FB02CE4FF00005E1FB6D
:1066D00002E506F00042E0FB03E54FF00006E1FBB7
:1066E00003569CF0000F18BF4EF0010EA4F1FF04FA
:1066F000B6F5007F64F5407404D25FEA4E0E6D413A
:1067000046EB060642EAC62141EA55514FEAC5204A
:1067100040EA5E504FEACE2EB4F1FD0C88BFBCF5C6
:10672000E06F1ED8BEF1004F08BF5FEA500E50F177
:10673000000041EB045170BD06F0004646EA01013D
:1067400040EA020081EA0301B4EB5C04C2BFD4EB6F
:106750000C0541EA045170BD41F480114FF0000E68
:10676000013C00F3AB8014F1360FDEBF002001F0D6
:10677000004170BDC4F10004203C35DA0C341BDC50
:1067800004F11404C4F1200500FA05F320FA04F022
:1067900001FA05F240EA020001F0004221F0004156
:1067A00010EBD37021FA04F642EB06015EEA430EC9
:1067B00008BF20EAD37070BDC4F10C04C4F12005F9
:1067C00000FA04F320FA05F001FA04F240EA0200AC
:1067D00001F0004110EBD37041F100015EEA430E7D
:1067E00008BF20EAD37070BDC4F1200500FA05F29D
:1067F0004EEA020E20FA04F301FA05F243EA02031C
:1068000021FA04F001F0004121FA04F220EA02002A
:1068100000EBD3705EEA430E08BF20EAD37070BD70
:1068200094F0000F0FD101F00046400041EB010150
:1068300011F4801F08BF013CF7D041EA060195F032
:10684000000F18BF704703F00046520043EB0303EC
:1068500013F4801F08BF013DF7D043EA06037047D9
:1068600094EA0C0F0CEA135518BF95EA0C0F0CD0E4
:1068700050EA410618BF52EA4306D1D181EA03012A
:1068800001F000414FF0000070BD50EA410606BF24
:106890001046194652EA430619D094EA0C0F02D169
:1068A00050EA013613D195EA0C0F05D152EA0336AE
:1068B0001CBF104619460AD181EA030101F00041CC
:1068C00041F0FE4141F470014FF0000070BD41F015
:1068D000FE4141F4780170BD70B54FF0FF0C4CF4EF
:1068E000E06C1CEA11541DBF1CEA135594EA0C0F0E
:1068F00095EA0C0F00F0A7F8A4EB050481EA030E5B
:1069000052EA03354FEA013100F088804FEA033341
:106910004FF0805545EA131343EA12634FEA02220F
:1069200045EA111545EA10654FEA00260EF00041D0
:106930009D4208BF964244F1FD0404F5407402D222
:106940005B084FEA3202B61A65EB03055B084FEAB3
:1069500032024FF480104FF4002CB6EB020E75EBB0
:10696000030E22BFB61A754640EA0C005B084FEAD8
:106970003202B6EB020E75EB030E22BFB61A754655
:1069800040EA5C005B084FEA3202B6EB020E75EBA0
:10699000030E22BFB61A754640EA9C005B084FEA18
:1069A0003202B6EB020E75EB030E22BFB61A754625
:1069B00040EADC0055EA060E18D04FEA051545EA14
:1069C00016754FEA06164FEAC30343EA52734FEABD
:1069D000C2025FEA1C1CC0D111F4801F0BD141EA36
:1069E00000014FF000004FF0004CB6E711F4801F9B
:1069F00004BF01430020B4F1FD0C88BFBCF5E06F7B
:106A00003FF6AFAEB5EB030C04BFB6EB020C5FEA8A
:106A1000500C50F1000041EB045170BD0EF0004EDF
:106A20004EEA113114EB5C04C2BFD4EB0C0541EA11
:106A3000045170BD41F480114FF0000E013C90E60E
:106A400045EA060E8DE60CEA135594EA0C0F08BFD2
:106A500095EA0C0F3FF43BAF94EA0C0F0AD150EAD1
:106A600001347FF434AF95EA0C0F7FF425AF104664
:106A700019462CE795EA0C0F06D152EA03353FF48C
:106A8000FDAE1046194622E750EA410618BF52EA09
:106A900043067FF4C5AE50EA41047FF40DAF52EADD
:106AA00043057FF4EBAE12E74FF0FF3C06E000BF7A
:106AB0004FF0010C02E000BF4FF0010C4DF804CD87
:106AC0004FEA410C7FEA6C5C4FEA430C18BF7FEA47
:106AD0006C5C1BD001B050EA410C0CBF52EA430C75
:106AE00091EA030F02BF90EA020F0020704710F1F5
:106AF000000F91EA030F58BF994208BF90422CBF84
:106B0000D8176FEAE37040F0010070474FEA410C7C
:106B10007FEA6C5C02D150EA013C07D14FEA430C9A
:106B20007FEA6C5CD6D152EA033CD3D05DF8040B0B
:106B3000704700BF8446104662468C46194663463D
:106B400000E000BF01B5FFF7B7FF002848BF10F114
:106B5000000F01BD4DF808EDFFF7F4FF0CBF012059
:106B600000205DF808FB00BF4DF808EDFFF7EAFFD5
:106B700034BF012000205DF808FB00BF4DF808ED90
:106B8000FFF7E0FF94BF012000205DF808FB00BF85
:106B90004DF808EDFFF7CEFF94BF012000205DF80F
:106BA00008FB00BF4DF808EDFFF7C4FF34BF01201C
:106BB00000205DF808FB00BF4FEA410212F5001209
:106BC00015D211D56FF47873B3EB625212D94FEA34
:106BD000C12343F0004343EA505311F0004F23FA1E
:106BE00002F018BF404270474FF00000704750EA73
:106BF000013005D111F0004008BF6FF00040704730
:106C00004FF00000704700BF4FEA4102B2F1E0438D
:106C100024BFB3F5001CDCF1FE5C0DD901F0004C83
:106C20004FEAC0024CEA5070B2F1004F40EB8300D3
:106C300008BF20F00100704711F0804F21D113F1FF
:106C40003872BCBF01F00040704741F480114FEA38
:106C50005252C2F11802C2F1200C10FA0CF320FAC1
:106C600002F018BF40F001004FEAC1234FEAD323DE
:106C700003FA0CFC40EA0C0023FA02F34FEA430348
:106C8000CCE77FEA625307D150EA01331EBF4FF0D1
:106C9000FE4040F44000704701F0004040F0FE40EC
:106CA00040F40000704700BF80F0004002E000BFE9
:106CB00081F0004142001FBF5FEA410392EA030FE7
:106CC0007FEA226C7FEA236C6AD04FEA1262D2EB31
:106CD0001363C1BFD218414048404140B8BF5B4236
:106CE000192B88BF704710F0004F40F4000020F0CF
:106CF0007F4018BF404211F0004F41F4000121F0E5
:106D00007F4118BF494292EA030F3FD0A2F101022E
:106D100041FA03FC10EB0C00C3F1200301FA03F16C
:106D200000F0004302D5494260EB4000B0F5000F8F
:106D300013D3B0F1807F06D340084FEA310102F14E
:106D40000102FE2A51D2B1F1004F40EBC25008BF00
:106D500020F0010040EA03007047490040EB0000CA
:106D600010F4000FA2F10102EDD1B0FA80FCACF1F9
:106D7000080CB2EB0C0200FA0CF0AABF00EBC250F8
:106D800052421843BCBFD0401843704792F0000FE6
:106D900081F4000106BF80F400000132013BB5E739
:106DA0004FEA41037FEA226C18BF7FEA236C21D0AF
:106DB00092EA030F04D092F0000F08BF0846704714
:106DC00090EA010F1CBF0020704712F07F4F04D1E2
:106DD000400028BF40F00040704712F100723CBFF5
:106DE00000F50000704700F0004343F0FE4040F41F
:106DF000000070477FEA226216BF08467FEA2363DD
:106E00000146420206BF5FEA412390EA010F40F4C7
:106E1000800070474FF0000304E000BF10F0004313
:106E200048BF40425FEA000C08BF704743F09643FA
:106E300001464FF000001CE050EA010208BF704715
:106E40004FF000030AE000BF50EA010208BF70479C
:106E500011F0004302D5404261EB41015FEA010CB1
:106E600002BF84460146002043F0B64308BFA3F1A9
:106E70008053A3F50003BCFA8CF2083AA3EBC2538B
:106E800010DB01FA02FC634400FA02FCC2F12002AA
:106E9000BCF1004F20FA02F243EB020008BF20F0E1
:106EA0000100704702F1200201FA02FCC2F1200247
:106EB00050EA4C0021FA02F243EB020008BF20EA3C
:106EC000DC7070474FF0FF0C1CEAD0521EBF1CEA6A
:106ED000D15392EA0C0F93EA0C0F6FD01A4480EA58
:106EE000010C400218BF5FEA41211ED04FF0006341
:106EF00043EA501043EA5111A0FB01310CF000406D
:106F0000B1F5000F3EBF490041EAD3715B0040EA92
:106F1000010062F17F02FD2A1DD8B3F1004F40EB62
:106F2000C25008BF20F00100704790F0000F0CF035
:106F3000004C08BF49024CEA502040EA51207F3AF9
:106F4000C2BFD2F1FF0340EAC250704740F40000D4
:106F50004FF00003013A5DDC12F1190FDCBF00F0C5
:106F600000407047C2F10002410021FA02F1C2F173
:106F7000200200FA02FC5FEA310040F1000053EA0F
:106F80004C0308BF20EADC70704792F0000F00F05D
:106F9000004C02BF400010F4000F013AF9D040EA63
:106FA0000C0093F0000F01F0004C02BF490011F4F7
:106FB000000F013BF9D041EA0C018FE70CEAD153F5
:106FC00092EA0C0F18BF93EA0C0F0AD030F0004C75
:106FD00018BF31F0004CD8D180EA010000F0004029
:106FE000704790F0000F17BF90F0004F084691F0E7
:106FF000000F91F0004F14D092EA0C0F01D1420221
:107000000FD193EA0C0F03D14B0218BF084608D1E9
:1070100080EA010000F0004040F0FE4040F4000033
:10702000704740F0FE4040F4400070474FF0FF0CC6
:107030001CEAD0521EBF1CEAD15392EA0C0F93EA0D
:107040000C0F69D0A2EB030280EA010C49024FEA5F
:10705000402037D04FF0805343EA111143EA101318
:107060000CF000408B4238BF5B0042F17D024FF4D0
:10707000000C8B4224BF5B1A40EA0C00B3EB510FAB
:1070800024BFA3EB510340EA5C00B3EB910F24BF94
:10709000A3EB910340EA9C00B3EBD10F24BFA3EB19
:1070A000D10340EADC001B0118BF5FEA1C1CE0D1E1
:1070B000FD2A3FF650AF8B4240EBC25008BF20F094
:1070C000010070470CF0004C4CEA50207F32C2BFE8
:1070D000D2F1FF0340EAC250704740F400004FF085
:1070E0000003013A37E792F0000F00F0004C02BFB6
:1070F000400010F4000F013AF9D040EA0C0093F080
:10710000000F01F0004C02BF490011F4000F013BD9
:10711000F9D041EA0C0195E70CEAD15392EA0C0F41
:1071200008D142027FF47DAF93EA0C0F7FF470AF79
:10713000084676E793EA0C0F04D14B023FF44CAFBC
:1071400008466EE730F0004C18BF31F0004CCAD151
:1071500030F000427FF45CAF31F000437FF43CAF8D
:107160005FE700BF4FEA4002B2F1FE4F0FD34FF08E
:107170009E03B3EB12620DD94FEA002343F00043A4
:1071800010F0004F23FA02F018BF404270474FF052
:107190000000704712F1610F01D1420205D110F0D9
:1071A000004008BF6FF0004070474FF0000070478C
:1071B00042000ED2B2F1FE4F0BD34FF09E03B3EB61
:1071C000126209D44FEA002343F0004323FA02F08D
:1071D00070474FF00000704712F1610F01D1420279
:1071E00002D14FF0FF3070474FF00000704700BFF2
:1071F00073B96AB9002908BF0028BCBF00204FF04E
:107200000041C4BF6FF000414FF0FF3000F03CB8C8
:1072100082B0EC462DE9005000F006F8DDF804E0FD
:1072200002B00CBC704700BF2DE9704F089E144699
:107230001D468046894600F029F804FB01F3A4FBB3
:1072400000AB00FB05329344B8EB0A0869EB0B096D
:10725000C6E90089BDE8708F2DE9704F089E14467D
:107260001D468046894600F061F900FB05F5A0FB4C
:1072700004AB04FB0154A344B8EB0A0869EB0B0907
:10728000C6E90089BDE8708F704700BF00292DE96D
:10729000F00FC0F2A1800024002BC0F298801546A8
:1072A00006460F46002B3FD18A4258D9B2FA82F3E4
:1072B0004BB1C3F1200201FA03F720FA02F29D401C
:1072C00000FA03F61743290CB7FBF1F201FB127722
:1072D000A8B200FB02F34FEA164C4CEA0747BB4248
:1072E00009D97F1902F1FF3C80F00581BB4240F2D1
:1072F0000281023A2F44FF1AB7FBF1F301FB13712D
:1073000000FB03F0B6B246EA0141884208D94919A8
:1073100003F1FF3780F0F180884240F2EE80023BBB
:1073200043EA0242002303E08B420AD900231A46B3
:107330001046194614B1404261EB4101BDE8F00F1F
:107340007047B3FA83F8B8F1000F40F088808B42A1
:1073500002D3824200F2E28000230122E8E712B960
:107360000123B3FBF2F5B5FA85F2002A3AD17F1B6F
:10737000280C1FFA85FC0123B7FBF0F100FB117705
:107380000CFB01F24FEA164848EA0747BA4207D910
:107390007F1901F1FF3802D2BA4200F2C48041469F
:1073A000BF1AB7FBF0F200FB12700CFB02FCB6B286
:1073B00046EA0040844507D9401902F1FF3702D25E
:1073C000844500F2AE803A4642EA0142B0E7E44327
:1073D000524263EB430362E7404261EB41014FF0ED
:1073E000FF3459E79540C2F1200927FA09F126FA3E
:1073F00009F99740280CB1FBF0F800FB18111FFAAF
:1074000085FC0CFB08F349EA07094FEA194747EAEC
:1074100001418B4206FA02F608D9491908F1FF32F8
:107420007AD28B4278D9A8F102082944C91AB1FB53
:10743000F0F300FB13170CFB03F21FFA89F949EA7A
:107440000747BA4207D97F1903F1FF3160D2BA4228
:107450005ED9023B2F44BF1A43EA08438CE7C8F1C8
:10746000200225FA02F103FA08FC27FA02F320FAB7
:1074700002F207FA08F741EA0C0C4FEA1C49B3FB89
:10748000F9F109FB11331FFA8CFA0AFB01FB1743D0
:107490003A0C42EA03439B4505FA08F008D913EB7E
:1074A0000C0301F1FF3235D29B4533D902396344D5
:1074B000CBEB0303B3FBF9F209FB12330AFB02FA2D
:1074C000BFB247EA0347BA4508D917EB0C0702F1E8
:1074D000FF331BD2BA4519D9023A674442EA014543
:1074E000A5FB0001CAEB07078F424FF000030AD348
:1074F00005D02A461CE76246FDE63B4610E706FA41
:1075000008F68642F5D26A1E002311E71A46E5E71F
:107510000B46A0E71146CBE7904687E74346424635
:1075200006E7023A50E702392F4439E72DE9F00F18
:10753000144605460E46002B43D18A4253D9B2FA6F
:1075400082F757B1C7F1200620FA06F601FA07F3D1
:1075500002FA07F400FA07F51E43210CB6FBF1F21C
:1075600001FB1266A0B200FB02F32F0C47EA0646AD
:10757000B34209D9361902F1FF3780F0FD80B342DA
:1075800040F2FA80023A2644F61AB6FBF1F301FB08
:10759000136100FB03F0ADB245EA0141884208D90E
:1075A000091903F1FF3680F0E980884240F2E68055
:1075B000023B43EA0242002310461946BDE8F00FA1
:1075C00070478B424CD8B3FA83F6002E4FD18B42D2
:1075D00002D3824200F2DD80BDE8F00F00230122D9
:1075E00010461946704712B90124B4FBF2F4B4FAFC
:1075F00084F2002A40F08280091B260CA7B20123E6
:10760000B1FBF6F006FB101107FB00F24FEA154C38
:107610004CEA01418A4207D9091900F1FF3C02D224
:107620008A4200F2C8806046891AB1FBF6F206FB76
:10763000121107FB02F7ADB245EA0145AF4208D986
:107640002C1902F1FF3180F09B80A74240F2988014
:10765000023A42EA004210461946BDE8F00F704770
:1076600000231A4610461946BDE8F00F7047C6F1D0
:10767000200522FA05F703FA06F421FA05F301FAC8
:1076800006FB20FA05F53C434FEA1448B3FBF8FC2F
:1076900008FB1C331FFA84F909FB0CFA45EA0B0BB3
:1076A0004FEA1B4545EA03439A4502FA06F204D91C
:1076B0001B190CF1FF356FD3AC46CAEB0303B3FBC8
:1076C000F8F508FB153309FB05F91FFA8BFB4BEAAC
:1076D0000347B94504D93F1905F1FF3362D31D466D
:1076E00045EA0C4CACFB0223C9EB07079F424FF065
:1076F00000054AD346D062462B465DE79440C2F16E
:10770000200921FA09FC914020FA09F9260CBCFB5A
:10771000F6F806FB18CCA7B207FB08F349EA010903
:107720004FEA194141EA0C4C634500FA02F509D9C8
:107730001CEB040C08F1FF323BD2634539D9A8F1A8
:107740000208A444C3EB0C0CBCFBF6F306FB13C10C
:1077500007FB03F21FFA89F949EA01418A4207D976
:10776000091903F1FF3022D28A4220D9023B214479
:10777000891A43EA084343E73A4605E7334618E7E0
:107780000A4666E7B0409042B5D20CF1FF320023C2
:1077900012E7334632460FE79A458DD9ACF1020C19
:1077A00023448AE7B9459AD9023D274498E703461E
:1077B000DEE79046C6E70238214435E7002100F0B5
:1077C00004B80C4B5B58435004310B480B4B421828
:1077D0009A42FFF4F6AF0A4A00F003B8002342F8D9
:1077E000043B084B9A42FFF4F9AFFAF73FFC00F074
:1077F0000DF870477C98010800000020BC050020AF
:10780000C0050020B43E0120FFF7FEBF08B562B6F8
:107810001D4C01214FF48040FBF772FEF0F72CFD68
:10782000F1F77EFFF0F70EFDF2F762F8F2F788FB52
:107830002078F1F723FB22696079A168F1F7AEFDAA
:10784000F3F7A4FAF2F7DEFDF1F732F8FAF77CFA73
:10785000F6F744F8F6F748FDF6F7C8FF0B4B04229D
:107860005A83F6F72BF9F6F740FDF6F7DDFFF0F750
:10787000D9FEF0F7F9FE0028F3D0F2F7C3FDF6F7D2
:107880002DF8F6F7B3FFECE70400002000100240EB
:1078900000210A2200F0ACB80F4B30B405461C683A
:1078A00002E0D01A16D1ABB115F8013BE2185078BE
:1078B0001A4600F00300012808BF03F1200211F866
:1078C000013BE018407800F003000128E9D12033A3
:1078D000D01AE9D030BC7047B40500202DE9F00F74
:1078E000424C82B0D4F800C001900E4600E026461B
:1078F000344614F8015B0CEB0500407800F00800FA
:1079000000F0FF0A0028F2D12D2D5BD02B2D04BFF3
:107910007578B41C33F010003CD09946BAF1000FD2
:107920000CBF6FF0004B4FF0004BBBFBF9F800278A
:1079300009FB18BB38460CE0303DAB4219DD7E1C1C
:1079400005D0404523D820D009FB0050012714F86A
:10795000015B0CEB0506767816F0040FECD116F0FF
:10796000030606D0012E14BF57263726AD1BAB42A7
:10797000E5DC7B1C15D0BAF1000F21D10AB1EFB9BB
:10798000116002B0BDE8F00F70475D45DCDD4FF0DF
:10799000FF37DCE7302D1AD0002BBED10A239946E1
:1079A000BCE70199BAF1000F4FF022030CBF6FF052
:1079B00000404FF000400B60002AE2D0611EDFE77C
:1079C0004042DBE7B41C75784FF0010AA2E720784B
:1079D00000F0DF00582803D0002B9ED108239CE73D
:1079E000102365789946023498E700BFB40500205B
:1079F00030B4044C0D46134601462A46206830BC7C
:107A0000FFF76CBFB0050020024B13B1024800F035
:107A100005B8704700000000297A010801460020DF
:107A20000246034600F018B838B5094D094C641BEE
:107A3000A41018BF05EB840505D0013C55F8043DA2
:107A40009847002CF9D1BDE8384001F007BF00BFCE
:107A5000789801087C980108F0B5274C85B0266815
:107A60000746D6F84841002C40D065681F2D1EDD22
:107A7000224818B94FF0FF3005B0F0BD4FF4C87080
:107A8000039102920193AFF3008003990446029A96
:107A9000019B0028EED0D6F8485100202560606098
:107AA0000546C6F84841C4F88801C4F88C013FB9BE
:107AB0006B1C00200235636044F8251005B0F0BD52
:107AC0000126AE4004EB8500C0F88820D4F8882158
:107AD000022F42EA0602C4F88821C0F80831E7D133
:107AE000D4F88C311E43C4F88C61E1E706F5A67426
:107AF000C6F84841B9E700BF409701080000000000
:107B00002DE9F0418AB004460D4600F06DF8DFF82B
:107B1000D080064698F900300F4601330BD020463E
:107B2000294600F059FA30B12046294600220023A8
:107B3000FFF738F820B1304639460AB0BDE8F08189
:107B4000234B98F800600890CDE90245CDE9044543
:107B5000019346BB1F4B4FF06042CDE90623204600
:107B6000294600220023FEF7F5FF70B102239E4252
:107B7000009322D0684600F057FAF0B1089B0BBB87
:107B8000DDE906010AB0BDE8F0810123022E009371
:107B90000ED0684600F048FA50B10F4800F046FA9F
:107BA000CDE90601EAE70D4B0022CDE90623D6E731
:107BB00000F042FA21230360EFE700F03DFA2223B0
:107BC0000360DBE700F038FA089B0360D8E700BFEA
:107BD00048980108FFFFEFC74C9801080000F0FF2C
:107BE000B8050020000000002DE9F04FB1F5801F1E
:107BF00087B002460B460F465BDA21F0004606438B
:107C000000F0F5800029C0F2A4810022B24BFEF7FB
:107C100039FD0F460B46B14902468F426FF03505DC
:107C20004BDCC7F3130606F5152101F6647101F468
:107C3000801484F07F5181F4401141EA060310461C
:107C400019460022A64BFEF769FB4FEA2758B31CE2
:107C5000A8F2FF38C3F31303A844022B08EB14580F
:107C600082468B464FF000022EDC0023FEF772FFA7
:107C7000002800F0C580B8F1000F00F07181404687
:107C8000FEF79AFC80A3D3E9002306460F46FEF7D1
:107C9000F9FC7FA3D3E9002304460D46304639465C
:107CA000FEF7F0FC02460B4620462946FEF738FB5D
:107CB00007E08A4900258F42B3DD10461946FEF7DA
:107CC0002FFB07B0BDE8F08F4FF08043FEF728FB95
:107CD00002460B4650465946FEF7FEFDCDE902012D
:107CE0004046FEF769FCCDE90401DDE902010246E8
:107CF0000B46FEF7C7FC02460B46CDE90001FEF736
:107D0000C1FC65A3D3E9002304460D46FEF7BAFC87
:107D100063A3D3E90023FEF703FB22462B46FEF7BD
:107D2000B1FC61A3D3E90023FEF7FAFA22462B4601
:107D3000FEF7A8FC5EA3D3E90023FEF7F1FADDE924
:107D40000023FEF79FFC5CA3D3E90023CDE90001EB
:107D500020462946FEF796FC59A3D3E90023FEF7F7
:107D6000DFFA22462B46FEF78DFC57A3D3E900230A
:107D7000FEF7D6FA22462B46FEF784FC0B46024657
:107D8000DDE90001FEF7CCFAA6F5C223C6F5D72639
:107D9000A3F27A4351361E43002E04460D4657DDAA
:107DA0000022504B50465946FEF76CFC52465B464B
:107DB000FEF768FC06460F46B8F1000F40F09680CB
:107DC00022462B46FEF7ACFADDE90223FEF75AFC09
:107DD00002460B4630463946FEF7A0FA02460B46ED
:107DE00050465946FEF79AFA07B0BDE8F08F0022D8
:107DF000002300203C49FEF76FFD07B0BDE8F08F7F
:107E000052465B4650465946FEF73CFC30A3D3E948
:107E1000002304460D4650465946FEF733FC024601
:107E20000B4600202F49FEF779FA02460B46204602
:107E30002946FEF727FC04460D46B8F1000F40F036
:107E400092805046594622462B46FEF767FA38E79D
:107E5000B8F1000F00F0AB800BA3D3E90023DDE9FC
:107E60000401FEF70FFC22462B4606460F465046FD
:107E70005946FEF753FADDE90223FEF703FC0446F8
:107E80000D46DDE904017CE00000E0FE422EE63F05
:107E9000763C7935EF39EA3D44523EDF12F1C23F7C
:107EA000DE03CB966446C73F599322942449D23FC0
:107EB000935555555555E53F9FC678D0099AC33F10
:107EC000AF788E1DC571CC3F04FA97999999D93F27
:107ED000555555555555D53F00005043FFFFEF7F91
:107EE0000000F03F0000E03F000050C336A3D3E99C
:107EF0000023DDE90401FEF7C5FB224680468946E2
:107F00002B4630463946FEF70BFADDE90223FEF731
:107F1000B9FB2FA3D3E9002304460D46DDE9040194
:107F2000FEF7B0FB02460B4620462946FEF7F8F95D
:107F300002460B4630463946FEF7F0F952465B469C
:107F4000FEF7ECF902460B4640464946FEF7E6F9D5
:107F5000B7E6FEF7E3F900220023FEF7BDFCB0E62A
:107F600000200021ADE64046FEF726FB16A3D3E92C
:107F7000002380468946FEF785FB06460F464046AD
:107F8000494613A3D3E90023FEF77CFB02460B46C8
:107F900020462946FEF7C2F952465B46FEF7BEF977
:107FA00002460B4630463946FEF7B8F989E60246E6
:107FB0000B4650465946FEF7B1F9DDE90223FEF7BC
:107FC00061FB0BE7AFF300800000E0FE422EE63FCE
:107FD000763C7935EF39EA3D31F0004310B408D0F2
:107FE0000F4AA3F5801494420AD804205DF8044B8C
:107FF000704700280CBF022003205DF8044B704737
:10800000B3F5801F01D20320F7E7064A934201D05F
:108010000020F2E7D0F1010038BF0020EDE700BFFB
:10802000FFFFDF7F0000F07F002070470020014944
:10803000704700BF0000F87F014B1868704700BF11
:10804000B005002050C3000088130000018008081C
:10805000000000000000010000000000000000001F
:10806000C8000000EF8D2100B81E050000000000D0
:10807000000000009033000000000000000000003D
:1080800000000000000000000000000000000000F0
:1080900000000000000000000000000000000000E0
:1080A00000000000000000000000000000000000D0
:1080B00000000000000000000000000000000000C0
:1080C00000000000000000000000000000000000B0
:1080D00000000000000000000000000000000000A0
:1080E0000000000000000000000000000000000090
:1080F0000000000000000000000000000000000080
:10810000000000000000000000000000000000006F
:108110000000000000000000524F52000001065213
:108120004F4C000002064D5354000003024D5650C0
:10813000000004075341500000050747415000006C
:1081400006035354415000070352534150000803A3
:108150005347500000090747475000000A03535493
:108160004750000B0352534750000C035246530034
:10817000000D0353494F00000E0747494F00000F01
:108180000353414300001D0753434F00001E0747A0
:10819000434F00001F0343434F0000200341434F60
:1081A00000002703554630000040075546310000C7
:1081B0004107554632000042075546330000430749
:1081C00055463400004407554635000045075546DE
:1081D00036000046075546370000470752554E0007
:1081E00000810553544F5000800042494E00008BDF
:1081F000000000000000000000000000100000006F
:10820000160000001B0000002000000023000000FA
:10821000270000002A0000002D00000030000000B0
:108220003200000035000000370000003900000077
:108230003B0000003D000000400000004100000045
:108240004300000045000000470000004900000016
:108250004B0000004C0000004E00000050000000E9
:1082600051000000530000005400000056000000C0
:1082700057000000590000005A0000005B00000099
:108280005D0000005E000000600000006100000072
:10829000620000006300000065000000660000004E
:1082A00067000000680000006A0000006B0000002A
:1082B0006C0000006D0000006E0000007000000007
:1082C00071000000720000007300000074000000E4
:1082D00075000000760000007700000078000000C4
:1082E000790000007A0000007B0000007C000000A4
:1082F0007D0000007E000000800000008000000083
:108300008100000082000000830000008400000063
:108310008500000086000000870000008800000043
:10832000890000008A0000008B0000008C00000023
:108330008D0000008E0000008F0000009000000003
:1083400090000000910000009200000093000000E7
:1083500094000000950000009600000096000000C8
:108360009700000098000000990000009A000000AB
:108370009B0000009B0000009C0000009D0000008E
:108380009E0000009F000000A0000000A000000070
:10839000A1000000A2000000A3000000A300000054
:1083A000A4000000A5000000A6000000A700000037
:1083B000A7000000A8000000A9000000AA0000001B
:1083C000AA000000AB000000AC000000AD000000FF
:1083D000AD000000AE000000AF000000B0000000E3
:1083E000B0000000B1000000B2000000B2000000C8
:1083F000B3000000B4000000B5000000B5000000AC
:10840000B6000000B7000000B7000000B800000090
:10841000B9000000B9000000BA000000BB00000075
:10842000BB000000BC000000BD000000BD0000005B
:10843000BE000000BF000000C0000000C00000003F
:10844000C1000000C1000000C2000000C300000025
:10845000C3000000C4000000C5000000C50000000B
:10846000C6000000C7000000C7000000C8000000F0
:10847000C9000000C9000000CA000000CB000000D5
:10848000CB000000CC000000CC000000CD000000BC
:10849000CE000000CE000000CF000000D0000000A1
:1084A000D0000000D1000000D1000000D200000088
:1084B000D3000000D3000000D4000000D40000006E
:1084C000D5000000D6000000D6000000D700000054
:1084D000D7000000D8000000D9000000D90000003B
:1084E000DA000000DA000000DB000000DB00000022
:1084F000DC000000DD000000DD000000DE00000008
:10850000DE000000DF000000E0000000E0000000EE
:10851000E1000000E1000000E2000000E2000000D5
:10852000E3000000E3000000E4000000E5000000BC
:10853000E5000000E6000000E6000000E7000000A3
:10854000E7000000E8000000E8000000E90000008B
:10855000EA000000EA000000EB000000EB00000071
:10856000EC000000EC000000ED000000ED00000059
:10857000EE000000EE000000EF000000F000000040
:10858000F0000000F1000000F1000000F200000027
:10859000F2000000F3000000F3000000F40000000F
:1085A000F4000000F5000000F5000000F6000000F7
:1085B000F6000000F7000000F7000000F8000000DF
:1085C000F8000000F9000000F9000000FA000000C7
:1085D000FA000000FB000000FB000000FC000000AF
:1085E000FC000000FD000000FD000000FE00000097
:1085F000FE000000FF00000001F0010002F0010099
:1086000004F0010005F0010007F0010008F001008E
:108610000AF001000BF001000DF001000EF0010066
:1086200010EE010011EE010013EE010015EE010045
:1086300016EE010018EE010019EE01001BEE01001C
:108640001CEC01001EEC01001FEC010021EC0100FC
:1086500022EC010024EA010025EA010027EA0100DA
:1086600028EA01002AE801002BE801002DE80100BA
:108670002EE8010030E6010031E6010033E601009A
:1086800034E4010036E4010037E4010039E201007E
:108690003AE201003CE201003DE001003EE0010061
:1086A00040E0010041DE010043DE010044DC010046
:1086B00046DC010047DC010049DA01004ADA01002A
:1086C0004CD801004DD801004FD6010050D6010012
:1086D00051D4010053D4010054D2010056D20100FC
:1086E00057D0010059D001005ACE01005BCE0100E5
:1086F0005DCC01005ECA010060CA010061C80100D2
:1087000062C8010064C6010065C4010067C40100BD
:1087100068C2010069C201006BC001006CBE0100AB
:108720006DBE01006FBC010070BA010072B801009B
:1087300073B8010074B6010076B4010077B401008B
:1087400078B201007AB001007BAE01007CAE01007E
:108750007EAC01007FAA010080A8010081A8010071
:1087600083A6010084A4010085A2010087A0010066
:10877000889E0100899E01008A9C01008C9A01005C
:108780008D9801008E9601008F9401009192010056
:108790009292010093900100948E0100968C01004A
:1087A000978A010098880100998601009A84010047
:1087B0009C8201009D8001009E7E01009F7C010043
:1087C000A07A0100A1780100A3760100A474010041
:1087D000A5720100A6700100A76E0100A86C01003F
:1087E000A96A0100AA680100AC660100AD6401003D
:1087F000AE620100AF600100B05E0100B15C01003B
:10880000B25A0100B3580100B4540100B55201003E
:10881000B6500100B74E0100B84C0100B94A010042
:10882000BA480100BB460100BC420100BD40010046
:10883000BE3E0100BF3C0100C03A0100C13801004A
:10884000C2340100C3320100C4300100C52E010052
:10885000C62C0100C7280100C8260100C924010058
:10886000C9220100CA1E0100CB1C0100CC1A010064
:10887000CD180100CE140100CF120100CF1001006D
:10888000D00E0100D10A0100D2080100D306010078
:10889000D4020100D4000100D5FE0000D6FC000087
:1088A000D7F80000D7F60000D8F40000D9F0000097
:1088B000DAEE0000DAEC0000DBE80000DCE60000A5
:1088C000DCE40000DDE00000DEDE0000DFDA0000B6
:1088D000DFD80000E0D60000E1D20000E1D00000C7
:1088E000E2CE0000E2CA0000E3C80000E4C40000D9
:1088F000E4C20000E5C00000E5BC0000E6BA0000EC
:10890000E7B60000E7B40000E8B20000E8AE0000FF
:10891000E9AC0000E9A80000EAA60000EAA2000015
:10892000EBA00000EB9E0000EC9A0000EC98000029
:10893000ED940000ED920000EE8E0000EE8C000041
:10894000EE880000EF860000EF820000F08000005B
:10895000F07C0000F07A0000F1780000F174000073
:10896000F1720000F26E0000F26C0000F26800008C
:10897000F3660000F3620000F3600000F45C0000A6
:10898000F45A0000F4560000F4540000F5500000C2
:10899000F54E0000F54A0000F5480000F6440000DE
:1089A000F6420000F63E0000F63C0000F6380000FB
:1089B000F7360000F7320000F7300000F72C000017
:1089C000F72A0000F7260000F7220000F720000039
:1089D000F81C0000F81A0000F8160000F814000057
:1089E000F8100000F80E0000F80A0000F808000077
:1089F000F8040000F8020000F8020200F804020087
:108A0000F8080200F80A0200F80E0200F81002004E
:108A1000F8140200F8160200F81A0200F81C02000E
:108A2000F7200200F7220200F7260200F72A0200D0
:108A3000F72C0200F7300200F7320200F73602008E
:108A4000F6380200F63C0200F63E0200F642020052
:108A5000F6440200F5480200F54A0200F54E020015
:108A6000F5500200F4540200F4560200F45A0200D9
:108A7000F45C0200F3600200F3620200F36602009D
:108A8000F2680200F26C0200F26E0200F172020063
:108A9000F1740200F1780200F07A0200F07C02002A
:108AA000F0800200EF820200EF860200EE880200F2
:108AB000EE8C0200EE8E0200ED920200ED940200B8
:108AC000EC980200EC9A0200EB9E0200EBA0020080
:108AD000EAA20200EAA60200E9A80200E9AC02004C
:108AE000E8AE0200E8B20200E7B40200E7B6020016
:108AF000E6BA0200E5BC0200E5C00200E4C20200E2
:108B0000E4C40200E3C80200E2CA0200E2CE0200AE
:108B1000E1D00200E1D20200E0D60200DFD802007C
:108B2000DFDA0200DEDE0200DDE00200DCE402004B
:108B3000DCE60200DBE80200DAEC0200DAEE02001A
:108B4000D9F00200D8F40200D7F60200D7F80200EC
:108B5000D6FC0200D5FE0200D4000300D4020300BC
:108B6000D3060300D2080300D10A0300D00E03008D
:108B7000CF100300CF120300CE140300CD18030062
:108B8000CC1A0300CB1C0300CA1E0300C922030039
:108B9000C9240300C8260300C7280300C62C03000D
:108BA000C52E0300C4300300C3320300C2340300E7
:108BB000C1380300C03A0300BF3C0300BE3E0300BF
:108BC000BD400300BC420300BB460300BA4803009B
:108BD000B94A0300B84C0300B74E0300B650030077
:108BE000B5520300B4540300B3580300B25A030053
:108BF000B15C0300B05E0300AF600300AE6203002F
:108C0000AD640300AC660300AA680300A96A030010
:108C1000A86C0300A76E0300A6700300A5720300F2
:108C2000A4740300A3760300A1780300A07A0300D4
:108C30009F7C03009E7E03009D8003009C820300B6
:108C40009A8403009986030098880300978A03009A
:108C5000968C0300948E030093900300929203007D
:108C6000919203008F9403008E9603008D98030069
:108C70008C9A03008A9C0300899E0300889E03004F
:108C800087A0030085A2030084A4030083A6030039
:108C900081A8030080A803007FAA03007EAC030024
:108CA0007CAE03007BAE03007AB0030078B2030011
:108CB00077B4030076B4030074B6030073B80300FE
:108CC00072B8030070BA03006FBC03006DBE0300EE
:108CD0006CBE03006BC0030069C2030068C20300DE
:108CE00067C4030065C4030064C6030062C80300D0
:108CF00061C8030060CA03005ECA03005DCC0300C4
:108D00005BCE03005ACE030059D0030057D00300B6
:108D100056D2030054D2030053D4030051D40300AD
:108D200050D603004FD603004DD803004CD80300A3
:108D30004ADA030049DA030047DC030046DC03009B
:108D400044DC030043DE030041DE030040E0030097
:108D50003EE003003DE003003CE203003AE2030092
:108D600039E2030037E4030036E4030034E403008F
:108D700033E6030031E6030030E603002EE803008B
:108D80002DE803002BE803002AE8030028EA03008B
:108D900027EA030025EA030024EA030022EC03008B
:108DA00021EC03001FEC03001EEC03001CEC03008D
:108DB0001BEE030019EE030018EE030016EE03008D
:108DC00015EE030013EE030011EE030010EE030096
:108DD0000EF003000DF003000BF003000AF0030097
:108DE00008F0030007F0030005F0030004F003009F
:108DF00002F0030001F0030001F1030002F103009F
:108E000004F1030005F1030007F1030008F103007A
:108E10000AF103000BF103000DF103000EF1030052
:108E200010EF030011EF030013EF030015EF030031
:108E300016EF030018EF030019EF03001BEF030008
:108E40001CED03001EED03001FED030021ED0300E8
:108E500022ED030024EB030025EB030027EB0300C6
:108E600028EB03002AE903002BE903002DE90300A6
:108E70002EE9030030E7030031E7030033E7030086
:108E800034E5030036E5030037E5030039E303006A
:108E90003AE303003CE303003DE103003EE103004D
:108EA00040E1030041DF030043DF030044DD030032
:108EB00046DD030047DD030049DB03004ADB030016
:108EC0004CD903004DD903004FD7030050D70300FE
:108ED00051D5030053D5030054D3030056D30300E8
:108EE00057D1030059D103005ACF03005BCF0300D1
:108EF0005DCD03005ECB030060CB030061C90300BE
:108F000062C9030064C7030065C5030067C50300A9
:108F100068C3030069C303006BC103006CBF030097
:108F20006DBF03006FBD030070BB030072B9030087
:108F300073B9030074B7030076B5030077B5030077
:108F400078B303007AB103007BAF03007CAF03006A
:108F50007EAD03007FAB030080A9030081A903005D
:108F600083A7030084A5030085A3030087A1030052
:108F7000889F0300899F03008A9D03008C9B030048
:108F80008D9903008E9703008F9503009193030042
:108F90009293030093910300948F0300968D030036
:108FA000978B030098890300998703009A85030033
:108FB0009C8303009D8103009E7F03009F7D03002F
:108FC000A07B0300A1790300A3770300A47503002D
:108FD000A5730300A6710300A76F0300A86D03002B
:108FE000A96B0300AA690300AC670300AD65030029
:108FF000AE630300AF610300B05F0300B15D030027
:10900000B25B0300B3590300B4550300B55303002A
:10901000B6510300B74F0300B84D0300B94B03002E
:10902000BA490300BB470300BC430300BD41030032
:10903000BE3F0300BF3D0300C03B0300C139030036
:10904000C2350300C3330300C4310300C52F03003E
:10905000C62D0300C7290300C8270300C925030044
:10906000C9230300CA1F0300CB1D0300CC1B030050
:10907000CD190300CE150300CF130300CF11030059
:10908000D00F0300D10B0300D2090300D307030064
:10909000D4030300D4010300D5FF0200D6FD020073
:1090A000D7F90200D7F70200D8F50200D9F1020083
:1090B000DAEF0200DAED0200DBE90200DCE7020091
:1090C000DCE50200DDE10200DEDF0200DFDB0200A2
:1090D000DFD90200E0D70200E1D30200E1D10200B3
:1090E000E2CF0200E2CB0200E3C90200E4C50200C5
:1090F000E4C30200E5C10200E5BD0200E6BB0200D8
:10910000E7B70200E7B50200E8B30200E8AF0200EB
:10911000E9AD0200E9A90200EAA70200EAA3020001
:10912000EBA10200EB9F0200EC9B0200EC99020015
:10913000ED950200ED930200EE8F0200EE8D02002D
:10914000EE890200EF870200EF830200F081020047
:10915000F07D0200F07B0200F1790200F17502005F
:10916000F1730200F26F0200F26D0200F269020078
:10917000F3670200F3630200F3610200F45D020092
:10918000F45B0200F4570200F4550200F5510200AE
:10919000F54F0200F54B0200F5490200F6450200CA
:1091A000F6430200F63F0200F63D0200F6390200E7
:1091B000F7370200F7330200F7310200F72D020003
:1091C000F72B0200F7270200F7230200F721020025
:1091D000F81D0200F81B0200F8170200F815020043
:1091E000F8110200F80F0200F80B0200F809020063
:1091F000F8050200F8030200F8030000F80500007B
:10920000F8090000F80B0000F80F0000F81100004A
:10921000F8150000F8170000F81B0000F81D00000A
:10922000F7210000F7230000F7270000F72B0000CC
:10923000F72D0000F7310000F7330000F73700008A
:10924000F6390000F63D0000F63F0000F64300004E
:10925000F6450000F5490000F54B0000F54F000011
:10926000F5510000F4550000F4570000F45B0000D5
:10927000F45D0000F3610000F3630000F367000099
:10928000F2690000F26D0000F26F0000F17300005F
:10929000F1750000F1790000F07B0000F07D000026
:1092A000F0810000EF830000EF870000EE890000EE
:1092B000EE8D0000EE8F0000ED930000ED950000B4
:1092C000EC990000EC9B0000EB9F0000EBA100007C
:1092D000EAA30000EAA70000E9A90000E9AD000048
:1092E000E8AF0000E8B30000E7B50000E7B7000012
:1092F000E6BB0000E5BD0000E5C10000E4C30000DE
:10930000E4C50000E3C90000E2CB0000E2CF0000AA
:10931000E1D10000E1D30000E0D70000DFD9000078
:10932000DFDB0000DEDF0000DDE10000DCE5000047
:10933000DCE70000DBE90000DAED0000DAEF000016
:10934000D9F10000D8F50000D7F70000D7F90000E8
:10935000D6FD0000D5FF0000D4010100D4030100B8
:10936000D3070100D2090100D10B0100D00F010089
:10937000CF110100CF130100CE150100CD1901005E
:10938000CC1B0100CB1D0100CA1F0100C923010035
:10939000C9250100C8270100C7290100C62D010009
:1093A000C52F0100C4310100C3330100C2350100E3
:1093B000C1390100C03B0100BF3D0100BE3F0100BB
:1093C000BD410100BC430100BB470100BA49010097
:1093D000B94B0100B84D0100B74F0100B651010073
:1093E000B5530100B4550100B3590100B25B01004F
:1093F000B15D0100B05F0100AF610100AE6301002B
:10940000AD650100AC670100AA690100A96B01000C
:10941000A86D0100A76F0100A6710100A5730100EE
:10942000A4750100A3770100A1790100A07B0100D0
:109430009F7D01009E7F01009D8101009C830100B2
:109440009A8501009987010098890100978B010096
:10945000968D0100948F0100939101009293010079
:10946000919301008F9501008E9701008D99010065
:109470008C9B01008A9D0100899F0100889F01004B
:1094800087A1010085A3010084A5010083A7010035
:1094900081A9010080A901007FAB01007EAD010020
:1094A0007CAF01007BAF01007AB1010078B301000D
:1094B00077B5010076B5010074B7010073B90100FA
:1094C00072B9010070BB01006FBD01006DBF0100EA
:1094D0006CBF01006BC1010069C3010068C30100DA
:1094E00067C5010065C5010064C7010062C90100CC
:1094F00061C9010060CB01005ECB01005DCD0100C0
:109500005BCF01005ACF010059D1010057D10100B2
:1095100056D3010054D3010053D5010051D50100A9
:1095200050D701004FD701004DD901004CD901009F
:109530004ADB010049DB010047DD010046DD010097
:1095400044DD010043DF010041DF010040E1010093
:109550003EE101003DE101003CE301003AE301008E
:1095600039E3010037E5010036E5010034E501008B
:1095700033E7010031E7010030E701002EE9010087
:109580002DE901002BE901002AE9010028EB010087
:1095900027EB010025EB010024EB010022ED010087
:1095A00021ED01001FED01001EED01001CED010089
:1095B0001BEF010019EF010018EF010016EF010089
:1095C00015EF010013EF010011EF010010EF010092
:1095D0000EF101000DF101000BF101000AF1010093
:1095E00008F1010007F1010005F1010004F101009B
:1095F00002F1010001F10100E0C0020060C00300BF
:1096000060C10300E0C10200E0C1000060C10100D0
:1096100060C00100E0C00000E0C0020060C00300C4
:1096200060C10300E0C10200E0C1000060C10100B0
:1096300060C00100E0C00000B4690100B46801002E
:10964000B4680300B4690300B4690100B4680100A0
:10965000B4680300B4690300B4690100B468010090
:10966000B4680300B4690300B4690100B468010080
:10967000B4680300B4690300E803000000040000BC
:10968000D007000000080000C4090000A00F00007F
:109690000010000088130000401F000000200000A0
:1096A0001027000000400000204E0000007D000058
:1096B00000800000409C000000000100FFFFFFFF51
:1096C000313331315631313100544D434D2D313329
:1096D000313120287669727475616C20434F4D29B1
:1096E000005472696E616D6963204D6F74696F6EAD
:1096F00020436F6E74726F6C00544D4331333131BF
:109700000056435020436F6E6669670056435020F1
:10971000496E74657266616365004142530052454B
:109720004C00434F4F524400535441525400535441
:109730004F50005354415455530000004300000063
:109740008801002000202020202020202020282800
:1097500028282820202020202020202020202020F1
:109760002020202020881010101010101010101031
:109770001010101010040404040404040404041061
:1097800010101010101041414141414101010101EF
:1097900001010101010101010101010101010101B9
:1097A00010101010101042424242424202020202C5
:1097B0000202020202020202020202020202020289
:1097C0001010101020000000000000000000000039
:1097D0000000000000000000000000000000000089
:1097E0000000000000000000000000000000000079
:1097F0000000000000000000000000000000000069
:109800000000000000000000000000000000000058
:109810000000000000000000000000000000000048
:109820000000000000000000000000000000000038
:109830000000000000000000000000000000000028
:1098400000000000000000006C6F670000000000D6
:10985000F8B500BFF8BC08BC9E467047F8B500BF1D
:08986000F8BC08BC9E467047ED
:0898680024DAFF7F010000007B
:08987000097A0108AD8100082E
:0498780089810008DA
:10987C00C096010800010200000800000100000071
:10988C0002000000000000000000000000000000CA
:10989C0000000000000000000000000000000000BC
:1098AC0000000000000000000000000000000000AC
:1098BC00000000001201000202000040D0162C072C
:1098CC0000020102030104030904000000C20100AC
:1098DC0000000800D7AA0008E5AA000841AB000860
:1098EC0025AB00085DAB000879AB000895AB000810
:1098FC00C9AA0008CBAA0008CDAA0008CFAA000864
:10990C00D1AA0008D3AA0008D5AA00080A060002AA
:10991C000000004001000000F1AA0008F5AA0008B0
:10992C00B1AB0008F9AA0008FDAA0008000E270731
:10993C0000000000000000000102030406070809F3
:10994C0000000000010203040102030406070809D9
:10995C00E4000020694B0108B54A01086B4A010874
:10996C00DB4901083D4A0108BF490108A949010822
:10997C00EB490108F9490108074A01081D4A010889
:10998C00FF00000009024300020100C0320904007C
:10999C000001020201000524001001052401000150
:1099AC00042402020524060001070582030800FFB7
:1099BC0009040100020A0000000705010240000032
:1099CC0007058102400000000D4E0108E54D01081D
:1099DC00254D010800000000414C0108614E0108B2
:1099EC00F54C01087D4C010800000000000000004F
:1099FC00714C0108000000000000000074040020FD
:109A0C00DC040020440500200000000000000000E1
:109A1C00000000000000000000000000000000003A
:109A2C000000000000000000000000003C9701084E
:109A3C00000000000000000000000000000000001A
:109A4C00000000000000000000000000000000000A
:109A5C0000000000000000000000000000000000FA
:109A6C0000000000000000000000000000000000EA
:109A7C0000000000000000000000000000000000DA
:109A8C0000000000000000000000000000000000CA
:109A9C0000000000000000000000000000000000BA
:109AAC0001000000000000000E33CDAB34126DE657
:109ABC00ECDE05000B0000000000000000000000C0
:109ACC00000000000000000000000000000000008A
:109ADC00000000000000000000000000000000007A
:109AEC00000000000000000000000000000000006A
:109AFC00000000000000000000000000000000005A
:0C9E2C008801002044970108010000009C
:04000005080177BDBA
:00000001FF
